:100000000C94E7270C94E12A0C940C2B0C94372BBE
:100010000C94622B0C948D2B0C94B82B0C94E32B2A
:100020000C940E2C0C9418280C9418280C94182856
:100030000C9418280C9418280C9418280C94182840
:100040000C9418280C940DAD0C9418280C941828B6
:100050000C9418280C9418280C94DF9E0C941A28E1
:100060000C9418280C94488B0C94F48B0C9418283E
:100070000C9418280C9418280C9418280C94182800
:100080000C9418280C9418280C9418280C941828F0
:100090000C9418280C9418280C9418280C941828E0
:1000A0000C9418280C9418280C9418280C941828D0
:1000B0000C9418280C9418280C9418280C941828C0
:1000C0000C9418280C9418280C9418280C941828B0
:1000D0000C9418280C9418280C9418280C941828A0
:1000E0000C94182857295C2961296B297529EE2958
:1000F0007F2987298F299929A329AD29BC29C629B8
:10010000EE29D029DA29E429122A152A042A082AF4
:100110000E2A4C2A192A1D2A232A272A2B2A312A59
:10012000352A392A4C2A3F2A432A472ABE5AA45A3A
:10013000A15AA75AAA5AAD5AB95AB05ACA5AB35A6A
:10014000B65A7B8B818B928B9D8BA58BBA8BA98B9F
:10015000BA8BAD8BB18BBA8BB78B5F985F98669873
:10016000669866986D986D986D987A98749874985A
:100170007498869F929F969FC09FCB9FA99FAD9F8B
:10018000769F084AD73B3BCE016E84BCBFFDC12F92
:100190003D6C74319ABD56833DDA3D00C77F11BE78
:1001A000D9E4BB4C3E916BAAAABE000000803F057B
:1001B000A84CCDB2D44EB93836A9020C50B99186AC
:1001C00088083CA6AAAA2ABE000000803F000D9421
:1001D0003F100D9416134E414E494E495459494E05
:1001E00046CDCCCC3D0AD7233C17B7D13877CC2BA2
:1001F000329595E6241FB14F0A000020410000C847
:100200004200401C4620BCBE4CCA1B0E5AAEC59DC7
:100210007400000A0B02090C0D0E0807030401000C
:1002200000000000000000000000000000000000CE
:10023000000000000000000000000000001211108B
:1002400000000000000000000000000000000000AE
:10025000000000000000000102102020080810200B
:100260004010204080020102010804020101020442
:100270000810204080804020100804020180040201
:100280000180402010080402010804020101020458
:100290000810204080010204081020408005050558
:1002A00005070508080808020202020A0A080804ED
:1002B000040404010101010101010103030303031B
:1002C000030303040707070C0C0C0C0C0C0C0C02AA
:1002D00002020206060606060606060B0B0B0B0BB1
:1002E0000B0B0B000020002300260029002C002F00
:1002F0000032000001000003010601090100002294
:1003000000250028002B002E0031003400020100DF
:1003100000050108010B0100002100240027002A2C
:10032000002D003000330001010000040107010A24
:100330000101060D00FE09016602D620FFFE0BFE3C
:100340000AFE0D0060221969808080808080800014
:1003500080183363A0A0A00357675050F850F8509E
:10036000500259692078A0A0702828F0200259690D
:1003700048A85010204050A89002586840A0A040C3
:10038000A0989068281363808080113B6B204040C8
:100390008080808080404020113B6B804040202046
:1003A00020202040408006556520A870A8200455D4
:1003B000652020F82020113363604080065161F8E9
:1003C00011336340E0400259690808101020404092
:1003D0008080025969205088888888885020025976
:1003E000692060A02020202020F8025969708888A8
:1003F0000810204080F8025969F808102070080899
:100400008870025969101030505090F8101002593D
:1004100069F88080B0C808088870025969708880BF
:1004200080F088888870025969F8081010202040F0
:10043000404002596970888888708888887002599D
:100440006970888888780808887011386840E040AA
:10045000000040E04011386840E04000006040800B
:10046000025969081020408040201008045464F8A4
:100470000000F802596980402010081020408002D6
:1004800059697088880810202000200259697088F6
:100490008898A8A8B080780259692050888888F880
:1004A000888888025969F048484870484848F002EE
:1004B0005969708880808080808870025969F0480E
:1004C000484848484848F0025969F8808080F080E0
:1004D0008080F8025969F8808080F08080808002F6
:1004E00059697088808080988888700259698888E6
:1004F0008888F888888888123969E0404040404000
:100500004040E0025969381010101010109060023D
:100510005969888890A0C0A0908888025969808015
:10052000808080808080F80259698888D8A8A8884F
:1005300088888802596988C8C8A8A89898888802B5
:100540005969708888888888888870025969F08815
:100550008888F080808080015A6A708888888888BE
:1005600088A87008025969F0888888F0A090888867
:10057000025969708880807008088870025969F88B
:1005800020202020202020200259698888888888FF
:10059000888888700259698888888850505020203F
:1005A00002596988888888A8A8A8A850025969882B
:1005B00088505020505088880259698888505020AF
:1005C00020202020025969F808101020404080F8AF
:1005D000113B6BE0808080808080808080E00259C9
:1005E00069808040402010100808113B6BE02020FB
:1005F00020202020202020E0085363205088015133
:1006000061F82A22628040025666700878889868ED
:10061000025969808080F088888888F00256667068
:1006200088808088700259690808087888888888D6
:10063000780256667088F8808870025969304840A0
:1006400040F04040404000586870888888780888AA
:1006500070025969808080B0C8888888881238689C
:100660004000C040404040E0004A6A100030101096
:10067000101090906002596980808090A0C0A09076
:1006800088123969C040404040404040E002566610
:10069000D0A8A8A8A888025666B0C888888888020A
:1006A0005666708888888870005868F0888888F056
:1006B0008080800058687888888878080808025602
:1006C00066B0C8808080800256667088601088702E
:1006D0000258684040F040404048300256668888E2
:1006E0008888986802566688888850502002566626
:1006F0008888A8A8A85002566688502020508800F4
:1007000058688888889868088870025666F81020AB
:100710004080F8015B6B1820202020C02020202082
:1007200018221969808080808080808080015B6BC6
:10073000C0202020201820202020C008536348A873
:1007400090FFFFFFFFFFFFFFFFFFFFFFFFFFFFFF28
:10075000FFFFFFFFFFFFFFFFFFFFFFFFFFFFFFFFA9
:10076000FFFF0D00602219698000808080808080FA
:10077000800358682070A8A0A0A870200259693092
:10078000484040E0404048B0035666887050507082
:100790008802596988885050F820F8202022196969
:1007A000808080800080808080124A6A60908060B3
:1007B0009090601090601A3262A0A003596970880E
:1007C000A8D8C8D8A88870045767700878887800B7
:1007D000F80356662850A0A05028045363F8080870
:1007E000163161E00359697088E8D8D8E8D8887074
:1007F0000A5161F8174464609090600357672020A5
:10080000F8202000F807356540A02040E007356556
:1008100040A04020C02A2262408000586888888812
:100820008898E8808002596978E8E8E8E86828282C
:1008300028262161C0202262408007356540C040E3
:1008400040E0045767708888887000F8035666A0F7
:1008500050282850A0025A6A40C04040E00818289A
:100860003808025A6A40C04040E010280810380298
:100870005A6A40A04020A048182838080259692028
:100880000020204080888870025A6A402000205052
:100890008888F88888025A6A10200020508888F8D2
:1008A0008888025A6A30480020508888F888880270
:1008B0005A6A28500020508888F88888025A6A505E
:1008C000500020508888F88888025A6A20502020DA
:1008D000508888F8888802596958A0A0A0B0E0A084
:1008E000A0B8005B6B70888080808080887020401A
:1008F000025A6A402000F88080F08080F8025A6A2C
:10090000102000F88080F08080F8025A6A30480099
:10091000F88080F08080F8025A6A505000F8808099
:10092000F08080F8123A6A804000E0404040404049
:10093000E0123A6A204000E04040404040E0124A65
:100940006A609000E04040404040E0123A6AA0A057
:1009500000E04040404040E0025969F0484848E823
:10096000484848F0025A6A2850008888C8A89888E1
:1009700088025A6A40200070888888888870025AE5
:100980006A10200070888888888870025A6A304807
:100990000070888888888870025A6A285000708899
:1009A0008888888870025A6A5050007088888888C1
:1009B00088700355658850205088015B6B087098DB
:1009C00098A8A8A8C8C87080025A6A4020008888E1
:1009D0008888888870025A6A1020008888888888E9
:1009E0008870025A6A30480088888888888870022F
:1009F0005A6A50500088888888888870025A6A101D
:100A000020008888502020202002596980F08888A2
:100A100088F0808080025969609090A0A0908888BA
:100A2000B0025969402000700878889868025969B6
:100A30001020007008788898680259693048007062
:100A40000878889868025969285000700878889852
:100A500068025969505000700878889868025A6A8C
:100A600030483000700878889868025666702870A0
:100A7000A0A8500058687088808088702040025973
:100A8000694020007088F880887002596910200041
:100A90007088F88088700259693048007088F88042
:100AA00088700259695050007088F8808870123937
:100AB00069804000C040404040E012396920400059
:100AC000C040404040E0124969609000C040404052
:100AD00040E0123969A0A000C040404040E0025A06
:100AE0006A50206010708888888870025969285080
:100AF00000B0C888888888025969402000708888BA
:100B0000888870025969102000708888888870026F
:100B1000596930480070888888887002596928505F
:100B200000708888888870025969505000708888E1
:100B3000888870035767202000F80020200158683B
:100B4000087098A8A8C87080025969402000888859
:100B50008888986802596910200088888888986871
:100B60000259693048008888888898680259695015
:100B70005000888888889868005B6B1020008888FF
:100B8000889868088870005A6A8080B0C88888C8C9
:100B9000B08080005B6B5050008888889868088817
:100BA0007001050700FE0500FB01F220FFFE05FEB7
:100BB00005FE02004002152580808000800532423B
:100BC000A0A002556550F850F8500146562070C05C
:100BD00030E0200255659010204048025565608045
:100BE0006890680512228080022535408080804010
:100BF0000225358040404080043343A040A00333A9
:100C00004340E0400122324080043141E0021121A2
:100C100080025565081020408002455560909090F4
:100C200060022535C040404040024555E0106080DC
:100C3000F0024555E0106010E00245552060A0F03C
:100C400020024555F080E010E00245556080E090BC
:100C500060024555F010204040024555609060907C
:100C6000600245556090701060031323800080027D
:100C700014248000808002354520408040200333CA
:100C800043E000E00235458040204080024555E0C9
:100C9000106000400255657088B8A8700245556024
:100CA0009090F090024555E090E090E0023545606C
:100CB00080808060024555E0909090E0023545E0EC
:100CC00080E080E0023545E080E08080024555709C
:100CD00080B090700245559090F09090023545E0BC
:100CE000404040E00245553010109060024555905C
:100CF000A0C0A09002354580808080E002556588C4
:100D0000D8A8888802455590D0B09090024555608B
:100D100090909060024555E09090E08001465660CA
:100D20009090906010024555E09090E090024555FB
:100D300070806010E0023545E0404040400245557B
:100D400090909090600245559090A0A0400255650B
:100D500088A8A8A8500245559090609090024555EB
:100D60009090701060023545E0204080E00225350B
:100D7000C0808080C0025565804020100802253563
:100D8000C0404040C005324240A0024151F005221F
:100D90003280400244547090907002455580E0903B
:100DA00090E002344460808060024555107090905D
:100DB0007002445460B0C0600235452040E04040BD
:100DC00000465670909070106002455580E09090FB
:100DD0009002152580008080800027374000404029
:100DE0004040800245558090A0E09002152580800B
:100DF000808080025464F0A8A8A8024454E0909037
:100E00009002445460909060004656E09090E080DC
:100E100080004656709090701010023444A0C0803C
:100E20008002445470C030E002354540E04040202C
:100E3000024454909090700244549090A040025408
:100E400064A8A85050023444A04040A000465690E8
:100E50009090701060024454F02040F002354560DC
:100E6000408040600215258080808080023545C02A
:100E7000402040C005425250A0FFFFFFFFFFFFFF90
:100E8000FFFFFFFFFFFFFFFFFFFFFFFFFFFFFFFF72
:100E9000FFFFFFFFFFFFFFFFFFFF020040FFFFFF1D
:100EA000FFFFFFFFFFFFFFFFFFFFFFFFFFFFFFFF52
:100EB000FFFFFFFFFFFFFFFFFFFFFFFFFFFFFFFF42
:100EC000FFFFFFFFFFFFFFFFFFFFFFFFFFFFFFFF32
:100ED000FFFFFFFFFFFFFFFFFFFFFFFFFFFFFFFF22
:100EE000FFFFFFFFFFFFFFFFFFFFFFFFFFFFFFFF12
:100EF000FFFFFFFFFFFFFFFFFFFFFFFF01050800F0
:100F0000FF060121023520FFFF07FF06FF09005001
:100F1000221656808080800080153353A0A0A00246
:100F200057575050F850F850500257572070A07043
:100F300028702013355580A040A02002475740A0BC
:100F4000A040A0A0502513538080801226564080D8
:100F500080808040122656804040404080024555A7
:100F60009060F060900255552020F82020113353F6
:100F7000604080044151F011335340E04002465636
:100F800010102040808012365640A0A0A0A0401231
:100F9000365640C0404040E00246566090106080A7
:100FA000F0024656F020601090600246562060A085
:100FB000F02020024656F080E01090600246566015
:100FC00080E0909060024656F0102020404002469B
:100FD00056609060909060024656609090701060ED
:100FE000122555C0C000C0C0113656606000604078
:100FF00080123656204080804020034353F000F09A
:1010000012365680402020408012365640A02040A4
:101010000040015858304898A8A8904030024656E1
:10102000609090F09090024656E090E09090E00240
:101030004656609080809060024656E09090909076
:10104000E0024656F080E08080F0024656F080E0F4
:10105000808080024656609080B090600246569034
:1010600090F0909090123656E040404040E00246AA
:101070005670202020A04002465690A0C0A0A0900C
:101080000246568080808080F002465690F0F090B4
:10109000909002465690D0F0B0B0900246566090C4
:1010A00090909060024656E09090E0808001475713
:1010B000609090D0B06010024656E09090E0909022
:1010C000024656609040209060123656E040404004
:1010D0004040024656909090909060024656909004
:1010E00090906060024656909090F0F090024656C4
:1010F0009090606090900256568888502020200280
:101100004656F010204080F0123656E080808080F5
:10111000E0024656808040201010123656E0202013
:101120002020E016325240A0014151F01622528098
:1011300040024454709090700246568080E0909037
:10114000E012345460808060024656101070909017
:101150007002445460B0C060024656205040E040E7
:101160004001455560907010600246568080E090C6
:1011700090901236564000C04040E0113757200092
:10118000202020A040024656808090E090901236A9
:1011900056C040404040E0025454D0A8A8A80244A1
:1011A00054E090909002445460909060014555E066
:1011B00090E080800145557090701010024454A05A
:1011C000D0808012345460C020C00246564040E0B7
:1011D00040502002445490909070123454A0A0A02B
:1011E0004002545488A8A850024454906060900172
:1011F00045559090709060024454F02040F00247B2
:1012000057304020C0204030221656808080808099
:1012100080024757C02040304020C006425250A0B4
:10122000FFFFFFFFFFFFFFFFFFFFFFFFFFFFFFFFCE
:10123000FFFFFFFFFFFFFFFFFFFFFFFFFFFFFFFFBE
:10124000FF0900502216568000808080800146569B
:101250002070A0A070200246562050E04050A0020E
:10126000555588705070880256568850F820F820DE
:10127000221757808080008080800247577080E06E
:10128000907010E0173151A002565670A8C8C8A837
:101290007014355560A06000E003435350A0501215
:1012A0003353E02020143151E002565670E8D8E85C
:1012B000D870173151E015335340A04012355540D6
:1012C000E04000E014355540A02040E0143555C002
:1012D00020C020C01622524080014555909090E0D9
:1012E0008002565678E8E868282824115180112297
:1012F00052408014355540C04040E014355540A060
:101300004000E0034353A050A0024757808080A0D4
:1013100060F0200247578080A0D01020700247570D
:1013200080408060A0F02012365640004080A040EF
:1013300002475740206090F090900247572040604D
:1013400090F0909002475760906090F09090024724
:101350005750A06090F0909002475790006090F036
:10136000909002475760906090F0909002465670BF
:10137000A0A0F0A0B001475760908080906040022C
:1013800047574020F080E080F00247572040F0802F
:10139000E080F00247576090F080E080F00247570D
:1013A0009000F080E080F01237578040E0404040ED
:1013B000E01237572040E0404040E012375740A04D
:1013C000E0404040E0123757A000E0404040E002DB
:1013D00056567048E848487002475750A090D0B021
:1013E00090900247574020609090906002475720AD
:1013F000406090909060024757609060909090603D
:1014000002475750A060909090600247579000604C
:1014100090909060123353A040A002465670B0B036
:10142000D0D0E002475740209090909060024757FC
:1014300020409090909060024757609090909090DC
:10144000600247579000909090906002575710208C
:10145000885020202002465680E09090E08002468E
:10146000566090A0A090A002475740200070909036
:1014700070024757204000709090700247572050EC
:10148000007090907002475750A0007090907002CA
:101490004656500070909070024757609060709070
:1014A0009070025454F068B07811355560808060B7
:1014B0004002475740200060B0C0600247572040BC
:1014C0000060B0C06002475760900060B0C060022A
:1014D0004656500060B0C060123757804000C04090
:1014E00040E0123757204000C04040E012375740DC
:1014F000A000C04040E0123656A000C04040E002CC
:101500004757A040A01070906002475750A000E0DD
:10151000909090024757402000609090600247579B
:10152000204000609090600247576090006090906B
:101530006002475750A000609090600246569000AD
:10154000609090601235554000E0004002445470B5
:10155000B0D0E0024757402000909090700247576B
:1015600020400090909070024757609000909090BB
:1015700070024656900090909070014858204000AC
:1015800090907090600147578080E090E0808001EB
:1015900047579000909070906025753A25303275CD
:1015A00000253032753A25303275002575642025C6
:1015B0003032753A2530327500871657169F166FF0
:1015C000163FFFF038007031863023871027879050
:1015D0002F87D02F03D020301020781020781020B3
:1015E00030102F03D02F87D0278790238710318684
:1015F000303800703FFFF03FFFF038007030FC30B3
:1016000020FC102078102030102C00D02E31D02F4C
:101610007BD02F7BD02E31D02C00D02030102078E2
:101620001020FC1030FC303800703FFFF0041040F8
:1016300002082002082004104008208010410010F9
:1016400041000820800410400000001FFFF81FFF29
:10165000F81FFFF81FFFF81FE02010231024901040
:10166000A011202210241037B00840048003001F6E
:10167000E03FF03CF03B701F601EE03DF03BF03877
:10168000700FC0078003001FE020102110231015E9
:101690002011202110211031300840048003001F48
:1016A000E03FF03EF03CF01AE01EE03EF03EF03E3F
:1016B000F00FC0078003004572723A2075746638D7
:1016C00020666F6E74206E6F7420696E6974696134
:1016D0006C697A65642E004572723A2075746638BA
:1016E00020666F6E74206E6F7420696E6974696114
:1016F0006C697A65642E004572723A20757466389A
:1017000020666F6E74206E6F7420696E69746961F3
:101710006C697A65642E00506C6561736520726532
:10172000736574005052494E5445522048414C5400
:1017300045440000060C00FE07022603BC017FFEA4
:1017400008FE08FE05080806000040F0C8888898D2
:101750007810050808060000C0F88888888888F88E
:101760000505050600012030F830200508080600B0
:10177000002070F820202020E00509090600FF2045
:1017800070A8A8B888887020050606060001E08CBD
:10179000EA8C8A0A0509090600FFF8A88888888863
:1017A00088A8F8050A0A0600FE205050505088A864
:1017B000A8887003030306000340A040FFFFFFFF5B
:1017C000FFFFFFFFFFFFFFFFFFFFFFFFFFFFFFFF29
:1017D000FFFF0000000605FF0107070602008080EA
:1017E0008080800080030303060105A0A0A00506F9
:1017F0000606000050F85050F8500509090600FF91
:101800002070A8A07028A87020050707060000C84F
:10181000C8102040989805070706000040A0A04087
:10182000A890680103030602058080800309090669
:1018300001FF2040408080804040200309090601CC
:10184000FF80404020202040408005070706000020
:1018500020A8702070A8200505050600012020F8AA
:1018600020200203030601FFC0408005010106009D
:1018700003F8020202060100C0C0050707060000C7
:101880000810102040408005070706000070889867
:10189000A8C8887003070706010040C040404040C8
:1018A000E0050707060000708808102040F80507CB
:1018B00007060000F80810300888700507070600C2
:1018C0000010305090F81010050707060000F8804F
:1018D000F008088870050707060000304080F0888F
:1018E0008870050707060000F80810102020200562
:1018F000070706000070888870888870050707064B
:10190000000070888878081060020505060100C094
:10191000C000C0C00206060601FFC0C000C0408073
:101920000305050601012040804020050303060051
:1019300002F800F8030505060101804020408005FB
:101940000707060000708810202000200507070602
:1019500000007088B8A8B8807005070706000070FE
:101960008888F8888888050707060000F0484870CE
:101970004848F0050707060000708880808088705E
:10198000050707060000F04848484848F0050707E3
:10199000060000F88080F08080F805070706000048
:1019A000F88080F08080800507070600007088803E
:1019B00080988870050707060000888888F888885E
:1019C00088030707060100E04040404040E005076B
:1019D0000706000038101010109060050707060079
:1019E000008890A0C0A090880507070600008080AE
:1019F00080808080F805070706000088D8A88888BE
:101A000088880507070600008888C8A89888880580
:101A10000707060000708888888888700507070611
:101A20000000F08888F080808005070706000070BD
:101A3000888888A89068050707060000F08888F065
:101A4000A0908805070706000070888070088870DD
:101A5000050707060000F8202020202020050707A2
:101A600006000088888888888870050707060000B7
:101A700088888888505020050707060000888888D5
:101A800088A8A850050707060000888850205088BD
:101A900088050707060000888850202020200507B9
:101AA00007060000F80810204080F8030909060125
:101AB000FFE080808080808080E0050707060000CE
:101AC000804040201010080309090601FFE0202093
:101AD0002020202020E00503030600052050880573
:101AE00001010600FEF803030306010580402005FE
:101AF00005050600007008788878050707060000CD
:101B00008080F0888888F0050505060000708080D8
:101B10008870050707060000080878888888780517
:101B200005050600007088F08070050707060000B4
:101B3000304840E04040400507070600FE708888B6
:101B4000887808700507070600008080F08888887C
:101B5000880307070601004000C0404040E0040938
:101B6000090601FE100030101010109060050707E4
:101B700006000080808890E0908803070706010037
:101B8000C04040404040E0050505060000D0A8A840
:101B9000A8A8050505060000B0C8888888050505C1
:101BA00006000070888888700507070600FEF08828
:101BB0008888F080800507070600FE788888887886
:101BC0000808050505060000B0C8808080050505E9
:101BD00006000078807008F0050707060000202046
:101BE000F8202020180505050600008888889868D8
:101BF00005050506000088888850200505050600B3
:101C0000008888A8A85005050506000088502050C7
:101C1000880507070600FE88888850204080050553
:101C200005060000F8102040F80309090601FF200E
:101C300040404080404040200109090602FF80806A
:101C4000808080808080800309090601FF804040F9
:101C500040204040408005030306000248A890FF52
:101C60001FFFFFFFFFFFFF600000000001FF4000BB
:101C700000000000FF8000000000007F83CF000014
:101C80000C303F87FF80000C301F867980000C00ED
:101C90000F8C30C7838C30E78C30CFC7CC31F38CBE
:101CA00030DCECEC33B98C30D86C6C33198C30D020
:101CB0006C0C33198C30D86C0C33198C30DC6C0EF6
:101CC0003B198C30CF7C079F198C30C77C038F1950
:101CD00040000000000002600000000000061FFF3E
:101CE000FFFFFFFFF8000000000000000000000000
:101CF00000000000000000000000000000000000E4
:101D000000000000000000000C00000000000000C7
:101D10000C000000000000001200000000000000A5
:101D2000230000000000000021000000000000006F
:101D30004C800000000000005E80000000000000F9
:101D40009240000000000000A140000000000001DF
:101D500021200000000000027F900000000000022F
:101D60000010000000000007FFF800000000000461
:101D70000008000000000008000400000000000847
:101D8000000600000000001000020000000000300B
:101D90001E010000000000207F81000000000041C3
:101DA000FFE0800000000043FCF08000000000879E
:101DB0003B7840000000018EDBFC60000000010F5A
:101DC000EBCC20000000021FEDB610000000021F47
:101DD000DEB6100000000439CD7F08000000043694
:101DE000E0FF08000000087EC0BB84000000187FF0
:101DF000005D86000000107FC0ED82000000203CE6
:101E0000C07301000000203B337F01000000701B05
:101E1000E77E03800000C81DEEDE04C00000880FCE
:101E2000DEDC04400001240FDF3C0920000126070E
:101E3000DBF8192000027203E7F013900002510151
:101E4000FFE02290000489007F802448000904807C
:101E50001E004824000BFE400000DFF4001000408C
:101E600000008002001FFFFFFFFFFFFE00000000D8
:101E70000000000000000000000000000000000062
:101E800000000000001022103C3C0E1F0010221029
:101E90000422110400102210082211040010221044
:101EA000083C11040010221010221104001022100E
:101EB00020221104001E1C1E3C3C0E0400000000E9
:101EC0000000000000000000000000000000000012
:101ED0000000000000000000000000000000000002
:101EE00000000000000000000000000000000000F2
:101EF00000000000000000000000000000000000E2
:101F000000000000000000000000000000000000D1
:101F100000000000000000000000000000000000C1
:101F200000000000060900FE06018902FE20FFFEF7
:101F300007FE06FE00000006000701060606020076
:101F4000808080800080030303060103A0A0A00519
:101F500007070600FF5050F850F8505005090906D1
:101F600000FE2070A8A07028A870200608080600AF
:101F7000FF40A84810204854080507070600FF60E6
:101F800090906098906801030306020380808002AD
:101F900007070602FF408080808080400207070616
:101FA00002FF804040404040800505050600008853
:101FB00050F850880505050600002020F820200272
:101FC00004040602FEC0404080050101060002F83C
:101FD000020202060200C0C004060606010010103C
:101FE000204080800406060601006090909090607A
:101FF00003060606010040C0404040E00406060615
:1020000001006090102040F0040606060100F02058
:10201000601010E005060606000010305090F81021
:10202000040606060100F080E01010E00406060633
:1020300001006080E0909060040606060100F01048
:1020400010204040040606060100609060909060F9
:1020500004060606010060909070106002050506F7
:102060000200C0C000C0C00207070602FEC0C000D8
:10207000C040408005050506000018608060180516
:102080000303060001F800F8050505060000C0304E
:102090000830C0040707060100609010604000404F
:1020A0000506060600007090A8B0807005060606BA
:1020B0000000205088F88888050606060000F08891
:1020C000F08888F004060606010060908080906029
:1020D000040606060100E090909090E004060606D3
:1020E0000100F080E08080F0040606060100F08028
:1020F000E0808080040606060100609080B0906059
:102100000406060601009090F090909003060606E3
:102110000100E040404040E005060606000038109F
:102120001010906004060606010090A0C0A09090D8
:102130000406060601008080808080F00506060601
:10214000000088D8A8A8888804060606010090D058
:10215000B090909005060606000070888888887008
:10216000040606060100E09090E080800407070660
:1021700001FF609090D0B06010040606060100E0F8
:102180009090E09090040606060100609040209038
:1021900060050606060000F8202020202004060620
:1021A0000601009090909090600406060601009051
:1021B0009090F060600506060600008888A8A8D800
:1021C000880506060600008850202050880506066F
:1021D000060000888850202020040606060100F032
:1021E00010204080F0030606060100E08080808019
:1021F000E004060606010080804020101003060659
:10220000060100E020202020E00503030600032053
:1022100050880501010600FEF80202020602048051
:102220004004040406010070909070040606060144
:10223000008080E09090E00404040601007080803B
:1022400070040606060100101070909070040404DB
:1022500006010060B0C07004060606010020504070
:10226000E040400406060601FE6090907010600495
:1022700006060601008080E09090900306060601A5
:10228000004000C04040E00308080601FE20006056
:10229000202020A0400406060601008080A0C0A0E7
:1022A00090030606060100C040404040E0050404DB
:1022B000060000D0A8A888040404060100E090905D
:1022C0009004040406010060909060040606060174
:1022D000FEE09090E080800406060601FE7090907B
:1022E000701010040404060100A0D08080040404CF
:1022F00006010070C030E00406060601004040E020
:1023000040502004040406010090909070040404DE
:102310000601009090606005040406000088A8A8EB
:102320005004040406010090606090040606060153
:10233000FE909090709060040404060100F020402C
:10234000F0030707060100204040804040200107BD
:10235000070602FF808080808080800307070601D7
:10236000008040402040408004020206010350A04B
:10237000FFFFFFFFFFFFFFFFFFFFFFFFFFFFFFFF6D
:10238000FFFFFFFFFFFFFFFFFFFFFFFFFFFFFFFF5D
:10239000FF0000000600070106060602008000801C
:1023A0008080800406060601FF2070A0A070200532
:1023B00007070600FF304840F04040F805050506D5
:1023C0000000A8508850A80506060600008850F8AE
:1023D00020F8200107070602FF80808000808080AF
:1023E0000407070601FF708060906010E0030101A0
:1023F000060105A0060707060000788494A49484CB
:102400007803050506010160A06000E005050506EA
:1024100000002850A05028040303060100F010100B
:10242000040101060102F00607070600007884B4E3
:10243000A4A48478040101060105F0040303060145
:10244000026090600507070600FF2020F8202000AA
:10245000F803050506010140A02040E0030505063C
:102460000101C0204020C002020206020440800494
:1024700005050601FF9090B0D08005060606000015
:1024800078E8E868282801010106020280020202B9
:102490000602FE408003050506010140C04040E001
:1024A00003050506010140A04000E0050505060002
:1024B00000A0502850A00508080600FF40C040506A
:1024C000703078100508080600FF40C040506808CA
:1024D00010380508080600FFC0204030F0307810A2
:1024E00004070706010020002060809060050707B0
:1024F000060000402020507088880507070600006D
:102500001020205070888805070706000020502002
:1025100050708888050707060000285020507088F2
:1025200088050707060000500020507088880507BE
:102530000706000020502050708888050606060017
:102540000078A0F0A0A0B80408080601FE60908002
:1025500080906020400407070601004020F080E0E2
:1025600080F00407070601002040F080E080F004BE
:1025700007070601002050F080E080F004070706FE
:1025800001005000F080E080F003070706010080A2
:1025900040E0404040E00307070601002040E040E3
:1025A0004040E003070706010040A0E0404040E053
:1025B000030707060100A000E0404040E0050606D2
:1025C0000600007048E848487004070706010050FC
:1025D000A090D0B0909004070706010040206090C2
:1025E0009090600407070601002040609090906082
:1025F00004070706010020506090909060040707D0
:1026000006010050A060909090600407070601004A
:1026100050006090909060050505060000885020ED
:1026200050880408080601FF1070B0B0D0D0E080D8
:10263000040707060100402090909090600407076F
:10264000060100204090909090600407070601006A
:102650002050909090906004070706010050009071
:1026600090909060050707060000102088502020F9
:102670002004060606010080E09090E08004060633
:102680000601006090A0A090A0040707060100408A
:102690002000709090700407070601002040007031
:1026A0009090700407070601002050007090907011
:1026B00004070706010050A0007090907004060601
:1026C000060100500070909070040707060100207A
:1026D00050207090907005040406000070A8B07837
:1026E0000406060601FE708080702040040707067D
:1026F000010040200060B0C0700407070601002000
:10270000400060B0C0700407070601002050006060
:10271000B0C070040606060100500060B0C070032F
:102720000707060100804000C04040E0030707069D
:102730000100204000C04040E003070706010040C0
:10274000A000C04040E0030606060100A000C04013
:1027500040E00407070601003060107090906004AC
:10276000070706010050A000E090909004070706BC
:1027700001004020006090906004070706010020DF
:102780004000609090600407070601002050006040
:1027900090906004070706010050A00060909060D0
:1027A00004060606010050006090906005050506CD
:1027B00000002000F8002004040406010070B0D0DE
:1027C000E004070706010040200090909070040785
:1027D0000706010020400090909070040707060152
:1027E00000205000909090700406060601005000F2
:1027F000909090700409090601FE2040009090908E
:102800007090600408080601FE8080E09090E080EF
:10281000800408080601FE5000909090709060506F
:1028200072696E742066726F6D2053440050726935
:102830006E742066726F6D20534400022E2E004D80
:1028400061696E0046696C616D656E7400537465F4
:1028500070732F6D6D004A65726B00416363656C28
:1028600065726174696F6E0056656C6F6369747927
:1028700000436F6E66696775726174696F6E0045BB
:102880003273746570732F6D6D00453273746570AB
:10289000732F6D6D00453173746570732F6D6D000E
:1028A000453173746570732F6D6D005A7374657064
:1028B000732F6D6D005A73746570732F6D6D0059B1
:1028C00073746570732F6D6D005973746570732F19
:1028D0006D6D005873746570732F6D6D005873744F
:1028E0006570732F6D6D00416476616E6365642061
:1028F00053657474696E67730056652D6A65726BF3
:102900000056652D6A65726B00567A2D6A65726B8A
:1029100000567A2D6A65726B0056792D6A65726B66
:102920000056792D6A65726B0056782D6A65726B58
:102930000056782D6A65726B00416476616E63653E
:10294000642053657474696E677300416D6178200B
:10295000453200416D617820453200416D6178203B
:10296000453100416D617820453100416D6178202D
:102970005A00416D6178205A00416D6178205900FC
:10298000416D6178205900416D6178205800416D9A
:102990006178205800412D74726176656C00412D7C
:1029A00074726176656C00412D7265747261637436
:1029B00000412D7265747261637400416363656CDC
:1029C00000416363656C00416476616E63656420F9
:1029D00053657474696E6773005654726176206D26
:1029E000696E005654726176206D696E00566D698D
:1029F0006E00566D696E00566D6178204532005646
:102A00006D617820453200566D6178204531005661
:102A10006D617820453100566D6178205A00566D01
:102A20006178205A00566D6178205900566D6178A2
:102A3000205900566D6178205800566D61782058F5
:102A400000416476616E6365642053657474696ED9
:102A50006773004C6F6164206D6D2032004C6F61B4
:102A600064206D6D2032004C6F6164206D6D2031EB
:102A7000004C6F6164206D6D2031004C6F616420EB
:102A80006D6D004C6F6164206D6D00556E6C6F61F3
:102A900064206D6D203200556E6C6F6164206D6D29
:102AA000203200556E6C6F6164206D6D20310055D1
:102AB0006E6C6F6164206D6D203100556E6C6F61BE
:102AC00064206D6D00556E6C6F6164206D6D00410A
:102AD0006476616E6365204B453200416476616EB9
:102AE0006365204B453200416476616E6365204B1F
:102AF000453100416476616E6365204B453100418C
:102B00006476616E6365642053657474696E67737F
:102B10000044697361626C652073746570706572DE
:102B200073004D3834004C6576656C205820417830
:102B3000697300004175746F20686F6D65004732DE
:102B400038004D6F76652061786973004D61696E5C
:102B5000004578747275646572203200457874722D
:102B600075646572203100457874727564657220F1
:102B7000004D6F7665205A004D6F76652059004DE7
:102B80006F76652058004D6F76656D656E740045F3
:102B90007874727564657220320045787472756459
:102BA00065722031004D6F766520302E316D6D00DD
:102BB0004D6F766520316D6D004D6F76652031303B
:102BC0006D6D004D6F7665206178697300486F7494
:102BD000656E6420746F6F20636F6C640045787459
:102BE000727564657220004D6F7665205A004D6FD6
:102BF00076652059004D6F76652058004D6F7665DB
:102C0000205A004D6F76652059004D6F766520582B
:102C1000005761697420666F720066696C616D654A
:102C20006E742070757267650000506C6561736525
:102C300020776169742E0050726573732062757419
:102C4000746F6E00746F20726573756D652070729D
:102C5000696E74005761697420666F720066696CF2
:102C6000616D656E74206C6F616400496E7365728E
:102C7000742066696C616D656E7400616E642070AD
:102C80007265737320627574746F6E00746F206365
:102C90006F6E74696E75650050726573732062752E
:102CA00074746F6E00746F2068656174206E6F7A43
:102CB0007A6C65004E6F7A7A6C652068656174691C
:102CC0006E6700506C6561736520776169742E2EA4
:102CD0002E005761697420666F720066696C616DC1
:102CE000656E7420756E6C6F616400576169742045
:102CF000666F720066696C616D656E7420636861F1
:102D00006E676500746F207374617274004368614C
:102D10006E67696E672046696C616D656E740055FB
:102D20004E4C4F41442046494C414D454E54004C79
:102D30004F41442046494C414D454E540020204EC1
:102D40006F7A7A6C653A20002000456E64206669CF
:102D50006C616D656E74206368616E6765005075A7
:102D6000726765206D6F726500004D36303020420D
:102D700030205431004D3630302042302054300065
:102D80004368616E67652066696C616D656E74206D
:102D90004532004368616E67652066696C616D65E8
:102DA0006E74204531004D61696E004368616E6745
:102DB000652066696C616D656E7400556E6C6F613F
:102DC000642066696C616D656E74004C6F6164208F
:102DD00066696C616D656E74004D3630302042302E
:102DE00020542564004D373032203B2564004D3798
:102DF000303220542564004D373031205425640092
:102E00005072656865617420437573746F6D00500E
:102E100072656865617420437573746F6D005072DC
:102E20006568656174204142530050726568656150
:102E30007420504C41004261636B004E6F2053443C
:102E40002063617264005072696E742066726F6DE7
:102E50002053440041626F7574205072696E74652E
:102E600072004368616E67652066696C616D656EAE
:102E70007400436F6E66696775726174696F6E0086
:102E800054656D7065726174757265004D6F76651D
:102E90006D656E7400526573756D65207072696E34
:102EA000740054756E650053746F70207072696E93
:102EB00074005061757365207072696E7400496E9C
:102EC000666F2073637265656E0053746F70207057
:102ED00072696E74004D61696E005072696E742083
:102EE00061626F72746564004D3234004D3235207A
:102EF000500A4D323400466C6F77203200466C6FBA
:102F000077203200466C6F77203100466C6F772057
:102F1000310046616E207370656564203100466142
:102F20006E207370656564203100426564004265FF
:102F300064004E6F7A7A6C652032004E6F7A7A6C3C
:102F4000652032004E6F7A7A6C652031004E6F7AC0
:102F50007A6C652031005370656564005370656557
:102F600064004D61696E00436F6F6C646F776E0033
:102F700046616E20737065656420320046616E2084
:102F8000737065656420320046616E2073706565FC
:102F90006420310046616E207370656564203100E5
:102FA00042656400426564004E6F7A7A6C65203237
:102FB000004E6F7A7A6C652032004E6F7A7A6C65BB
:102FC0002031004E6F7A7A6C652031004D61696E58
:102FD00000526573746F7265206661696C73616617
:102FE00065004C6F61642073657474696E6773006B
:102FF00053746F72652073657474696E67730054DF
:103000006F6F6C204368616E676500416476616E26
:103010006365642053657474696E6773004D6169FC
:103020006E005A205261697365005A2052616973BB
:1030300065004D61696E004C756C7A426F74205466
:10304000415A20352072656164792E005072696E94
:1030500074696E672E2E2E005072696E7420706136
:103060007573656400436172642072656D6F766587
:1030700064004361726420696E73657274656400F4
:103080004D33310043616E6E6F7420656E746572EE
:10309000207375626469723A20006F70656E2066F5
:1030A00061696C65642C2046696C653A2000617525
:1030B000746F25632E67006572726F722077726974
:1030C00074696E6720746F2066696C650A004E6FC4
:1030D00074205344207072696E74696E670A0053DD
:1030E00044207072696E74696E672062797465201D
:1030F0000044656C6574696F6E206661696C656417
:103100002C2046696C653A200046696C6520646530
:103110006C657465643A0057726974696E672074EF
:103120006F2066696C653A20006F70656E2066617D
:10313000696C65642C2046696C653A20006F706587
:103140006E206661696C65642C2046696C653A2066
:103150000046696C652073656C65637465640A007C
:103160002053697A653A200046696C65206F706566
:103170006E65643A20002066696C653A20006672CC
:1031800065736800646F696E67004E6F7720004555
:103190004E4420535542524F5554494E450A002241
:1031A00020706F73002220706172656E743A220085
:1031B000535542524F5554494E452043414C4C20A3
:1031C0007461726765743A2200747279696E67205F
:1031D000746F2063616C6C207375622D67636F641C
:1031E000652066696C6573207769746820746F6FF9
:1031F000206D616E79206C6576656C732E204D4173
:1032000058206C6576656C2069733A310A004D323E
:1032100034004D32332025730053442063617264BF
:10322000206F6B0A006F70656E526F6F742066615D
:10323000696C65640A00766F6C756D652E696E69E0
:1032400074206661696C65640A00534420696E6984
:1032500074206661696C0A00286E6F2066696C656F
:10326000290043616E6E6F74206F70656E207375F8
:103270006264697220007C3C3E5E2B3D3F2F5B5DAB
:103280003B2C2A225C004F4646004F4E0065636887
:103290006F3A004572726F723A004572726F722017
:1032A00077726974696E6720746F20454550524F7C
:1032B0004D210A00507265737320627574746F6ECD
:1032C00020286F72204D3130382920746F206865B6
:1032D0006174206E6F7A7A6C650A00507265737340
:1032E00020627574746F6E20286F72204D313038F3
:1032F0002920746F20726573756D650A00496E73BD
:103300006572742066696C616D656E7420616E64AF
:1033100020707265737320627574746F6E20286FED
:1033200072204D313038290A004D3630303A205461
:103330006F6F20636F6C6400486F74656E642074F7
:103340006F6F20636F6C640A00486F74656E642051
:10335000746F6F20636F6C640A00496E73657274DA
:103360002066696C616D656E7420616E6420707298
:1033700065737320627574746F6E20286F72204DB0
:10338000313038290A0063616E63656C00726573C1
:10339000756D656400726573756D65007061757338
:1033A000656400706F7765726F6666002F2F6163CA
:1033B00074696F6E3A0020573A0020573A004578FA
:1033C00074727564657220256920436F6F6C696E35
:1033D000672E2E2E004578747275646572202569FB
:1033E0002048656174696E672E2E2E00202F002004
:1033F00040002042403A0020403A004D38342058E6
:103400002059205A204500546865726D616C205225
:10341000756E6177617900453120544845524D41C0
:103420004C2052554E415741590045322054484591
:10343000524D414C2052554E41574159004245444E
:1034400020544845524D414C2052554E4157415908
:1034500000202D20496E76616C6964206578747255
:1034600075646572206E756D62657220210A004870
:10347000656174696E67206661696C6564004265A8
:10348000642068656174696E67206661696C656453
:103490000048656174696E67206661696C656400E7
:1034A00045312048656174696E67206661696C65A5
:1034B000640045322048656174696E672066616901
:1034C0006C6564004D494E54454D502074726967D7
:1034D0006765726564004531204572723A204D4936
:1034E0004E54454D50004532204572723A204D49A8
:1034F0004E54454D50004572723A204D494E544548
:103500004D5020424544004D415854454D50207483
:103510007269676765726564004531204572723A69
:10352000204D415854454D50004532204572723A65
:10353000204D415854454D50004572723A204D413E
:103540005854454D5020424544006265640A002CA1
:103550002073797374656D2073746F707065642166
:10356000204865617465725F49443A2000236465B0
:1035700066696E652044454641554C545F004B6476
:1035800020004B6920004B702000006265640050F1
:103590004944204175746F74756E652066696E6963
:1035A00073686564212050757420746865206C61AF
:1035B0007374204B702C204B6920616E64204B6427
:1035C00020636F6E7374616E74732066726F6D200A
:1035D00062656C6F7720696E746F20436F6E6669E9
:1035E0006775726174696F6E2E680A0050494420D5
:1035F0004175746F74756E65206661696C656421D0
:103600002074696D656F75740A00546865726D6128
:103610006C2052756E6177617900453120544845C0
:10362000524D414C2052554E415741590045322090
:10363000544845524D414C2052554E415741590036
:1036400042454420544845524D414C2052554E412C
:103650005741590048656174696E67206661696CFD
:1036600065640045312048656174696E6720666154
:10367000696C65640045322048656174696E672035
:103680006661696C6564004265642068656174699F
:103690006E67206661696C6564005049442041751D
:1036A000746F74756E65206661696C656421205461
:1036B000656D706572617475726520746F6F2068D6
:1036C0006967680A00204B643A2000204B693A2061
:1036D00000204B703A20000A20436C6173736963C9
:1036E00020504944200A002054753A2000204B7590
:1036F0003A2000206D61783A2000206D696E3A20F2
:103700000020643A200020626961733A2000504929
:1037100044204175746F74756E65207374617274A2
:103720000A00504944204175746F74756E652066B7
:1037300061696C6564212054656D70657261747592
:10374000726520746F6F20686967680A001000ADA9
:103750000330016A0150022B0170030A019004F545
:1037600000B005E500D006D800F007CE001009C56E
:1037700000300ABE00500BB700700CB100900DABCA
:1037800000B00EA600D00FA200F0109D00101299FC
:1037900000301395005014920070158E0090168B17
:1037A00000B0178700D0188400F0198100101B7E2C
:1037B00000301C7B00501D7900701E7600901F7336
:1037C00000B0207000D0216E00F0226B0010246940
:1037D0000030256600502663007027610090285E47
:1037E00000B0295C00D02A5900F02B5600102D544F
:1037F00000302E5100502F4E0070304B0090314859
:1038000000B0324500D0334200F0343E0010363B69
:1038100000303737005038330070392E00903A2985
:1038200000B03B2300D03C1B00F03D1100103F01D5
:1038300000F03F00001000C90210012C01400122DD
:103840000170011801B0010E01F00104015002FAEB
:1038500000B002F0003003E600D003DC009004D298
:10386000007005C800A006BE000008B400B009AA98
:1038700000D00BA000600E960060118C0000158235
:103880000020197800C01D6E00A0226400B0275AE5
:1038900000902C500000314600E0343C00103832DB
:1038A00000903A2800603C1E00A03D1400803E0AB3
:1038B00000203F00006F70656E0054524947474535
:1038C000524544003A20007A5F6D6178007A5F6D5E
:1038D000696E00795F6D696E00785F6D696E005288
:1038E00065706F7274696E6720656E6473746F7053
:1038F000207374617475730A00456E6473746F701D
:103900007320256320256320256320256300205A2A
:103910003A0020593A0020583A00656E6473746F7B
:103920007073206869743A2000486F6D696E672073
:103930006661696C656400496E76616C69642065D6
:10394000787472756465720A0041637469766520E3
:1039500045787472756465723A200045313A2000EA
:1039600045303A20005A3A2000593A20004D533150
:103970002C4D53322C4D53332050696E730A583AF4
:1039800020004D6963726F737465707320756E618A
:103990007661696C61626C650A00205A3A002059B0
:1039A0003A0020436F756E7420583A00C23100000F
:1039B0001C260000F4190000D80F0000EB080000DE
:1039C000C0040000750200004001000024F4D4305F
:1039D00050C38E20C2A24017828B7011127A910DB3
:1039E000816CD90AA861E108C7586607615143068E
:1039F0001E4B5D05C145A7041A411104093D9803FA
:103A0000713931034036DB0265339102D430540200
:103A1000802E1D02632CEE01752AC501B028A0017D
:103A2000102781018F2564012B244B01E0223401F2
:103A3000AC211F018D200D01801FFC00841EED00B4
:103A4000971DDF00B81CD200E61BC600201BBC007F
:103A5000641AB200B219A8000A19A0006A189900E5
:103A6000D117910040178B00B516840031167E00E7
:103A7000B31579003A157300C7146F0058146A0023
:103A8000EE1366008813630025135E00C7125B0007
:103A90006C12570015125400C111510070114F00E3
:103AA00021114B00D61049008D10470046104400EC
:103AB00002104200C00F4000800F3E00420F3C0049
:103AC000060F3B00CB0E3800930E37005C0E35001E
:103AD000270E3400F30D3200C10D3100900D30007F
:103AE000600D2E00320D2D00050D2C00D90C2B0081
:103AF000AE0C2900850C29005C0C2700350C270032
:103B00000E0C2600E80B2400C40B2400A00B23009D
:103B10007D0B23005A0B2100390B2100180B2000CC
:103B2000F80A1F00D90A1E00BB0A1E009D0A1D00CC
:103B3000800A1D00630A1C00470A1B002C0A1B0098
:103B4000110A1A00F7091A00DD091900C409190041
:103B5000AB091900920917007B09180063091700C7
:103B60004C09160036091600200916000A0915002E
:103B7000F5081500E0081400CC081400B80814007B
:103B8000A4081400900813007D0812006B081300AD
:103B900058081200460812003408110023081100CA
:103BA0001208110001081100F0071000E0071000D2
:103BB000D0071000C0071000B0070F00A1071000C9
:103BC00091070E0083070F0074070F0065070E00B2
:103BD00057070E0049070E003B070D002E070E0089
:103BE00020070D0013070D0006070D00F9060C0055
:103BF000ED060D00E0060C00D4060C00C8060C0013
:103C0000BC060C00B0060C00A4060B0099060C00C4
:103C10008D060B0082060B0077060B006C060B006E
:103C200061060A0057060B004C060A0042060A000D
:103C300038060A002E060A0024060A001A060A00A0
:103C40001006090007060A00FD050900F405090031
:103C5000EB050900E2050900D9050900D0050900B6
:103C6000C7050900BE050900B5050800AD05080037
:103C7000A50509009C050800940508008C050800AE
:103C8000840508007C050800740508006C05070021
:103C9000650508005D050700560508004E0507008C
:103CA00047050700400508003805070031050700F3
:103CB0002A050700230507001C0506001605070056
:103CC0000F0507000805060002050700FB040600B3
:103CD000F5040700EE040600E8040600E20407000D
:103CE000DB040600D5040600CF040600C904060064
:103CF000C3040600BD040600B7040600B1040500B5
:103D0000AC040600A6040600A00405009B040600FF
:103D100095040500900406008A040500850405004A
:103D2000800406007A04050075040500700405008F
:103D30006B04050066040500610405005C040500D1
:103D400057040500520405004D0405004804050011
:103D5000430405003E0404003A0405003504050050
:103D6000300404002C04050027040400230405008B
:103D70001E0404001A0404001604050011040400C3
:103D80000D040400090405000404040000040400F8
:103D9000FC030400F8030400F4030400F00304002F
:103DA000EC030400E8030400E4030400E00304005F
:103DB000DC030400D8030400D4030400D00304008F
:103DC000CC030400C8030300C503030024F404D992
:103DD000201BC40C5C0E9804C4095F0265077101C6
:103DE000F405F900FB04B30048048700C10369002F
:103DF0005803550003034500BE023A008402310017
:103E000053022A002902250004022000E4011C00BC
:103E1000C8011900AF0117009801140084011300B4
:103E2000710110006101100051010E0043010D00ED
:103E300036010B002B010B0020010B0015010900BE
:103E40000C01090003010800FB000800F300080052
:103E5000EB000700E4000600DE000600D8000600C4
:103E6000D2000600CC000500C7000500C200050016
:103E7000BD000400B9000400B5000400B100040056
:103E8000AD000400A9000400A5000300A200030087
:103E90009F0004009B0003009800030095000200AF
:103EA00093000300900003008D0002008B000300CC
:103EB00088000200860002008400030081000200E6
:103EC0007F0002007D0002007B00020079000200FA
:103ED0007700010076000200740002007200010009
:103EE000710002006F0002006D0001006C00020012
:103EF0006A0001006900020067000100660001001D
:103F00006500010064000200620001006100010020
:103F1000600001005F0002005D0001005C00010024
:103F20005B0001005A000100590001005800010027
:103F30005700010056000100550001005400010027
:103F40005300000053000100520001005100010025
:103F5000500001004F0001004E0000004E00010023
:103F60004D0001004C0001004B0000004B0001001F
:103F70004A0001004900010048000000480001001B
:103F80004700010046000000460001004500000017
:103F9000450001004400010043000000430001000F
:103FA0004200000042000100410000004100010009
:103FB000400001003F0000003F0001003E00000003
:103FC0003E0001003D0000003D0001003C000000FB
:103FD0003C0000003C0001003B0000003B000100F1
:103FE0003A0000003A0001003900000039000100E9
:103FF00038000000380000003800010037000000E1
:1040000037000100360000003600000036000100D5
:1040100035000000350000003500010034000000CC
:1040200034000000340001003300000033000000C1
:1040300033000100320000003200000032000100B5
:1040400031000000310000003100010030000000AC
:1040500030000000300001002F0000002F000000A1
:104060002F0000002F0001002E0000002E00000095
:104070002E0001002D0000002D0000002D0000008A
:104080002D0001002C0000002C0000002C0000007E
:104090002C0001002B0000002B0000002B00000072
:1040A0002B0001002A0000002A0000002A00000066
:1040B0002A0001002900000029000000290000005A
:1040C000290000002900010028000000280000004D
:1040D0002800000028000000280001002700000040
:1040E0002700000027000000270000002700010033
:1040F0002600000026000000260000002600000028
:104100002600010025000000250000002500000019
:10411000250000002500000025000100240000000B
:1041200024000000240000002400000024000100FE
:1041300023000000230000002300000023000000F3
:1041400023000000230000002300010022000000E3
:1041500022000000220000002200000022000000D7
:1041600022000100210000002100000021000000C9
:1041700021000000210000002100000021000100BA
:1041800020000000200000002000000020000000AF
:10419000200000002000000020000000200001009E
:1041A0001F0000001F0000001F0000001F00000093
:1041B0001F0000001F0000001F0001001E00000083
:1041C0001E0000001E0000001E00000020286D6D73
:1041D0002900546F6F6C2D6368616E67696E673A72
:1041E0000A002055005431204C0020550054302046
:1041F0004C0046696C616D656E74206C6F61642F54
:10420000756E6C6F6164206C656E677468733A0AD2
:1042100000204B0020204D3930302054004C696E76
:1042200065617220416476616E63653A0A002044DC
:104230000020490020204D3330342050002044001D
:1042400020490020204D33303120500020440020F0
:10425000490020500020204D333031204500504986
:10426000442073657474696E67733A0A00204600CF
:1042700020420020480020204D3134352053004D8D
:104280006174657269616C20686561747570207015
:104290006172616D65746572733A0A00205900207D
:1042A000580020204D323138205400486F74656E1C
:1042B00064206F6666736574733A0A0020450020B7
:1042C0005A0020590020580020540020530020207C
:1042D0004D32303520420020453C6D61785F655F8E
:1042E0006A65726B3E0020583C6D61785F785F6A4A
:1042F00065726B3E20593C6D61785F795F6A6572CB
:104300006B3E205A3C6D61785F7A5F6A65726B3EE6
:1043100000416476616E6365643A20423C6D696E6B
:104320005F7365676D656E745F74696D655F7573E6
:104330003E20533C6D696E5F6665656472617465AD
:104340003E20543C6D696E5F74726176656C5F6689
:10435000656564726174653E00205400205200203F
:10436000204D323034205000416363656C657261CA
:1043700074696F6E2028756E6974732F7332293AD1
:1043800020503C7072696E745F616363656C3E209F
:10439000523C726574726163745F616363656C3E05
:1043A00020543C74726176656C5F616363656C3E3A
:1043B0000A0020450020204D323031205400205A80
:1043C0000020590020204D3230312058004D6178B6
:1043D000696D756D20416363656C65726174696FA9
:1043E0006E2028756E6974732F7332293A0A002083
:1043F000450020204D323033205400205A002059EF
:104400000020204D3230332058004D6178696D75A1
:104410006D206665656472617465732028756E69C8
:1044200074732F73293A0A00537465707320706592
:104430007220756E69743A0A0020204D313439209B
:1044400043203B20556E69747320696E2043656C70
:10445000736975730A002020473231202020203BE9
:1044600020556E69747320696E206D6D0020204D9B
:10447000363033200048617264636F6465642044A1
:10448000656661756C742053657474696E6773201A
:104490004C6F616465640A00282300002823000033
:1044A0006400000028230000282300000000964339
:1044B00000009643000040400000C8410000C84191
:1044C0000000C9420000C9420000C84400804F44B7
:1044D00000804F44290A002062797465733B206391
:1044E000726320002073746F726564207365747446
:1044F000696E6773207265747269657665642028D9
:1045000000202863616C63756C6174656429210AFD
:104510000020213D2000454550524F4D204352433D
:10452000206D69736D61746368202D202873746F2A
:104530007265642920002053697A653A2000496E2B
:104540006465783A2000204D61726C696E3D563684
:1045500034290A0028454550524F4D3D00454550ED
:10456000524F4D2076657273696F6E206D69736D61
:10457000617463682000290A002062797465733BC6
:1045800020637263200053657474696E67732053EF
:10459000746F726564202800454550524F4D206469
:1045A00061746173697A65206572726F722E0A0098
:1045B0005761726E696E673A20486F6D696E672049
:1045C00042756D702044697669736F72203C2031AA
:1045D0000A00020204486F6D652025732573257358
:1045E000206669727374002066697273740A005AD7
:1045F0000059005800486F6D65200020746F6F20CF
:104600006C6F6E6720657874727573696F6E207059
:10461000726576656E7465640A0020636F6C642051
:10462000657874727573696F6E2070726576656EE9
:104630007465640A0020453A00205A3A0020593A2D
:1046400000583A0000004842000048420000404044
:10465000FFFFFF0000A0400000A04000000040005D
:1046600000904300008A4300007A43000000C0002D
:104670000000000000000000008F4300008A43009B
:10468000007A43000000C00000000000000000208D
:10469000746F6F206C6F6E672065787472757369C4
:1046A0006F6E2070726576656E7465640A002063B3
:1046B0006F6C6420657874727573696F6E207072A8
:1046C0006576656E7465640A00627573793A207068
:1046D000617573656420666F7220696E7075740A07
:1046E00000627573793A2070617573656420666F36
:1046F0007220757365720A00627573793A20707260
:104700006F63657373696E670A0020496E76616C2A
:10471000696420657874727564657220004D313467
:104720003520533C696E6465783E206F7574206F48
:10473000662072616E67652028302D31290A00439A
:104740006C69636B20746F20726573756D652E2EB6
:104750002E00556E6B6E6F776E20636F6D6D616EA0
:10476000643A202200454550524F4D204F4B0A00DD
:104770004E6F206D6F76652E004543484F00494EC1
:10478000464F004552524F52530044525952554ED3
:1047900000434F4D4D554E49434154494F4E006FD4
:1047A00066660079477E4783478A4791474445427A
:1047B00055473A004C756C7A426F742054415A2028
:1047C00035204F46462E00205A0020590058002020
:1047D000204D61783A2000205A00205900580020CE
:1047E000204D696E3A2000536F667420656E6473C5
:1047F000746F70733A20002569730025696D202558
:104800006973002569682025696D20256973002575
:104810006964202569682025696D20256973002554
:10482000697920256964202569682025696D20251E
:104830006973005072696E742074696D653A200066
:104840004D3131332053002F2F20004361703A0047
:104850004D4F54494F4E5F4D4F44455300544845CA
:10486000524D414C5F50524F54454354494F4E00B6
:104870004155544F5245504F52545F53445F535427
:10488000415455530050524F4D50545F5355505062
:104890004F525400454D455247454E43595F504194
:1048A0005253455200434153455F4C494748545F7A
:1048B0004252494748544E45535300544F47474C82
:1048C000455F4C494748545300534F465457415253
:1048D000455F504F574552004255494C445F504543
:1048E0005243454E54004C4556454C494E475F4453
:1048F000415441005A5F50524F4245004155544F78
:104900004C4556454C005052494E545F4A4F420068
:1049100050524F4752455353004155544F52455002
:104920004F52545F54454D5000564F4C554D4554D1
:1049300052494300454550524F4D0053455249415D
:104940004C5F584F4E5F584F4646004649524D57B0
:104950004152455F4E414D453A4D61726C696E2042
:10496000204649524D574152455F56455253494F93
:104970004E3A322E302E302E39342045585452556E
:104980004445525F545950453A4475616C457874BA
:10499000727564657220763220534F555243455FDD
:1049A000434F44455F55524C3A68747470733A2FC4
:1049B0002F636F64652E616C6570686F626A6563F2
:1049C00074732E636F6D2F646966667573696F6E9D
:1049D0002F4D41524C494E2050524F544F434F4C53
:1049E0005F56455253494F4E3A312E30204D414388
:1049F00048494E455F545950453A4C756C7A426F60
:104A0000742054415A20352045585452554445523B
:104A10005F434F554E543A3220555549443A63331B
:104A20003235356339362D343039372D3438383412
:104A30002D386564302D646564326666396261655F
:104A400036310A002020536D6F6F7468696E6720DD
:104A5000286D6D293A202020202020202020202091
:104A6000202020202020530020204261636B6C61B5
:104A700073682044697374616E636520286D6D29C5
:104A80003A20202020202020200020202020202824
:104A900046312E30203D2066756C6C2C2046302E21
:104AA00030203D206E6F6E65290A002020436F7212
:104AB00072656374696F6E20416D6F756E742F46F9
:104AC0006164652D6F75743A2020202020460061B6
:104AD00063746976653A0A00696E004261636B6CC3
:104AE00061736820636F7272656374696F6E2069A9
:104AF000732000486F6D6520585920666972737481
:104B00000A00486F6D6520585920666972737400F9
:104B100043757272656E742066696C653A20004553
:104B20006E642066696C65206C6973740A00426566
:104B300067696E2066696C65206C6973740A004150
:104B40006476616E6365204B003F4B2076616C7527
:104B500065206F7574206F662072616E676520280E
:104B6000302D3130292E0A003F542076616C756556
:104B7000206F7574206F662072616E67652E0A0063
:104B800020466C6F773A2000205A0020643A0020BB
:104B9000693A0020703A00204500204D39322054F7
:104BA00000205A00205900204D3932205800486F0B
:104BB00074656E64206F6666736574733A0043298A
:104BC0000A0061626C656420286D696E2074656DF1
:104BD00070200064697300656E00436F6C6420652B
:104BE00078747275646573206172652000205400CA
:104BF000205200416363656C65726174696F6E3A3F
:104C0000205000496E76616C696420657874727515
:104C10006465720A0020643A0020693A0020703A04
:104C200000536C6565702E2E2E0047322F473320BF
:104C300062616420706172616D65746572730A00EF
:104C4000446F6E6520736176696E672066696C6576
:104C50002E0A0053442072656164206572726F727F
:104C60000A00446F6E65207072696E74696E672009
:104C700066696C650A0053544F505045442E20001D
:104C80005072696E7465722073746F707065642001
:104C900064756520746F206572726F72732E204682
:104CA000697820746865206572726F7220616E6425
:104CB00020757365204D39393920746F2072657302
:104CC000746172742E202854656D706572617475FC
:104CD00072652069732072657365742E2053657444
:104CE00020697420616674657220726573746172E4
:104CF00074696E67290A004E6F20436865636B73A1
:104D0000756D2077697468206C696E65206E756DAD
:104D10006265722C204C617374204C696E653A2078
:104D2000004E6F20436865636B73756D20776974FF
:104D300068206C696E65206E756D6265722C204C02
:104D4000617374204C696E653A2000636865636B1B
:104D500073756D206D69736D617463682C204C618F
:104D60007374204C696E653A20004C696E65204E64
:104D7000756D626572206973206E6F74204C61736B
:104D800074204C696E65204E756D6265722B312CF6
:104D9000204C617374204C696E653A20004D3131AE
:104DA0003000526573656E643A2000204200205046
:104DB000006F6B00656E7175657565696E672022A1
:104DC00000504944204175746F74756E65206661AA
:104DD000696C656421204261642065787472756431
:104DE0006572206E756D6265720A004265642063AB
:104DF0006F6F6C696E672E2E2E00426564206865A9
:104E00006174696E672E2E2E006F6B00473020583C
:104E100031373020593239302046333030300A4D66
:104E2000313137205072696E742061626F7274651F
:104E3000642E002020506C616E6E6572427566664D
:104E4000657242797465733A200020467265652068
:104E50004D656D6F72793A2000436F6D70696C65B6
:104E6000643A2046656220323620323031390A00F9
:104E7000207C20417574686F723A2028416C6570FF
:104E800068204F626A6563747320496E632E2C201C
:104E90004C756C7A426F7420476974205265706F4C
:104EA0007369746F7279290A0000204C6173742051
:104EB000557064617465643A2000322E302E302EB5
:104EC00039340A004D61726C696E0020536F66744C
:104ED000776172652052657365740A0020576174AA
:104EE0006368646F672052657365740A00204272BC
:104EF0006F776E206F75742052657365740A002099
:104F000045787465726E616C2052657365740A0031
:104F1000506F77657255700A0073746172740A007D
:104F20004B494C4C45442E20005072696E7465729A
:104F30002068616C7465642E206B696C6C28292074
:104F400063616C6C6564210A004B494C4C206361C1
:104F50007573656420627920746F6F206D75636866
:104F600020696E6163746976652074696D65202DB2
:104F70002063757272656E7420636F6D6D616E640F
:104F80003A200050726F7465637465642050696ED6
:104F90000A0025301D0C282924311C0B4527232FFE
:104FA0001B0A1E4443222B1A4142212A193F400367
:104FB0003809FF3607FF37030608020200014D3E9D
:104FC000086DC276DC8EC2E5E700E900E2761124C6
:104FD0001FBECFEFD1E2DEBFCDBF00E00CBF13E0BC
:104FE000A0E0B2E0E0EDFEE302E00BBF02C00790FC
:104FF0000D92A43AB107D9F725E1A4EAB3E001C0C4
:105000001D92A13FB207E1F717E2C6EED7E200E03A
:1050100006C021970109802FFE010F947817CF3D1C
:10502000D10780E00807A9F70E9452330D94571F5B
:105030000C9400001F920F920FB60F9211242F9321
:105040003F938F939F93AF93BF938091A5039091CC
:10505000A603A091A703B091A8033091A40323E075
:10506000230F2D3720F40196A11DB11D05C026E8A0
:10507000230F0296A11DB11D2093A4038093A503C5
:105080009093A603A093A703B093A8038091A903CC
:105090009091AA03A091AB03B091AC030196A11D1E
:1050A000B11D8093A9039093AA03A093AB03B0937F
:1050B000AC03BF91AF919F918F913F912F910F9032
:1050C0000FBE0F901F9018952FB7F8946091A5030D
:1050D0007091A6038091A7039091A8032FBF089514
:1050E0003FB7F8948091A9039091AA03A091AB03D4
:1050F000B091AC0326B5A89B05C02F3F19F00196CF
:10510000A11DB11D3FBFBA2FA92F982F8827820F4D
:10511000911DA11DB11DBC01CD0142E0660F771F9D
:10512000881F991F4A95D1F708958F929F92AF9249
:10513000BF92CF92DF92EF92FF926B017C01D0DFA2
:105140004B015C01C114D104E104F104F1F091D3ED
:10515000C7DFDC01CB0188199909AA09BB09883E80
:105160009340A105B10570F321E0C21AD108E1080E
:10517000F10888EE880E83E0981EA11CB11CC114B2
:10518000D104E104F10421F7DDCFFF90EF90DF902F
:10519000CF90BF90AF909F908F900895789484B5F2
:1051A000826084BD84B5816084BD85B5826085BD23
:1051B00085B5816085BDEEE6F0E080818160808309
:1051C000E1E8F0E0108280818260808380818160EC
:1051D0008083E0E8F0E0808181608083E1EBF0E0B3
:1051E000808184608083E0EBF0E080818160808357
:1051F000E1E9F0E08081826080838081816080834A
:10520000E0E9F0E0808181608083E1EAF0E0808184
:1052100082608083808181608083E0EAF0E0808129
:1052200081608083E1E2F1E080818260808380811F
:1052300081608083E0E2F1E0808181608083EAE741
:10524000F0E08081846080838081826080838081BF
:10525000816080838081806880831092C10008957E
:105260001F93CF93DF93182FEB0161E016D12097A6
:1052700011F460E004C0CF3FD10531F461E0812F2B
:10528000DF91CF911F9145C1E12FF0E0EF5EFD4F1F
:10529000E4914E2F50E0FA013197E231F10508F028
:1052A0009DC08827EE58FF4F8F4F0D94781784B517
:1052B000806884BDC7BD97C084B5806284BDC8BD09
:1052C00092C080918000806880938000D093890094
:1052D000C093880088C080918000806280938000A5
:1052E000D0938B00C0938A007EC08091800088603C
:1052F00080938000D0938D00C0938C0074C0809107
:10530000B00080688093B000C093B3006CC08091FF
:10531000B00080628093B000C093B40064C08091FC
:105320009000806880939000D0939900C09398007B
:105330005AC080919000806280939000D0939B002F
:10534000C0939A0050C08091900088608093900034
:10535000D0939D00C0939C0046C08091A0008068BF
:105360008093A0008091A0008F7B8093A000D093B9
:10537000A900C093A80037C08091A00080628093EC
:10538000A000D093AB00C093AA002DC08091A000D4
:1053900088608093A000D093AD00C093AC0023C080
:1053A00080912001806880932001D0932901C093CF
:1053B000280119C080912001806280932001D09340
:1053C0002B01C0932A010FC0809120018860809337
:1053D0002001D0932D01C0932C0105C0C038D10508
:1053E0000CF04CCF46CFDF91CF911F91089590E004
:1053F000FC013197E231F10508F04EC08827EC57E7
:10540000FF4F8F4F0D947817809180008F7703C0E6
:10541000809180008F7D809380000895809180002E
:10542000877FF9CF84B58F7702C084B58F7D84BD27
:1054300008958091B0008F7703C08091B0008F7D78
:105440008093B0000895809190008F7707C080917D
:1054500090008F7D03C080919000877F80939000A3
:1054600008958091A0008F7707C08091A0008F7D64
:1054700003C08091A000877F8093A0000895809151
:1054800020018F7707C0809120018F7D03C080911C
:105490002001877F809320010895CF93DF9390E0D0
:1054A000FC01E95AFD4F2491FC01E356FD4F849124
:1054B000882361F190E0880F991FFC01E95EFC4FA1
:1054C000C591D491FC01E350FD4FA591B4916111B8
:1054D00009C09FB7F8948881209582238883EC9136
:1054E0002E230BC0623061F49FB7F8943881822F6D
:1054F000809583238883EC912E2B2C939FBF06C02D
:105500008FB7F894E8812E2B28838FBFDF91CF913E
:1055100008951F93CF93DF93282F30E0F901EF5EBA
:10552000FD4F8491F901E95AFD4FD491F901E356F9
:10553000FD4FC491CC23C1F0162F811158DFEC2F01
:10554000F0E0EE0FFF1FE350FD4FA591B4918FB730
:10555000F894111105C09C91ED2FE095E92302C04C
:10556000EC91ED2BEC938FBFDF91CF911F910895BC
:10557000CF93DF93282F30E0F901EF5EFD4F849148
:10558000F901E95AFD4FD491F901E356FD4FC49159
:10559000CC2389F081112BDFEC2FF0E0EE0FFF1F01
:1055A000ED51FD4FA591B491EC91ED2381E090E098
:1055B00021F480E002C080E090E0DF91CF91089577
:1055C00008951F920F920FB60F9211240BB60F92EF
:1055D0002F933F934F935F936F937F938F939F93FB
:1055E000AF93BF93EF93FF93E0910402F091050214
:1055F0001995FF91EF91BF91AF919F918F917F91FD
:105600006F915F914F913F912F910F900BBE0F9033
:105610000FBE0F901F9018951F920F920FB60F920A
:1056200011240BB60F922F933F934F935F936F9379
:105630007F938F939F93AF93BF93EF93FF93E091EB
:105640000602F09107021995FF91EF91BF91AF917A
:105650009F918F917F916F915F914F913F912F918A
:105660000F900BBE0F900FBE0F901F9018951F92BA
:105670000F920FB60F9211240BB60F922F933F93F8
:105680004F935F936F937F938F939F93AF93BF934A
:10569000EF93FF93E0910802F09109021995FF91B1
:1056A000EF91BF91AF919F918F917F916F915F919A
:1056B0004F913F912F910F900BBE0F900FBE0F9007
:1056C0001F9018951F920F920FB60F9211240BB6D0
:1056D0000F922F933F934F935F936F937F938F938B
:1056E0009F93AF93BF93EF93FF93E0910A02F091E2
:1056F0000B021995FF91EF91BF91AF919F918F91FF
:105700007F916F915F914F913F912F910F900BBEC1
:105710000F900FBE0F901F9018951F920F920FB60B
:105720000F9211240BB60F922F933F934F935F93D9
:105730006F937F938F939F93AF93BF93EF93FF9359
:10574000E0910002F09101021995FF91EF91BF9154
:10575000AF919F918F917F916F915F914F913F9109
:105760002F910F900BBE0F900FBE0F901F901895AA
:105770001F920F920FB60F9211240BB60F922F9318
:105780003F934F935F936F937F938F939F93AF93C9
:10579000BF93EF93FF93E0910202F09103021995FA
:1057A000FF91EF91BF91AF919F918F917F916F91F9
:1057B0005F914F913F912F910F900BBE0F900FBEB5
:1057C0000F901F9018951F920F920FB60F921124F1
:1057D0000BB60F922F933F934F935F936F937F93EB
:1057E0008F939F93AF93BF93EF93FF93E0910C023E
:1057F000F0910D021995FF91EF91BF91AF919F919B
:105800008F917F916F915F914F913F912F910F9069
:105810000BBE0F900FBE0F901F9018951F920F9206
:105820000FB60F9211240BB60F922F933F934F9305
:105830005F936F937F938F939F93AF93BF93EF93F8
:10584000FF93E0910E02F0910F021995FF91EF91F5
:10585000BF91AF919F918F917F916F915F914F9188
:105860003F912F910F900BBE0F900FBE0F901F9086
:10587000189508951F93CF93DF93EC011D821C822E
:105880001F821E82198681E0888782E28A871F86AE
:105890001E86FE01B396CE01C1962FEF2193E81725
:1058A000F907E1F711E018A3CE01E1D51F8B188E9F
:1058B000198E80E48A8F1B8E88E090E39AAB89ABC7
:1058C000DF91CF911F910895DB01ED91FC91199427
:1058D000EF92FF921F93CF93DF931F921F92CDB74A
:1058E000DEB77C01DC01D196ED91FC91D29782E08C
:1058F00069837A83199520E030E04AE069817A81F2
:10590000C701E2DF182FD701D196ED91FC91D29714
:1059100083E01995D701D196ED91FC91D29780E063
:105920001995812F0F900F90DF91CF911F91FF90CC
:10593000EF9008950F931F93CF93DF93EC018B01AA
:10594000E9A9FAA982E01995E9A9FAA981E01995CE
:1059500020E030E044E1B801CE01B6DF9E012D5CCD
:105960003F4F47E1B801CE01AFDFE9A9FAA980E0D6
:10597000DF91CF911F910F911994EF92FF921F9396
:10598000CF93DF93EC017B01E9A9FAA982E0199595
:10599000E9A9FAA981E0199520E030E045E1B701D5
:1059A000CE0192DF182F882339F09E012D5C3F4FE6
:1059B00047E1B701CE0188DFE9A9FAA980E019958E
:1059C000812FDF91CF911F91FF90EF900895FC01FF
:1059D000448F258F9C01245E3F4F42E375CFCF93C8
:1059E000DF931F92CDB7DEB79E012F5F3F4F46E496
:1059F0006BDF89810F90DF91CF910895CF93DF9373
:105A00001F92CDB7DEB79E012F5F3F4F47E45CDFAB
:105A100089810F90DF91CF91089520E030E048E434
:105A200053CFCF93DF93EC016A817B81D8DF8883EA
:105A30006A817B81CE01E2DF89836A817B81CE012D
:105A4000ECDF8B879E012D5C3F4F6A817B8147E1B4
:105A5000CE01DF91CF9138CFCF93DF93EC016A81F4
:105A60007B8136DF882319F0CE01DBDF81E0DF9117
:105A7000CF9108958F929F92AF92BF92CF92EF9263
:105A80000F93CF93DF931F921F92CDB7DEB74C01D8
:105A90005B012A834983EEDEF401B382A28249814D
:105AA00047A32A8120A705A3E4A2C3A2C4010F90A3
:105AB0000F90DF91CF910F91EF90CF90BF90AF906B
:105AC0009F908F90C9CFFC016281738133CFCF93B8
:105AD000DF93EC01EE85FF85309709F019956A8117
:105AE0007B81CE01DF91CF9148CF362F242FFC014F
:105AF00062817381432F6BCF0F93FC01828193816D
:105B0000648F458F278F068F9F01245E3F4F4BE3A5
:105B1000BC01CF010F91D8CEFC0160A30895BF92C4
:105B2000CF92DF92EF92FF920F931F93CF93DF9369
:105B30006C01D62FB42EC22F7801CC2369F0F70167
:105B4000049120E04B2D6D2FC601D6DFFFEFEF1A39
:105B5000FF0AC150D85FF1CFDF91CF911F910F9114
:105B6000FF90EF90DF90CF90BF9008958F929F921B
:105B7000AF92BF92CF92DF92EF92FF920F931F935B
:105B8000CF93DF935C01C62EC42FD22ED02F220FCD
:105B9000220F220F1ED0882379F0DC0F8D2C912C40
:105BA000CD1751F087012D2D4C2F6C2DC501B7DF7E
:105BB000E80CF91CCF5FF4CFDF91CF911F910F91CB
:105BC000FF90EF90DF90CF90BF90AF909F908F901D
:105BD00008950F93FC010150040F84A996A994170E
:105BE00018F0081728F402C0081750F0041740F402
:105BF0002150260F83A995A9961720F4281720F481
:105C000080E007C0281720F481E0261710F0F8CFB5
:105C100081E00F91089581E008952EE93FE000971B
:105C200029F0F9013197F1F70197F9CF0895FC01B7
:105C3000128280818150838314820895FC018081C7
:105C40009281980F92832181921760F494819F5FD3
:105C500094839381890F821710F08FEF820F8383D3
:105C600081E0089580E00895FC0191E0838186172A
:105C700008F490E031E0461708F030E0832F892BDC
:105C800021E05281451708F420E02823832F89233F
:105C9000822B0895DC01FB01108212968C911297E1
:105CA000818315968C9115978150828313968C91E0
:105CB00083830895FB0141812381213029F0233022
:105CC00031F468EF640F04C0642F485F01C0642F93
:105CD000CBCFDC0115962C9115971696ED91FC9182
:105CE0001797CF01820F911D820F911D1192E81716
:105CF000F907E1F70895FC01A681B7818281481B6D
:105D00008581483018F0A80FB11D4770382F36959F
:105D100036953695562F577080E890E002C09595DD
:105D200087955A95E2F7439F402D11246695669515
:105D30006695E62FF0E0E40FF11DEA0FFB1F3081BE
:105D4000222311F0832B02C0809583238083089542
:105D5000FB014181DC0112962C911297421760F0F1
:105D600013962C911397241738F0608115962C9177
:105D7000621710F42481BFCF0895CF92DF92FF9273
:105D80000F931F93CF93DF936C01EB01FA809B81FC
:105D9000913051F030F0923049F0933051F41FEFD0
:105DA00009C010E001E007C011E004C010E00FEFEF
:105DB00002C010E000E0F7FE03C0BE01C601C8DF6C
:105DC0009881900F98839981910F9983FF0C99F78F
:105DD000DF91CF911F910F91FF90DF90CF900895A9
:105DE0000F931F93CF93DF938901FB01C281D3816E
:105DF0004233D9F058F44531E1F0473109F14431EB
:105E000041F5CE0166DFCE0112DF23C04634E1F05A
:105E10004734E1F04B33E9F4B901CE014BDF88237D
:105E2000C1F0B801CE01A9DF14C0B901CE0190DFE5
:105E300010C0CE0103DF882369F0CE014ADF09C01C
:105E4000B901CE0127DF05C08D8101C08981F8012C
:105E5000808381E0DF91CF911F910F910895CF92C0
:105E6000DF92EF92FF920F931F93CF93DF937C010A
:105E7000D62FD42EC22F122FC62EC20E6C2D611B10
:105E8000183038F00FEF20E04D2DC70135DE1850E7
:105E9000F5CF6C2F687F6D0F2C2F277071F097E076
:105EA00029272F5F27700FEF10E001C0000F2A9500
:105EB000EAF720E04D2DC7011FDEDF91CF911F9142
:105EC0000F91FF90EF90DF90CF900895CF92DF92E7
:105ED000EF92FF920F931F93CF93DF937C01D62E07
:105EE000D42FC22F122FC42EC20E4C2D411B18309E
:105EF00038F00FEF21E06D2DC701FEDD1850F5CF12
:105F00004C2F487F4D0F2C2F277071F097E02927D9
:105F10002F5F27700FEF10E001C0000F2A95EAF7FE
:105F200021E06D2DC701E8DDDF91CF911F910F9129
:105F3000FF90EF90DF90CF900895DF92EF92FF9265
:105F40000F931F93CF93DF937C01162FC42FD22E74
:105F5000D02F3FDE8823F9F02D2D4C2F612FC70164
:105F60007EDF2D2F4C2F612FC701B0DF6FEF6D0D3E
:105F7000610F2D2F4C2FC701A9DF4FEF4D0F4C0F95
:105F80002D2D612FC701DF91CF911F910F91FF90B0
:105F9000EF90DF9064CFDF91CF911F910F91FF9031
:105FA000EF90DF900895EF92FF920F931F93CF939E
:105FB000DF937C01D62F122FC42F040F212F4C2FDB
:105FC0006D2FC7014CDFCF5F0C13F8CFDF91CF915E
:105FD0001F910F91FF90EF900895DF92EF92FF9243
:105FE0000F931F93CF93DF93EC01162FF42EE22E25
:105FF000F0DD882329F02E2D4F2D612FCE01D3DF28
:10600000DF91CF911F910F91FF90EF90DF90089556
:106010000895FC01E60FF11D849190E0982F8827E8
:106020003196E4918E0F911D0895FC01849108959D
:10603000FCDF882321F0823011F083E0089586E0B0
:10604000089580E00895FC018081089566E0E1CF25
:1060500068E0DFCF0A96FC01849108950B96FC015D
:1060600084910895DC011496ED91FC911597319679
:1060700084910895BF92CF92DF92EF92FF920F9397
:106080001F93CF93DF938C01E62EDC011496CD9104
:10609000DC911597CE01C9DFF82EF8018481958136
:1060A000C7DFC82EF1E0FF1203C02FE0B22E02C0FE
:1060B000BB24BA94D80114968D919C911597CADF90
:1060C000F82EF80184819581C9DFD82ED801149665
:1060D0008D919C911597BCDFB0E6BE1538F4009702
:1060E00029F0C80FD91F91E6F92E0FC0F80184815D
:1060F0009581ACDFF0E4FE1538F4009729F0C80F65
:10610000D91F81E4F82E01C06196DE1490F4D80105
:1061100050961C92509753961C92539754961C92EB
:10612000549751961C92519752961C9280E090E0A1
:1061300066C0DF1460F38C2D90E0FE0124912F3FA8
:1061400011F4219657C0FE104CC0D80114968D91C1
:106150009C9115976ADF9E012F5F3F4FFE018823B8
:1061600011F08230E1F48491D80153968C935397C7
:10617000F901249154962C935497FE013396E4919F
:106180005096EC935097FE013496E4915196EC931F
:106190005197FE013596E4915296EC9320C084917C
:1061A000982F9F709250D80152969C935297829547
:1061B0008F7051968C935197F9012491822F8F7093
:1061C00054968C93549722952F7053962C935397F3
:1061D000FE013296E491E295EF705096EC93CE0179
:1061E0000EC0FE013296E491EB219C012E0F311D71
:1061F000C20FD31FFD1409F48ACFF3949ECFDF9111
:10620000CF911F910F91FF90EF90DF90CF90BF90B3
:1062100008954F925F926F927F929F92AF92BF923A
:10622000CF92DF92EF92FF920F931F93CF93DF9362
:106230001F92CDB7DEB72C01C62E942E622F1ADF27
:106240007C01892B09F43AC0F20184819581F0DE4A
:10625000B82EF201138904898189C80E8289981A9F
:10626000D92CD01A212F4D2D6C2DC201B2DC8823E0
:1062700011F1EB0CF11C195F169516951695612E10
:10628000712CD914C1F03C2D57018A2D8E1981171C
:1062900070F4F501049120E04D2D632FC201398384
:1062A0002BDCFFEFAF1ABF0A3981385FEECFE60C67
:1062B000F71CD394E6CFF201808901C080E00F90F3
:1062C000DF91CF911F910F91FF90EF90DF90CF90D2
:1062D000BF90AF909F907F906F905F904F90089588
:1062E0000F931F93CF93DF9300D0CDB7DEB78C0110
:1062F000DC015596ED91FC9156972B834A83698377
:1063000019954A81480F2B816981C8010F900F9020
:106310000F90DF91CF911F910F917BCFAF92BF92E2
:10632000DF92EF92FF920F931F93CF93DF931F9211
:106330001F92CDB7DEB77C01D62E042FDC01559617
:10634000ED91FC91569729833A831995080F29817D
:10635000A22E3A81B32E10E0F50121915F01222394
:1063600039F0402F6D2DC70154DFD80E180FF4CF30
:10637000812F0F900F90DF91CF911F910F91FF9080
:10638000EF90DF90BF90AF900895DF92EF92FF9271
:106390000F931F93CF93DF937C01D62FD42E8901C7
:1063A000DC015596ED91FC9156971995D80EC0E0F9
:1063B000F8012491222349F04D2D6D2FC70129DFCB
:1063C000D80FC80F0F5F1F4FF3CF8C2FDF91CF91E6
:1063D0001F910F91FF90EF90DF900895DC011496CC
:1063E0002D913C9115972115310509F43FC0579621
:1063F0008C915797F901811108C03596E491589610
:10640000EC935897F9013C9611C0813041F43F96C6
:10641000E4915896EC935897F901709607C03D9611
:10642000E4915896EC935897F9013E96E491599669
:10643000EC93599758968C915897082E000C990B0D
:1064400059962C915997821B910927FD93955A963D
:106450002C915A97203441F0829FC001112426E0EC
:10646000969587952A95E1F75B968C93089521E29E
:1064700030E3FC01368B258B0895CF92DF92EF92AB
:10648000FF920F931F93CF93DF938C017B016A01DF
:10649000CB01FA011995D82F882311F1682FC80173
:1064A000E9DDF801C189C195FFEFEF1AFF0AC701C5
:1064B000F6011995F801882351F08089C80FC701AA
:1064C000F6011995D82F682FC801D4DDEDCFD03251
:1064D00021F091898389890F01C080898C0F01C0C7
:1064E00080E0DF91CF911F910F91FF90EF90DF90AF
:1064F000CF90089543E250E3C0CFCF93DF93FC01E8
:10650000248135812617370741F0EC0175836483B8
:1065100065DF81E290E39E8B8D8BDF91CF910895B3
:106520004F925F926F927F92AF92BF92CF92DF9223
:10653000EF92FF920F931F93CF93DF93CDB7DEB708
:1065400029013A019B01AC01241935094609570973
:106550008A899B89AC89BD89BC01CD016A197B09F7
:106560008C099D090F94F816A80197012419350983
:10657000460957090F945C17CA01B9016A0D7B1DC2
:106580008C1D9D1DDF91CF911F910F91FF90EF907A
:10659000DF90CF90BF90AF907F906F905F904F90C3
:1065A000089580E090E008950895CF92DF92EF92F1
:1065B000FF920F931F93CF93DF936C017A018B01AE
:1065C000C0E0D0E0CE15DF0589F0D8016D918D01D6
:1065D000D601ED91FC910190F081E02DC601199555
:1065E000892B11F47E0102C02196ECCFC701DF9107
:1065F000CF911F910F91FF90EF90DF90CF90089572
:10660000DC01ED91FC910190F081E02D1994CF9384
:10661000CFB7F8948091AD03811127C0E2EDF2E08D
:106620008491ECE8F2E09491E82FF0E0EE0FFF1F88
:10663000E95EFC4FA591B491EC91E92321F461E06E
:1066400085E30E94892A61E085E30E944D2A8CB58A
:1066500080618CBD8CB580648CBD61E084E30E9458
:106660004D2A61E083E30E944D2A8091AD038F5F44
:106670008093AD03CFBFCF910895CF92EF920F9348
:10668000FC0113AE14AE15AE0496F4D90F91EF9041
:10669000CF9008958EBD00000DB407FEFDCF8EB5DE
:1066A000089508950E94CE28FCDF0F946E12C0E07A
:1066B000D0E00F94F3122097E1F30E940000F9CF8D
:1066C000E9ECF3E083AF64AF0895EF92FF920F938C
:1066D0001F93CF93DF937A016F3F71058105910579
:1066E00009F048F489EC93E08BDF8DEC93E0BADCA1
:1066F000282F30E014C0C0910404D09105044D2F20
:1067000050E0EC2FF0E08B019C01BF018DEC93E099
:1067100034D6C80FC0930404D09305049C01C9016A
:10672000DF91CF911F910F91FF90EF900895EF921D
:10673000FF920F931F93CF93DF938B01C9ECD3E0AC
:10674000FBACECAC4E2D50E06F2D70E09C018DEC5D
:1067500093E06AD6F80EFBAEECAEDF91CF911F91BD
:106760000F91FF90EF900895EF92FF920F931F9378
:10677000CF93DF938B01C9ECD3E0FBACECAC4E2D97
:1067800050E06F2D70E09C018DEC93E098D6F80EF0
:10679000FBAEECAEDF91CF911F910F91FF90EF9088
:1067A00008956FEF7FEFC3CF4FEF5FEF8ECFCF93A3
:1067B00087E895E00E944467C82F60E870E087E8AA
:1067C00095E0B5DFC63138F460E270E080E090E03B
:1067D000EBDFCF5FF7CFCF9108952F923F924F928B
:1067E0005F926F927F928F929F92AF92BF92CF9261
:1067F000DF92EF92FF920F931F93CF93DF93CDB76A
:10680000DEB762970FB6F894DEBF0FBECDBF8091A2
:106810007D05882309F4A1C06091AE0B7091AF0B88
:10682000072E000C880B990B0F94961411E0209101
:10683000B60B3091B70B4091B80B5091B90B0F9438
:10684000F71518160CF010E06091B00B7091B10BB9
:10685000072E000C880B990B0F9496142091BA0BFD
:106860003091BB0B4091BC0B5091BD0B0F94F715B1
:1068700018160CF412606091A20B7091A30B072EF6
:10688000000C880B990B0F9496142091A60B309155
:10689000A70B4091A80B5091A90B0F94F715181650
:1068A0000CF410681093C003C090870CD090880C33
:1068B000E090890CF0908A0C20E030E0A901C7013B
:1068C000B6010F94F41387FD05C020E030E040E0EE
:1068D0005FE304C020E030E040E05FEBC701B601B9
:1068E0000F941B130F946314CB010E940F85BC01FE
:1068F0008BEB93E00F940E1CC0908B0CD0908C0C03
:10690000E0908D0CF0908E0C20E030E0A901C701E2
:10691000B6010F94F41387FD05C020E030E040E09D
:106920005FE304C020E030E040E05FEBC701B60168
:106930000F941B130F946314CB010E940F85BC01AD
:1069400086EB93E00F940E1C8FE89CE00E94408938
:10695000BC018EEA93E00F940E1C0E943668182F3B
:1069600081E06ED62091C00327FF03C048E00CE011
:1069700002C042E102E08091010490E0449774F487
:1069800080910304841750F027FD68C281E596E1E9
:106990007C0123E060E58DEC93E0E8D88091010470
:1069A0008431B0F480910304823090F0112309F413
:1069B00058C28091AC0B882309F453C281EC95E155
:1069C0007C0102E123E042E068E68DEC93E0CED862
:1069D000809101048C3108F06CC156EB852E5BE090
:1069E000952E6EEA262E6BE0362E2EE02E87C12CD9
:1069F000D12C73E0A72EB12CFC2C8091C00390E029
:106A00000C2C02C0959587950A94E2F7082F017027
:106A1000F4014080518062807380F1016081718156
:106A2000072E000C880B990B0F9496146F87788BA8
:106A3000898B9A8B80910104843100F58091030445
:106A40008830E0F0C114D10409F411C260E2F6010B
:106A5000E150FD4F2081EF2DE1700E2E000CFF0B59
:106A6000EE0FFF1F002309F4FFC1E354FA4EE59037
:106A7000F4900CE048E08DEC93E078D8809101042C
:106A80008830B0F5F601E05CF44F8081111102C04E
:106A900081112EC020E030E040E05FE36F8578890F
:106AA00089899A890F941B130F946314CB010E9458
:106AB000D9847C01FC018081803209F0DCC1F701BE
:106AC0008181803209F0D5C101E0902F990F900F9C
:106AD00067E08E858F5F891BF3DDC501801B9109FF
:106AE0008E0D9F1D5EDE69E070E080E090E05CDE70
:106AF000809101048C3180F580910304853160F12F
:106B000020E030E040E05FE3C301B2010F941B13CB
:106B10000F946314CB010E94D9847C01FC01808115
:106B2000803209F0ACC1F7018181803209F0A5C142
:106B300001E0902F990F900F6CE18E858F5F891B7C
:106B4000BFDDC501801B91098E0D9F1D2ADE69E006
:106B500070E080E090E028DEFFEFCF1ADF0A2E859C
:106B6000285E2E8744E0840E911C52E0250E311CD5
:106B70002E3309F041CF4090A60B5090A70B6090A8
:106B8000A80B7090A90B8091A20B9091A30B209160
:106B900001042830B8F52091860B111102C0211193
:106BA00031C0BC01990F880B990B0F94961420E00B
:106BB00030E040E05FE30F941B130F946314CB01AC
:106BC0000E94D9847C01FC018081803209F05BC184
:106BD000F7018181803209F054C101E0902F990FB3
:106BE000900F892F819567E0845A6ADD83E090E0F9
:106BF000801B91098E0D9F1DD4DD69E070E080E05F
:106C000090E0D2DD809101048C3188F580910304FD
:106C1000853168F120E030E040E05FE3C301B2017C
:106C20000F941B130F946314CB010E94D9847C0131
:106C3000FC018081803209F02AC1F7018181803214
:106C400009F023C101E0902F990F900F892F8195B2
:106C50006CE1845A35DD83E090E0801B91098E0D54
:106C60009F1D9FDD69E070E080E090E09DDD8091F8
:106C700001048C31F0F4809103048531D0F000914F
:106C8000AC0B0023B1F06CE187E61ADDF4E60F9F50
:106C9000C001112481589F4F6FEF70E00F942717A8
:106CA000CB010E94D9847DDD65E270E080E090E058
:106CB0007BDD8091ED0783FF27C080911D0688232F
:106CC00019F1809101048433F8F4809103048A322D
:106CD000D8F007E028E04AE26AE28DEC93E07DD943
:106CE00005E022E04CE262E38DEC93E076D904E02B
:106CF0002AE041E36AE28DEC93E01FD94BE262E3C4
:106D00008DEC93E00E94752D80910104853328F469
:106D100080910304813308F0BCC00E946E68823009
:106D200048F090910104943328F490910304923335
:106D300008F0B7C0809101048F3208F05EC08091E6
:106D40000304883208F459C00F9496102B013C01BB
:106D50008CE3C82ED12CE12CF12CC301B201A70188
:106D600096010F943A17CA01B901A70196010F9431
:106D70003A17CA01062FD72E4901AE014F5F5F4F68
:106D80007A0150E8451651E5550651E06506710453
:106D900008F4A1C0B90128E130E040E050E00F94D0
:106DA0003A1729013A01DF920F93C40168E170E0BC
:106DB0000F9413179F938F935F924F928BEA95E1F5
:106DC0009F938F93FF92EF920F943D1C0FB6F89410
:106DD000DEBF0FBECDBF5AE04516510461047104F9
:106DE00008F0A3C098E0892F880F980F892F81950C
:106DF0006FE2855A65DCC701D4DC809101048632DC
:106E0000A0F4809103048E3180F008E020E84EE188
:106E100060E08DEC93E0E1D880910104863228F4A3
:106E2000809103048F3108F082C080910104823385
:106E300028F4809103048B3208F008C1809101048A
:106E4000813408F01FC180910304873308F41AC10C
:106E50006EE380E035DC812FAADC14C18DE296E17F
:106E600097CD87EF95E1ACCDE754FA4E00CE68E0C0
:106E7000EECD02E02ACE03E028CE02E05ACE03E0B7
:106E800058CE02E0ABCE03E0A9CE02E0DCCE03E0B8
:106E9000DACE04E02AE441E366E38DEC93E04DD8DA
:106EA0003CCFF8E48F9FB0011124072E000C880B13
:106EB000990B0F9496142AE037ED43E25CE30F94AC
:106EC00032160F946814262F02E042E367E38DEC3C
:106ED00093E083D82FCF84E68816910498F4DF924C
:106EE0000F933F932F9381EA95E19F938F93FF92A6
:106EF000EF920F943D1C0FB6F894DEBF0FBECDBFCE
:106F000095E071CFDF920F933F932F9389E995E13D
:106F10009F938F93FF92EF920F943D1C0FB6F894BE
:106F2000DEBF0FBECDBF96E05ECF99E05CCF60E0E4
:106F30008DEC93E00E948C2D65E283E0C1DB68E577
:106F400070E080E090E030DC65E28BE0B9DB11239B
:106F500021F08BEB93E025DC1BC08091990C80FD28
:106F6000F8CF3BEBE32E33E0F32EF70161917F0185
:106F7000662371F06F3234F4062E000C770B880B09
:106F8000990B04C06FE370E080E090E00DDCEDCF82
:106F900065E288E295DB69E570E080E090E004DC82
:106FA00065E280E38DDB112321F086EB93E0F9DBD2
:106FB0001BC08091990C81FDF8CF26EBE22E23E0D7
:106FC000F22EF70161917F01662371F06F3234F484
:106FD000062E000C770B880B990B04C06FE370E052
:106FE00080E090E0E1DBEDCF65E28DE469DB6AE50E
:106FF00070E080E090E0D8DB65E285E561DB11239D
:1070000021F08EEA93E0CDDB1BC08091990C82FDCC
:10701000F8CF9EEAE92E93E0F92EF70161917F0106
:10702000662371F06F3234F4062E000C770B880B58
:10703000990B04C06FE370E080E090E0B5DBEDCF2A
:1070400061E08DEC93E00E948C2DEFCE83E0F8D2CE
:1070500062E383E035DB66E070E080E090E0A4DB93
:1070600081E0EED262E38CE02BDB80914D029091C7
:107070004E020E94D98495DB65E270E080E090E0EA
:1070800093DBDCCE62960FB6F894DEBF0FBECDBFA9
:10709000DF91CF911F910F91FF90EF90DF90CF90F4
:1070A000BF90AF909F908F907F906F905F904F9028
:1070B0003F902F9008950F931F93CF93DF93CDB7F9
:1070C000DEB728970FB6F894DEBF0FBECDBF8A019A
:1070D00023E0660F771F2A95E1F7680F791F48E0D4
:1070E00050E0CE0101960F94711B29813A81F8017D
:1070F000808191812817390790F08217930760F0FB
:107100009C818281981758F081E090E03B81238137
:10711000231738F080E005C081E090E002C08FEFD7
:107120009FEF28960FB6F894DEBF0FBECDBFDF915C
:10713000CF911F910F910895EF92FF920F931F939C
:10714000CF93DF93EC018B017A018A859B858617AB
:10715000970729F088819981D0D91B870A8788856C
:107160009985019681F00E811F81B70188819981EF
:10717000C1D9080F111D888599858017910718F4CA
:1071800081E090E010C06E818A81680F97014C8188
:1071900088819981C3D82E813F81280F311D3F837B
:1071A0002E8380E090E0DF91CF911F910F91FF90AF
:1071B000EF9008954F925F926F927F928F929F927D
:1071C000AF92BF92CF92DF92EF92FF920F931F93F5
:1071D000CF93DF93CDB7DEB72D970FB6F894DEBF10
:1071E0000FBECDBF6C012A013B01490158011B862E
:1071F0001C86CE0101967C0188E0F70111928A95E8
:10720000E9F7DB01CA0127E0B695A7959795879521
:107210002A95D1F79A838983F42FFF77FD878F2FE3
:1072200080588B838C831A8619864F3F51056105E0
:10723000710509F018F460E070E026C06091C303A6
:107240007091C4038E01075F1F4F97014BE558E310
:107250008091C1039091C2030E94956597FDEBCF89
:1072600069857A8583E0660F771F8A95E1F78091BB
:10727000C1039091C203680F791F48E050E0C70135
:107280000F94711B6F8178856115710519F44B8618
:10729000B60106C0C616D70619F08D8580688B87A3
:1072A000AE01455F5F4FC401F50119952D960FB6EC
:1072B000F894DEBF0FBECDBFDF91CF911F910F912C
:1072C000FF90EF90DF90CF90BF90AF909F908F9006
:1072D0007F906F905F904F9008956F927F928F9202
:1072E0009F92AF92BF92CF92DF92EF92FF920F9355
:1072F0001F93CF93DF9300D01F92CDB7DEB76C0101
:107300007B013A015901480119821A821B821C82B1
:10731000AE014F5F5F4FB301C7010E94F5657C016D
:1073200049815A816B817C81411551056105710547
:1073300029F084019501C6013DDFE6CF0F900F9043
:107340000F900F90DF91CF911F910F91FF90EF90D1
:10735000DF90CF90BF90AF909F908F907F906F9075
:10736000089521E02093C503E1ECF3E0918380834D
:107370007383628380E090E008957F92AF92BF9222
:10738000CF92DF92EF92FF920F931F93CF93DF93F1
:10739000CDB7DEB72C970FB6F894DEBF0FBECDBFCA
:1073A0006C01762EF72F842FE52FB901A801D601A5
:1073B0001496AD90BC9015979091C50391110AC099
:1073C00027EF36E1482F672DC6010E94C53180E0C6
:1073D00090E018C0DA82C9827B82FC838D83EE83C1
:1073E00018861F82FA86E9861C861B860CE918E33C
:1073F0009E012F5F3F4FC501DDDEB501C6017DD87F
:107400008F8198852C960FB6F894DEBF0FBECDBF46
:10741000DF91CF911F910F91FF90EF90DF90CF9070
:10742000BF90AF907F900895CF92DF92EF92FF923E
:107430000F931F93CF93DF93CDB7DEB72C970FB683
:10744000F894DEBF0FBECDBF7C01C901F701C48037
:10745000D5802091C503211108C027ED36E1C70171
:107460000E94C53180E090E01BC0FA82E9826B8304
:107470007C834D835E8318861F821A8709871C864A
:107480001B860CE918E39E012F5F3F4F4FE855E63E
:10749000BC01C60122DFB601C7012FD88F819885B4
:1074A0002C960FB6F894DEBF0FBECDBFDF91CF9103
:1074B0001F910F91FF90EF90DF90CF900895CF92A2
:1074C000DF92EF92FF920F931F93CF93DF93CDB78D
:1074D000DEB72C970FB6F894DEBF0FBECDBF7C0190
:1074E000C901F701C480D5802091C503211108C0CE
:1074F00027EB36E1C7010E94C53180E090E01CC057
:10750000FA82E9826B837C834D835E8318861F82B7
:107510001A8709871C861B860CE918E39E012F5FDA
:107520003F4F42E955E6BC01C601D7DEB601C701AF
:107530000E947D328F8198852C960FB6F894DEBF1D
:107540000FBECDBFDF91CF911F910F91FF90EF90B4
:10755000DF90CF900895CF93DF93EC01262F4CADB1
:107560006BAD04960E9470312BAD082E000C990B68
:10757000820F911D8BAF81E090E0DF91CF91089554
:107580000F939CE0899F802D112421E0280F2093E8
:10759000C803845F8093C70390E002964091010482
:1075A00050E08417950714F480E033C0822F90E0F8
:1075B0002091030430E082179307B4F76623A9F003
:1075C00061E08DEC93E00E948C2D4091C8034E5FEA
:1075D0000BE020E860E08DEC93E00E94ED2F60E08E
:1075E0008DEC93E00E948C2D05C061E08DEC93E062
:1075F0000E948C2D6091C703809101046817A0F24E
:107600009091C80380910304891770F280E058D8E4
:1076100081E00F910895CF93DF93FC0185ADEF01D9
:107620002496811105C081E085AFCE010E942C2DEA
:10763000CE01DF91CF910C94632D6FEF7FEF94C853
:10764000482F50E02091C603022E000C330B421746
:10765000530781F08093C603813031F463E27FE108
:107660008DEC93E00C947D3263E377E18DEC93E055
:107670000C947D320895EF92FF920F9389EC93E082
:10768000CADF85EEE82E8CE1F82E00E428E040E029
:1076900060E08DEC93E00E94B62D61E373E08DEC29
:1076A00093E00E947D3221E033E041E169E38DEC1B
:1076B00093E00E948E3161EA7BE08DEC93E00E94C2
:1076C0007D3227E033E04CE16AE38DEC93E00E94E9
:1076D0008E316CEF7EE08DEC93E00E947D3227E1ED
:1076E00033E049E26BE38DEC93E00E948E316CEF66
:1076F0007EE08DEC93E00E947D3223E233E04EE3A6
:107700006DE38DEC93E00E948E3125E233E04EE391
:1077100062E48DEC93E00E948E318DEC93E00E9448
:10772000672D8111AECF64EC79E080E090E00E949B
:107730006F8463E377E18DEC93E00F91FF90EF901E
:107740000C947D3261E085EE9CE195DF64EC79E09C
:1077500080E090E00C946F84CF92DF92EF92FF92E2
:107760000F931F93CF93DF93EDDFC091CD03009173
:10777000CE03D0E0BE016853710977FF02C06F5F8E
:107780007F4F75956795D62E89EC93E044DFCE0147
:10779000C09796958795182FC257D109D695C7954A
:1077A0004EEEC42EC00EDAEFD00F80E6E82E8CE14C
:1077B000F82E03E127E04CE06D2D8DEC93E00E9464
:1077C000B62D83E03DDF25E233E04C2D612F8DECBB
:1077D00093E00E948E312EE233E04D2F6C2F8DEC22
:1077E00093E00E948E318DEC93E00E94672D811111
:1077F000DCCF64EC79E080E090E0DF91CF911F91E5
:107800000F91FF90EF90DF90CF900C946F8460E029
:1078100070E083E29FE1A5CD1F93CF93DF93C091EA
:10782000CE03C695C69589EC93E0F5DEDC2FDD0F1F
:107830001D2F1C0F83E004DF6C2F80E00E9460335B
:1078400087E895E00E94D1336D2F80E00E9460337D
:1078500084E297E1F2DE612F80E00E94603387E1ED
:1078600097E1EBDE8DEC93E00E94672D8111E2CF72
:10787000DF91CF911F9108950895CF93DF93C62F85
:107880006CE0869F602D112481E0860F8093C803F1
:10789000645F6093C703462F50E04E5F5F4F2091B7
:1078A000010430E0421753070CF44FC090E02091E0
:1078B000030430E0821793070CF047C08EE30E9468
:1078C000603365E470E080E090E00E94D43361E3CF
:1078D0006C0F062E000C770B880B990B0E94D4338B
:1078E00060E270E080E090E00E94D433D0E0FE01DE
:1078F000EE0FFF1FEE0FFF1FEA54F44F60817181FE
:10790000828193810F946314CB010E94D9840E94D9
:10791000D1336FE270E080E090E00E94D4330E94A7
:107920003668811106C0FE01E05CF44F8081811150
:107930000CC0CC0FDD1FC255D44F888199810E94A5
:10794000D984DF91CF910C94D133DF91CF910895F9
:10795000CF92DF92EF92FF920F931F93CF93DF931B
:107960001F921F92CDB7DEB77B01622F498308DEDD
:107970004981882309F444C0442311F101151105FC
:10798000F9F4C7010E94656726E130E0281B310940
:1079900037FF02C02F5F3F4F3595279530E82158BC
:1079A000822F830F87FD0DC060E270E080E090E0E1
:1079B0002A8339830E94D433398131502A81F0CF10
:1079C00030E8C32ED12CB601C7010E94B433760132
:1079D000E81AF90A0115110511F41E2D07C0FF243C
:1079E000B701C8010E9497331E2D181B173040F0B5
:1079F00060E270E080E090E00E94D433181BF6CF84
:107A00000F900F90DF91CF911F910F91FF90EF900A
:107A1000DF90CF9008950F93CF93DF93982F862F09
:107A2000EA01692FADDD882331F168E770E0CE010E
:107A30000E94B433C8E7C81BC73040F060E270E072
:107A400080E090E00E94D433C81BF6CF6091C7035A
:107A50008AE70E946033602F000F770B880B990B29
:107A60000E94D43360E270E080E090E0DF91CF913B
:107A70000F910C94D433DF91CF910F910895CF9251
:107A8000DF92EF92FF920F931F93CF93DF93982F84
:107A9000862F6A017901692F73DD882309F447C0B5
:107AA000C701002321F00E946567182F03C00E94C0
:107AB0004467182FC4E1D0E0C11BD1098C2F880F77
:107AC000C80FCC0FD0E0BE01C6010E94B433C81B62
:107AD0006AE370E080E090E00E94D433C73040F069
:107AE00060E270E080E090E00E94D433C81BF6CFE3
:107AF0008AEF189F802D11246091C70380580E943F
:107B00006033C701002349F0DF91CF911F910F919E
:107B1000FF90EF90DF90CF9090CDDF91CF911F91AC
:107B20000F91FF90EF90DF90CF900C94D133DF91C5
:107B3000CF911F910F91FF90EF90DF90CF9008951C
:107B4000BF92CF92DF92EF92FF920F931F93CF934A
:107B5000DF936C017B010E946567C82FC7010E94FB
:107B6000446704E110E0081B11098C2F90E0BB244E
:107B7000B394081719071CF0B12CC5E201C0CFE17E
:107B80002C2F30E0A9014E5F5F4F8091010490E0FF
:107B90004817590744F0295031098091030490E0B7
:107BA00082179307BCF5D0E0E114F104D9F16AE340
:107BB00070E080E090E00E94D433BB2081F0C45F8D
:107BC00080910104C81770F12C2F30E02950310941
:107BD0008091030490E0821793071CF423C0DD23F7
:107BE00009F1802F880F800F6C2F880F0E9460335F
:107BF00060E270E080E090E00E94D433C701DF9142
:107C0000CF911F910F91FF90EF90DF90CF90BF9099
:107C10000C94D1336C2F80E00E946033C6010DDDDF
:107C2000D1E0C2CFDF91CF911F910F91FF90EF90E4
:107C3000DF90CF90BF900895EF92FF920F93CF9374
:107C4000DF93D82FC62F7901682F8C2F99DC8823DA
:107C5000F1F0002331F062E070E080E090E00E94FB
:107C6000D4332D2F4C2F65E1C7010E94E7676EE7E3
:107C700070E00E949733CEE7C81BC73040F060E247
:107C800070E080E090E00E94D433C81BF6CFDF9113
:107C9000CF910F91FF90EF900895CF92EF920F93B5
:107CA000CF93DF93C9ECD3E01B821A8286E493E082
:107CB00099838883CC24CA94EE24EA9406E427E4CA
:107CC00048E460E172E0CE010E943D3382E593E03A
:107CD00099838883DF91CF910F91EF90CF90089592
:107CE0009091050194709093030187FD76C0A3984D
:107CF00090910501909594709093030190910501E6
:107D0000947090930301982F990F86FD72C0A398E9
:107D10008091050180958470809303018091050115
:107D2000847080930301292F220F96FD60C0A398D1
:107D300080910501809584708093030180910501F5
:107D4000847080930301922F990F26FD4EC0A39853
:107D500080910501809584708093030180910501D5
:107D6000847080930301292F220F96FD3CC0A398B5
:107D700080910501809584708093030180910501B5
:107D8000847080930301922F990F26FD2AC0A39837
:107D90008091050180958470809303018091050195
:107DA000847080930301292F220F96FD18C0A39899
:107DB0008091050180958470809303018091050175
:107DC00084708093030126FD16C0A398809105015D
:107DD00080958470809303010895A39A89CFA39A14
:107DE000E7CFA39AD5CFA39AC3CFA39AB1CFA39A33
:107DF0009FCFA39A8DCFA39A80910501809584701F
:107E00008093030108952F923F925F927F929F92F9
:107E1000AF92BF92CF92DF92EF92FF920F931F9398
:107E2000CF93DF937C011B01942E69018AE04817F0
:107E300009F47BC0A5E14A134EC0DB011296ED9117
:107E4000FC9113971281C681D781A49A88E28A9502
:107E50000000E9F700EE010F80E1582E510E98E284
:107E6000792E88EF3DDF872D8A950000E9F71032E3
:107E700008F046C0812F8077806832DF812F82959D
:107E8000807F2EDF872D8A950000E9F780E828DFC4
:107E900080E026DF872D8A950000E9F78AEF20DF52
:107EA000872D8A950000E9F75E01B0E1AB0EB11CA9
:107EB0008881807F15DF89918295807F11DFCA15C7
:107EC000DB05B1F7872D8A950000E9F71F5F0F5F8B
:107ED0001511C7CFA4989601492DB101C701DF91B3
:107EE000CF911F910F91FF90EF90DF90CF90BF90B7
:107EF000AF909F907F905F903F902F900C94F02ECA
:107F0000802F80778068ECDE802F8295807FE8DE8E
:107F1000872D8A950000E9F780E8E2DE80E8E0DE60
:107F2000872D8A950000E9F7B9CF9C9AA4989B9A6F
:107F3000A3988091040184608093040180910501DD
:107F40008095847080930301A49AC8E28C2F8A954F
:107F50000000E9F788E790E00E940D2E88EFC0DE70
:107F60008C2F8A950000E9F780E2BADE80E0B8DE67
:107F70008C2F8A950000E9F780E0B2DE80E8B0DE61
:107F80008C2F8A950000E9F780E0AADE80E1A8DE68
:107F90008C2F8A950000E9F78FE090E00E940D2E6B
:107FA00080E29EDE80E49CDE8C2F8A950000E9F75B
:107FB00080E296DE80E694DECA950000E9F710E0E4
:107FC000D8E208E2812F807780688ADE812F82954F
:107FD000807F86DE8D2F8A950000E9F780E880DEBD
:107FE00080E07EDE8D2F8A950000E9F78AEF78DE4B
:107FF0008D2F8A950000E9F7C0E280E071DE80E015
:108000006FDE9D2F9A950000E9F7C150B1F788EF18
:1080100067DE802F8A950000E9F71F5F103209F0B4
:10802000D1CF80E05DDE80EC5BDE88E28A950000E7
:10803000E9F7A49850CF0E94817541E050E060E0DC
:1080400070E0811103C040E050E0BA01409379052F
:1080500050937A0560937B0570937C0510925205CE
:1080600081E080932C0583E080931F020895CF92D6
:10807000DF92EF92FF920F931F93CF93DF930E94B3
:108080007E766C0161E081E00E940165C09152053D
:10809000D0E081E0C81AD108C11117C080911B053A
:1080A000811104C00E94316881119BC080911F0220
:1080B000882359F081E090911B05911180E004E044
:1080C00024E04FE358E26D2FA6DC60EE77E087E610
:1080D00097E00E94677C8091E0078F3201F18091E8
:1080E000ED0783FF1CC0C130C1F480911B058130B6
:1080F00021F40E94316881117CC080911F02882385
:1081000061F081E090911B05913009F080E000E280
:108110002EE34BE358E26D2F7EDC92E001C091E04C
:1081200080911F02882309F454C0760111E01C0FCE
:108130008FEFE816F80609F44CC0C91345C060E09B
:1081400070E0C7010E94A7729091ED0780911B0516
:1081500094FF22C08C1354C00E943168882309F414
:108160004FC080EE97E00E942B751092520582E07E
:1081700090E0A0E0B0E08093790590937A05A09319
:108180007B05B0937C0581E080932C0510927E05E1
:1081900083E080931F0250C08C1304C00E9431689A
:1081A00081113DC080911F02882361F081E0909190
:1081B0001B059C1380E000E02AEE35E14FE158E218
:1081C0006D2F3ADD912F01C09F5F81E0E81AF10821
:1081D000AFCFDF5FCF5FD53009F05ECF90931A0548
:1081E0002BC00E94516480912C05882309F45ECF36
:1081F00023C021DF80912C05882309F47ECF1CC089
:1082000080911F028823F1F281E090911B059C135D
:1082100080E001E02AEE35E14DE258E2D1CF80EE78
:1082200097E00E9432710E944B640E94E86C80913A
:108230002C05882309F4B6CFDF91CF911F910F91C0
:10824000FF90EF90DF90CF900895CF93DF93EC01F4
:10825000CB01BA010F9496142AE037ED43E25CE3B8
:108260000F943216688379838A839B83DF91CF9141
:108270000895CF93DF93EC01CB01BA010F949614CC
:10828000688379838A839B83DF91CF910895CF930D
:10829000DF93EC01CB01BA010F94961420E030E09B
:1082A00048EC52E40F943216688379838A839B8367
:1082B000DF91CF910895CF93DF93EC01CB01BA0109
:1082C0000F94961420E030E048EC52E40F943216FC
:1082D0000F946814688379838A839B83DF91CF919D
:1082E0000895CF93DF93EC01CB01BA010F9496145C
:1082F0002AE037ED43E25CE30F943216688379831A
:108300008A839B83DF91CF910895CF93DF93EC0114
:10831000CB01BA010F9496142AE037ED43E25CE3F7
:108320000F943216688379838A839B83DF91CF9180
:10833000089565E271E48EED91E40C94656469E35F
:1083400071E488E592E40C94656467E471E48BEF72
:1083500091E40C9465646BE571E484E792E40C9419
:10836000656461E771E488E192E40C94656465E812
:1083700071E481EC91E40C9465640C9432E50C9406
:1083800098E5CF93DF9300D01F92CDB7DEB70F945F
:1083900096142AE037ED43E25CE30F9432166983CA
:1083A0007A838B839C83CE0101960E947F880F90F5
:1083B0000F900F900F90DF91CF910895CF93DF939F
:1083C00000D01F92CDB7DEB70F9496142AE037ED98
:1083D00043E25CE30F94321669837A838B839C8338
:1083E000CE0101960E9478850F900F900F900F900C
:1083F000DF91CF910895CF93DF9300D01F92CDB737
:10840000DEB70F94961420E030E048EC52E40F946D
:10841000321669837A838B839C83CE0101960E94F6
:1084200026870F900F900F900F90DF91CF910895B6
:10843000CF93DF9300D01F92CDB7DEB70F94961481
:108440002AE037ED43E25CE30F94321669837A83C6
:108450008B839C83CE0101960E94DE870F900F9044
:108460000F900F90DF91CF910895CF92DF92EF920E
:10847000FF926B017C0120E030E0A9010F94F4131E
:1084800087FD05C020E030E040E05FE304C020E06D
:1084900030E040E05FEBC701B6010F941B130F946F
:1084A0006314CB01FF90EF90DF90CF900C94D984B0
:1084B0000F949614DACFCF93DF9300D01F92CDB7ED
:1084C000DEB70F9468140F94941469837A838B83B6
:1084D0009C83CE0101960E9426870F900F900F90EB
:1084E0000F90DF91CF9108950F94961420E030E023
:1084F00048EC52E40F943216DECFCF93DF931F92F5
:108500001F92CDB7DEB789839A830E94806340E0D3
:1085100050E0BA0189819A810F900F90DF91CF913D
:108520000C9426649091760C891302C00C9432E569
:10853000089580E0F7CF81E0F5CFCF93DF9390915E
:10854000760C891304C0DF91CF910C9498E590E0EC
:10855000EC01CC0FDD1FCC0FDD1FCE5DD24F880F9D
:10856000991F880F991FFC01EE59F24F208131812C
:108570004281538160E070E080E89FE30F94FB1339
:10858000688379838A839B83DF91CF91089580E00C
:10859000D4CF81E0D2CF0F93CF93DF9361E081E01E
:1085A0000E940165C0915205D0E0C11119C08091AF
:1085B0001B05811104C00E9431688111AAC08091FD
:1085C0001F02882309F45DC081E090911B05911181
:1085D00080E004E024E041E758E26D2F1CDA51C04E
:1085E000C130D1F480911B05813021F40E943168A3
:1085F000811197C080911F02882309F442C081E055
:1086000090911B05913009F080E003E02EE348E6ED
:1086100058E26D2F00DA35C0C230C9F480911B05D5
:10862000823021F40E943168811184C080911F0240
:10863000882339F181E090911B05923009F080E0A8
:1086400003E02EE34BE558E26D2FE5D91AC0C330A5
:10865000C1F480911B05833021F40E94316881119F
:1086600072C080911F02882361F081E090911B0508
:10867000933009F080E003E02EE346E558E26D2FE9
:10868000CAD90E940F6481111CC0C430E1F48091EA
:108690001B05843021F40E94316881115DC08091F6
:1086A0001F02882309F461C081E090911B0594307A
:1086B00009F080E003E02EE34DE458E26D2FABD9E2
:1086C00054C084E001C085E0C8131AC080911B0526
:1086D0008C1304C00E943168811149C080911F022F
:1086E000882369F081E090911B059C1380E003E0F2
:1086F0002EE344E458E26D2F8ED98C2F01C08C2FCD
:10870000DF5FCF5FD53009F050CF8F5F80931A05C0
:1087100036C00E94516480912C05882309F44FCF04
:108720002EC08AED96E4E9DE80912C05882309F4B9
:1087300061CF25C08BE69BE4E0DE80912C05882389
:1087400009F474CF1CC083EE98E4D7DE80912C0529
:10875000882309F486CF13C08DE79EE4CEDE809196
:108760002C05882309F49BCF0AC085E0C9CF86E396
:1087700094E4C3DE80912C05882309F4AFCFDF9108
:10878000CF910F9108952F923F924F925F926F92E7
:108790007F928F929F92AF92BF92CF92DF92EF9291
:1087A000FF920F931F93CF93DF93CDB7DEB7279739
:1087B0000FB6F894DEBF0FBECDBF1C017F836E8362
:1087C0009C2C8D2CA982CA01B9010F9463149B01C2
:1087D000AC01EE81FF8160817181828193812A8366
:1087E0003B834C835D830F9463142A813B814C81CE
:1087F0005D815B016C01A21AB30AC40AD50AC801E3
:10880000B7010F9463142A813B814C815D817B0108
:108810008C01E21AF30A040B150BF981FF938F9276
:108820009F928FE9882E81E4982E6E817F81C1010D
:108830000E94A2630F900F900F9027960FB6F894A6
:10884000DEBF0FBECDBFDF91CF911F910F91FF9083
:10885000EF90DF90CF90BF90AF909F908F907F90E0
:108860006F905F904F903F902F9008956F927F92FE
:108870008F929F92AF92BF92CF92DF92EF92FF9230
:108880000F931F93CF93DF9300D01F92CDB7DEB726
:1088900061E081E00E94016560905205712C6110D9
:1088A00019C080911B05811104C00E94316881119B
:1088B00069C180911F02882309F45BC181E0909116
:1088C0001B05911180E004E024E04FEF5AE2672D90
:1088D000A2D84FC181E068122BC080911B05813066
:1088E00021F40E943168811155C180911F028823B3
:1088F00009F43FC111E080911B05813009F010E0BF
:108900008091C70C9091C80CA091C90CB091CA0C71
:1089100089839A83AB83BC83CE0101960E947885BC
:1089200000E09C0147EE5AE2672D812FA8D821C1B3
:1089300082E068122BC080911B05823021F40E94D6
:108940003168811158C180911F02882309F411C137
:1089500011E080911B05823009F010E08091CB0C72
:108960009091CC0CA091CD0CB091CE0C89839A83C0
:10897000AB83BC83CE0101960E94788500E09C0108
:108980004FEC5AE2672D812F7AD8F3C083E068124A
:1089900028C080911B05833021F40E943168811129
:1089A0005BC180911F02882309F4E3C011E080912C
:1089B0001B05833009F010E0E091760C88E0E89F19
:1089C000F0011124E554F54F60817181828193811A
:1089D0004CDD00E09C014BEB5AE2672D812F4FD814
:1089E000C8C084E0681224C080911B05843021F443
:1089F0000E94316881114EC180911F02882309F4C1
:108A0000B8C011E080911B05843009F010E060913E
:108A1000BB0A7091BC0A8091BD0A9091BE0A25DD07
:108A200000E09C0143EA5AE2672D812F28D8A1C0BB
:108A300085E0681224C080911B05853021F40E94D6
:108A4000316881113FC180911F02882309F491C0D0
:108A500011E080911B05853009F010E06091C30A98
:108A60007091C40A8091C50A9091C60AFEDC00E0AC
:108A70009C014BE85AE2672D812F01D87AC086E02D
:108A8000681229C080911B05863021F40E9431684C
:108A9000811130C180911F02882309F46AC011E05E
:108AA00080911B05863009F010E0E091760C88E09B
:108AB000E89FF0011124E554F54F648175818681AA
:108AC0009781D3DC00E09C014BE75AE2672D812FB0
:108AD0000E943F3D4EC087E0681225C080911B0573
:108AE000873021F40E943168811122C180911F02D8
:108AF000882309F43EC011E080911B05873009F0FE
:108B000010E06091BF0A7091C00A8091C10A9091F3
:108B1000C20AABDC00E09C0147E65AE2672D812FD8
:108B20000E943F3D26C088E0681223C080911B054B
:108B3000883021F40E943168811112C180911F0296
:108B40008823B9F011E080911B05883009F010E00E
:108B50006091C70A7091C80A8091C90A9091CA0AA7
:108B600084DC00E09C0143E55AE2672D812F0E94DE
:108B70003F3D7394639485E0781291CE89E08093B1
:108B80001A0505C10E94516480912C05882309F4BF
:108B900090CEFDC020E030E048EC52E46091C70C7C
:108BA0007091C80C8091C90C9091CA0C0F94321628
:108BB0000F9463141F921F921F92A9E98A2EA1E4B9
:108BC0009A2E5B016C011CE3E12E16E8F12E01E008
:108BD00010E020E030E0A90167EC7CE083EF9AE24E
:108BE0000E94A2630F900F900F9080912C05882314
:108BF00009F47BCECCC020E030E048EC52E4609138
:108C0000CB0C7091CC0C8091CD0C9091CE0C0F942C
:108C100032160F9463141F921F921F92E9E98E2E51
:108C2000E1E49E2E5B016C011CE3E12E16E8F12EBF
:108C300001E010E020E030E0A9016BEC7CE08BED7E
:108C40009AE20E94A2630F900F900F9080912C05E2
:108C5000882309F478CE9BC081E00E942668609149
:108C6000760C88E0689FB00111246554754FA12CE3
:108C7000C12CD12CE12CF12C08E413E420E030E0ED
:108C8000A90185EC9AE27FDD80912C05882309F407
:108C900088CE7DC081E00E942668A12CC12CD12CF9
:108CA000E12CF12C08E413E420E030E0A9016BEBA7
:108CB0007AE08FEA9AE267DD80912C05882309F437
:108CC0009BCE65C081E00E942668A12CC12CD12CCE
:108CD000E12CF12C08E413E420E030E0A90163EC7E
:108CE0007AE087E99AE24FDD80912C05882309F428
:108CF000AACE4DC081E00E9426686091760C88E083
:108D0000689FB00111246154754FA12CC12CD12C46
:108D1000E12CF12C08E413E420E030E0A90183E821
:108D20009AE231DD80912C05882309F4B3CE2FC05F
:108D300081E00E942668A12CC12CD12CE12CF12CC1
:108D400008E413E420E030E0A9016FEB7AE081E76A
:108D50009AE219DD80912C05882309F4C7CE17C04B
:108D600081E00E942668A12CC12CD12CE12CF12C91
:108D700008E413E420E030E0A90167EC7AE08DE537
:108D80009AE201DD80912C05882309F4D7CE0F905B
:108D90000F900F900F90DF91CF911F910F91FF9047
:108DA000EF90DF90CF90BF90AF909F908F907F908B
:108DB0006F900895AF92CF92DF92EF92FF920F9350
:108DC0001F93CF93DF9361E081E00E940165D09112
:108DD0005205C0E0D1111AC080911B05811104C059
:108DE0000E94316881112AC180911F02882309F4F1
:108DF0001CC181E090911B05911180E004E024E00A
:108E000041E45AE26C2F0E940B3D0FC1D13029F58D
:108E100080911B05813021F40E943168811116C1B7
:108E200080911F02882309F400C111E080911B0585
:108E3000813009F010E060916A0D70916B0D8091A6
:108E40006C0D90916D0D11DB00E09C0143E35AE243
:108E50006C2F812F0E943F3DE8C0D23029F58091D0
:108E60001B05823021F40E943168811109C1809173
:108E70001F02882309F4D9C011E080911B058230BC
:108E800009F010E060916E0D70916F0D8091700D82
:108E90009091710DEADA00E09C0145E25AE26C2FF4
:108EA000812F0E943F3DC1C0D33029F580911B0521
:108EB000833021F40E9431688111FCC080911F022F
:108EC000882309F4B2C011E080911B05833009F0BA
:108ED00010E06091720D7091730D8091740D9091FE
:108EE000750DC3DA00E09C0147E15AE26C2F812F37
:108EF0000E943F3D9AC0D43029F580911B058430F3
:108F000021F40E9431688111EFC080911F028823F3
:108F100009F48BC011E080911B05843009F010E04A
:108F20006091760D7091770D8091780D9091790D0B
:108F30009CDA00E09C0147E05AE26C2F812F0E94EE
:108F40003F3D73C0D53029F580911B05853021F454
:108F50000E9431688111E2C080911F02882309F4C8
:108F600064C011E080911B05853009F010E060912C
:108F70007A0D70917B0D80917C0D90917D0D75DA4D
:108F800000E09C0147EF59E26C2F812F0E943F3D8A
:108F90004CC0D63029F580911B05863021F40E9403
:108FA00031688111D5C080911F02882309F43DC02A
:108FB00011E080911B05863009F010E060918A0D68
:108FC00070918B0D80918C0D90918D0D4EDA00E09B
:108FD0009C014DEE59E26C2F812F0E943F3D25C030
:108FE000D73019F580911B05873021F40E94316834
:108FF0008111C7C080911F028823B9F011E08091D0
:109000001B05873009F010E060918E0D70918F0D77
:109010008091900D9091910D28DA00E09C0149ED2E
:1090200059E26C2F812F0E943F3DCF5FDF5FC5303B
:1090300009F0D0CE88E080931A05BBC00E9451642D
:1090400080912C05882309F4CFCEB3C081E00E9423
:109050002668A12CC12CD12CE12C10ECF12E09E7B3
:1090600014E420E030E040E85FE36AE67DE08AE374
:109070009AE289DB80912C05882309F4D1CE99C02E
:1090800081E00E942668A12CC12CD12CE12C10EC8F
:10909000F12E09E714E420E030E040E85FE36EE6FB
:1090A0007DE08CE29AE26FDB80912C05882309F445
:1090B000DECE7FC081E00E942668A12CC12CD12C7D
:1090C000E12C10ECF12E09E714E420E030E040E858
:1090D0005FE362E77DE08EE19AE255DB80912C054B
:1090E000882309F4EBCE65C081E00E942668A12C9C
:1090F000C12CD12CE12C10ECF12E09E714E420E076
:1091000030E040E85FE366E77DE08FE09AE23BDB3A
:1091100080912C05882309F4F8CE4BC081E00E9491
:109120002668A12CC12CD12CE12C10ECF12E09E7E2
:1091300014E420E030E040E85FE36AE77DE08FEF91
:1091400099E221DB80912C05882309F405CF31C0F9
:1091500081E00E942668A12CC12CD12CE12C10ECBE
:10916000F12E09E714E420E030E0A9016AE87DE08F
:1091700082EF99E208DB80912C05882309F413CF54
:1091800018C081E00E942668A12CC12CD12CE12CB2
:1091900010ECF12E09E714E420E030E0A9016EE8BC
:1091A0007DE083EE99E2EFDA80912C05882309F4C3
:1091B00021CFDF91CF911F910F91FF90EF90DF9022
:1091C000CF90AF9008956F927F928F929F92AF92BF
:1091D000BF92CF92DF92EF92FF920F931F93CF93A4
:1091E000DF9300D01F92CDB7DEB761E081E00E942F
:1091F000016560905205712C61101AC080911B05A9
:10920000811104C00E9431688111BFC080911F028A
:10921000882309F4B2C081E090911B05911180E090
:1092200004E024E049E359E2672D0E940B3DA5C00C
:1092300021E0621225C080911B05813021F40E943B
:1092400031688111AAC080911F02882309F495C05A
:1092500011E080911B05813009F010E06091060D4E
:109260007091070D8091080D9091090DFED800E0D6
:109270009C0149E259E2672D812F0E943F3D7DC04C
:1092800082E0681225C080911B05823021F40E9483
:10929000316881119CC080911F02882309F46DC040
:1092A00011E080911B05823009F010E060910A0DF9
:1092B00070910B0D80910C0D90910D0DD6D800E0A2
:1092C0009C0149E159E2672D812F0E943F3D55C025
:1092D00023E062122CC080911B05833021F40E9490
:1092E000316881118EC080911F02882309F445C026
:1092F00011E080911B05833009F010E080910E0D84
:1093000090910F0DA091100DB091110D89839A834A
:10931000AB83BC83CE0101960E94DE8700E09C01F6
:1093200049E059E2672D812F0E943F3D26C084E02D
:10933000681223C080911B05843021F40E9431689B
:10934000811199C080911F028823B9F011E08091AA
:109350001B05843009F010E06091120D7091130D1F
:109360008091140D9091150D80D800E09C0149EF7B
:1093700058E2672D812F0E943F3D7394639425E04E
:1093800072123ACF70921A058FC00E945164809178
:109390002C05882309F43ACF87C081E00E94266813
:1093A000A12CC12CD12CE12C10E8F12E07E714E4FC
:1093B00020E030E040E85FE366E07DE081E399E2B1
:1093C000E2D980912C05882309F43DCF6DC081E05E
:1093D0000E942668A12CC12CD12CE12C10E8F12E82
:1093E00007E714E420E030E040E85FE36AE07DE076
:1093F00081E299E2C8D980912C05882309F44BCFEA
:1094000053C081E00E94266820E030E048EC52E43E
:1094100060910E0D70910F0D8091100D9091110DB6
:109420000F9432160F9463145B016C012AE0A21AA8
:10943000B108C108D1081F921F921F9291EB892E8B
:1094400091E4992E1EEAE12E12E8F12E01E010E0DF
:109450002AE030E040E050E06EE07DE081E199E21A
:109460000E94A2630F900F900F9080912C0588238B
:1094700009F439CF19C081E00E942668A12CC12CC3
:10948000D12CE12C10E8F12E07E714E420E030E0C5
:1094900040E85FE362E17DE081E099E274D9809188
:1094A0002C05882309F44ECF0F900F900F900F904A
:1094B000DF91CF911F910F91FF90EF90DF90CF90B0
:1094C000BF90AF909F908F907F906F9008952F9254
:1094D0003F924F925F926F927F928F929F92AF9244
:1094E000BF92CF92DF92EF92FF920F931F93CF9391
:1094F000DF93CDB7DEB727970FB6F894DEBF0FBE68
:10950000CDBF1C017F836E83CA01B901E982FA8253
:109510000B831C839C2C8D2CAD822AE037ED43E21B
:109520005CE30F9432160F9463142B013C012AE084
:1095300037ED43E25CE3EE81FF81608171818281DE
:1095400093810F9432160F9463145B016C01A4187D
:10955000B508C608D7082AE037ED43E25CE3C80146
:10956000B7010F9432160F9463147B018C01E41839
:10957000F50806091709FD81FF938F929F9285EAEE
:10958000882E81E4982EA30192016E817F81C10112
:109590000E94A2630F900F900F9027960FB6F89439
:1095A000DEBF0FBECDBFDF91CF911F910F91FF9016
:1095B000EF90DF90CF90BF90AF909F908F907F9073
:1095C0006F905F904F903F902F9008952F923F9211
:1095D0004F925F926F927F928F929F92AF92BF92C3
:1095E000CF92DF92EF92FF920F931F93CF93DF936F
:1095F000CDB7DEB727970FB6F894DEBF0FBECDBF4D
:109600001C017F836E83E982FA820B831C839C2C6E
:109610008D2CAD82CA01B9010F9494142AE037ED64
:1096200043E25CE30F9432160F9463142B013C0168
:10963000EE81FF8160817181828193810F94941406
:109640002AE037ED43E25CE30F9432160F94631483
:109650005B016C01A418B508C608D708C801B7019A
:109660000F9494142AE037ED43E25CE30F94321632
:109670000F9463147B018C01E418F508060917099F
:10968000FD81FF938F929F928BEA882E81E4982E22
:10969000A30192016E817F81C1010E94A2630F909C
:1096A0000F900F9027960FB6F894DEBF0FBECDBF78
:1096B000DF91CF911F910F91FF90EF90DF90CF90AE
:1096C000BF90AF909F908F907F906F905F904F90E2
:1096D0003F902F9008959F92AF92BF92CF92DF92CA
:1096E000EF92FF920F931F93CF93DF9300D01F92BF
:1096F000CDB7DEB761E081E00E9401659090520530
:10970000B12C91101AC080911B05811104C00E94D8
:10971000316881117DC180911F02882309F46FC1D6
:1097200081E090911B05911180E004E024E047EC7A
:1097300059E26B2D0E940B3D62C181E098122CC052
:1097400080911B05813021F40E943168811168C12C
:1097500080911F02882309F452C111E080911B05FA
:10976000813009F010E080917E0D90917F0DA091E5
:10977000800DB091810D89839A83AB83BC83CE0128
:1097800001960E94268700E09C014BEB59E26B2D6D
:10979000812F0E943F3D33C182E098122CC08091FE
:1097A0001B05823021F40E943168811153C18091E0
:1097B0001F02882309F423C111E080911B05823028
:1097C00009F010E08091820D9091830DA091840D9D
:1097D000B091850D89839A83AB83BC83CE010196BA
:1097E0000E94268700E09C0147EA59E26B2D812FF9
:1097F0000E943F3D04C183E098122CC080911B055C
:10980000833021F40E94316881113EC180911F0292
:10981000882309F4F4C011E080911B05833009F01E
:1098200010E08091860D9091870DA091880DB091E8
:10983000890D89839A83AB83BC83CE0101960E94F4
:10984000268700E09C0145E959E26B2D812F0E949B
:109850003F3DD5C084E0981228C080911B0584301C
:1098600021F40E943168811129C180911F0288234F
:1098700009F4C5C011E080911B05843009F010E0A7
:1098800060913E0D70913F0D8091400D9091410D82
:109890000F9494140E945B4200E09C0147E859E257
:1098A0006B2D812F0E943F3DAAC085E0981228C0F1
:1098B00080911B05853021F40E94316881111BC104
:1098C00080911F02882309F49AC011E080911B0542
:1098D000853009F010E06091420D7091430D809148
:1098E000440D9091450D0F9494140E945B4200E04A
:1098F0009C0149E759E26B2D812F0E943F3D7FC0BB
:1099000086E0981228C080911B05863021F40E94C1
:10991000316881110DC180911F02882309F46FC045
:1099200011E080911B05863009F010E06091460D32
:109930007091470D8091480D9091490D0F949414AA
:109940000E945B4200E09C014BE659E26B2D812FA7
:109950000E943F3D54C087E0981228C080911B05AB
:10996000873021F40E9431688111FFC080911F026D
:10997000882309F444C011E080911B05873009F069
:1099800010E060914A0D70914B0D80914C0D9091BB
:109990004D0D0F9494140E945B4200E09C014BE536
:1099A00059E26B2D812F0E943F3D29C088E098121B
:1099B00026C080911B05883021F40E9431688111F6
:1099C000F1C080911F028823D1F011E080911B0526
:1099D000883009F010E060914E0D70914F0D80912C
:1099E000500D9091510D0F9494140E945B4200E031
:1099F0009C014BE459E26B2D812F0E943F3DB394B3
:109A0000939485E0B8127DCE89E080931A05E6C074
:109A10000E94516480912C05882309F47CCEDEC01D
:109A200081E00E942668A12CC12CD12CE12C1CE5E0
:109A3000F12E01EC17E420E030E040E251E46EE763
:109A40007DE081EC99E243DD80912C05882309F4C7
:109A50007FCEC4C081E00E942668A12CC12CD12CED
:109A6000E12C1CE5F12E01EC17E420E030E048EC9D
:109A700052E462E87DE081EB99E229DD80912C05DA
:109A8000882309F494CEAAC081E00E942668A12C04
:109A9000C12CD12CE12C1CE5F12E01EC17E420E0C7
:109AA00030E048EC52E466E87DE08EE999E20FDDB3
:109AB00080912C05882309F4A9CE90C081E00E94F2
:109AC0002668A12CEDEBCE2EE1E4DE2E18EBE12E84
:109AD00012E8F12E01E010E024E630E040E050E032
:109AE0006EE37DE08EE899E271DD80912C0588239C
:109AF00009F4BBCE73C081E00E942668A12C6DEBF7
:109B0000C62E61E4D62E18EBE12E12E8F12E01E00C
:109B100010E024E630E040E050E062E47DE080E8E0
:109B200099E254DD80912C05882309F4C9CE56C0F2
:109B300081E00E942668A12C4DEBC42E41E4D42E76
:109B400018EBE12E12E8F12E01E010E02AE030E0FF
:109B500040E050E066E47DE082E799E237DD809105
:109B60002C05882309F4D7CE39C081E00E942668ED
:109B7000A12C29E9C22E22E4D22E18EBE12E12E804
:109B8000F12E01E010E024E630E040E050E06AE42D
:109B90007DE083E699E21ADD80912C05882309F4A3
:109BA000E5CE1CC081E00E942668A12C8BE9C82E5E
:109BB00082E4D82E18EBE12E12E8F12E01E010E03D
:109BC00024E630E040E050E06EE47DE083E599E299
:109BD000FDDC80912C05882309F4F3CE0F900F90C3
:109BE0000F900F90DF91CF911F910F91FF90EF9009
:109BF000DF90CF90BF90AF909F9008952F923F92AB
:109C00004F925F926F927F928F929F92AF92BF928C
:109C1000CF92DF92EF92FF920F931F93CF93DF9338
:109C2000CDB7DEB727970FB6F894DEBF0FBECDBF16
:109C30001C017F836E83CA01B901E982FA820B831A
:109C40001C839C2C8D2CAD8220E030E048EC52E44B
:109C50000F9432160F9463142B013C0120E030E086
:109C600048EC52E4EE81FF816081718182819381B1
:109C70000F9432160F9463145B016C01A418B5089D
:109C8000C608D70820E030E048EC52E4C801B7012C
:109C90000F9432160F9463147B018C01E418F508BD
:109CA00006091709FD81FF938F929F9287EB882EFB
:109CB00081E4982EA30192016E817F81C1010E94EF
:109CC000A2630F900F900F9027960FB6F894DEBF07
:109CD0000FBECDBFDF91CF911F910F91FF90EF90FD
:109CE000DF90CF90BF90AF909F908F907F906F90BC
:109CF0005F904F903F902F9008959F92AF92BF92A8
:109D0000CF92DF92EF92FF920F931F93CF93DF9347
:109D100000D01F92CDB7DEB761E081E00E940165FF
:109D200090905205B12C91101AC080911B058111A1
:109D300004C00E943168811104C180911F028823F0
:109D400009F4F6C081E090911B05911180E004E0D8
:109D500024E047EE58E26B2D0E940B3DE9C081E004
:109D600098122CC080911B05813021F40E9431682B
:109D70008111EFC080911F02882309F4D9C011E03E
:109D800080911B05813009F010E08091560D909173
:109D9000570DA091580DB091590D89839A83AB83CB
:109DA000BC83CE0101960E947F8800E09C0143EDB8
:109DB00058E26B2D812F0E943F3DBAC082E098127D
:109DC0002CC080911B05823021F40E9431688111E2
:109DD000DCC080911F02882309F4AAC011E08091A1
:109DE0001B05823009F010E080915A0D90915B0DB7
:109DF000A0915C0DB0915D0D89839A83AB83BC8388
:109E0000CE0101960E947F8800E09C014FEB58E252
:109E10006B2D812F0E943F3D8BC083E098122CC098
:109E200080911B05833021F40E9431688111C9C0E3
:109E300080911F02882309F47BC011E080911B05EB
:109E4000833009F010E080915E0D90915F0DA0913C
:109E5000600DB091610D89839A83AB83BC83CE0181
:109E600001960E947F8800E09C014BEA58E26B2D2E
:109E7000812F0E943F3D5CC084E098122CC08091ED
:109E80001B05843021F40E9431688111B6C0809195
:109E90001F02882309F44CC011E080911B05843017
:109EA00009F010E08091620D9091630DA091640D16
:109EB000B091650D89839A83AB83BC83CE010196F3
:109EC0000E947F8800E09C0145E958E26B2D812FBC
:109ED0000E943F3D2DC085E098122AC080911B054D
:109EE000853021F40E9431688111A3C080911F0246
:109EF0008823F1F011E080911B05853009F010E016
:109F00008091660D9091670DA091680DB091690DDB
:109F100089839A83AB83BC83CE0101960E947F889C
:109F200000E09C014FE758E26B2D812F0E943F3DDE
:109F3000B394939485E0B812F6CE86E080931A0528
:109F400093C00E94516480912C05882309F4F5CEBA
:109F50008BC081E00E942668A12CEFEBCE2EE1E4BD
:109F6000DE2EE12C1CE3F12E0CE116E420E030E0C3
:109F700040EA50E466E57DE08DED98E23FDE8091B9
:109F80002C05882309F4F6CE6FC081E00E94266874
:109F9000A12C6FEBC62E61E4D62EE12C1CE3F12E32
:109FA0000CE116E420E030E040EA50E46AE57DE0B0
:109FB00089EC98E223DE80912C05882309F409CFEF
:109FC00053C081E00E942668A12C4FEBC42E41E4CF
:109FD000D42EE12C1CE3F12E0CE116E420E030E05D
:109FE00040EA50E46EE57DE085EB98E207DE809183
:109FF0002C05882309F41CCF37C081E00E94266815
:10A00000A12C27ECC22E22E4D22EE12C1CE3F12E4F
:10A010000CE116E420E030E040EA50E462E67DE046
:10A0200080EA98E2EBDD80912C05882309F42FCF9C
:10A030001BC081E00E942668A12C89ECC82E82E416
:10A04000D82EE12C1CE3F12E0CE116E420E030E0E8
:10A0500040EA50E466E67DE08AE898E2CFDD809150
:10A060002C05882309F442CF0F900F900F900F908A
:10A07000DF91CF911F910F91FF90EF90DF90CF90E4
:10A08000BF90AF909F9008950F93CF93DF9361E0BF
:10A0900081E00E940165D0915205C0E0D1111AC043
:10A0A00080911B05811104C00E9431688111C6C0D6
:10A0B00080911F02882309F4B8C081E090911B05AC
:10A0C000911180E004E024E046E85BE26C2F0E94FE
:10A0D0000B3DABC0D130D9F480911B05813021F408
:10A0E0000E9431688111B2C080911F02882309F457
:10A0F0009CC081E090911B05913009F080E003E065
:10A100002EE34FE75BE26C2F0E940B3D8EC0D230F6
:10A11000D9F480911B05823021F40E9431688111AD
:10A120009FC080911F02882309F47FC081E0909135
:10A130001B05923009F080E003E02EE348E75BE284
:10A140006C2F0E940B3D71C0D330D9F480911B0558
:10A15000833021F40E94316881118CC080911F02EC
:10A16000882309F462C081E090911B05933009F0C7
:10A1700080E003E02EE341E75BE26C2F0E940B3DA1
:10A1800054C0D430D9F480911B05843021F40E944E
:10A190003168811179C080911F02882309F445C07C
:10A1A00081E090911B05943009F080E003E02EE3FC
:10A1B00047E65BE26C2F0E940B3D37C0D530D1F4EF
:10A1C00080911B05853021F40E943168811166C0A1
:10A1D00080911F02882349F181E090911B05953001
:10A1E00009F080E003E02EE34CE55BE26C2F0E9477
:10A1F0000B3D1BC0D630C9F480911B05863021F47D
:10A200000E943168811154C080911F02882369F037
:10A2100081E090911B05963009F080E003E02EE389
:10A2200041E55BE26C2F0E940B3DCF5FDF5FC530E5
:10A2300009F034CF87E080931A0543C00E9451642F
:10A2400080912C05882309F433CF3BC084E495E545
:10A250000E947D4280912C05882309F445CF31C0AE
:10A2600089E495E50E947D4280912C05882309F4BC
:10A2700058CF27C08EE495E50E947D4280912C0541
:10A28000882309F46BCF1DC083E595E50E947D42CC
:10A2900080912C05882309F47ECF13C088E595E5CD
:10A2A0000E947D4280912C05882309F491CF09C03A
:10A2B0008DE595E50E947D4280912C05882309F467
:10A2C000A3CFDF91CF910F910895CF92DF92EF92BC
:10A2D000FF92CF93C82F833029F467FD6091760CED
:10A2E000609365050E9464286B017C0124EA30E7D5
:10A2F0004DE75FE360916A0570916B0580916C0595
:10A3000090916D050F94F41387FD05C08AEF90E0DE
:10A31000A0E0B0E003C080E090E0DC01C80ED91EF0
:10A32000EA1EFB1EC0926605D0926705E0926805A2
:10A33000F0926905C0932002CF91FF90EF90DF90DB
:10A34000CF9008952F923F924F925F926F927F929B
:10A350008F929F92AF92BF92CF92DF92EF92FF9235
:10A360001F93CF93DF93CDB7DEB72A970FB6F8943C
:10A37000DEBF0FBECDBF1C01162F0E94316888239F
:10A3800029F0109283050E945164DBC08091790509
:10A3900090917A05A0917B05B0917C058F83988779
:10A3A000A987BA87892B8A2B8B2B09F492C0E4E00A
:10A3B0001E9FD0011124BE83AD83FD01E957F34FE9
:10A3C000408051806280738020E030E04AE754E4AE
:10A3D000C301B2010F941B136B017C0180914C02ED
:10A3E0008823F9F01130A9F058F01230D1F4C09060
:10A3F0004802D0904902E0904A02F0904B0211C00E
:10A40000C0904002D0904102E0904202F09043029E
:10A4100008C0C0904402D0904502E0904602F090FF
:10A4200047026F81788589859A850F9496142091CB
:10A430006A0530916B0540916C0550916D050F9444
:10A4400032169B01AC01C301B2010F941B134B01E7
:10A450005C018D819E818957934F9E838D83DC01A2
:10A460008D929D92AD92BC9213978F819885A9850C
:10A47000BA85B7FF1AC020E030E04AE754E4C301D0
:10A48000B2010F941A136B017C019B01AC01C50151
:10A49000B4010F94F41387FF16C0AD81BE81CD9235
:10A4A000DD92ED92FC9213970EC0A7019601C501B3
:10A4B000B4010F94F715181634F4ED81FE81C082B3
:10A4C000D182E282F3826FEF812FFFDE81E0809301
:10A4D0001F021092790510927A0510927B05109256
:10A4E0007C0580911F02882361F124E0129FF00116
:10A4F0001124E957F34F80819181A281B38189832F
:10A500009A83AB83BC832DEC3CEC4CEC5DE3609117
:10A510006A0570916B0580916C0590916D050F94A3
:10A52000F71587FD05C0CE0101960E94168605C06D
:10A5300060E2CE0101960E948E86BC01C1010E949C
:10A54000A03D2A960FB6F894DEBF0FBECDBFDF91B7
:10A55000CF911F91FF90EF90DF90CF90BF90AF9081
:10A560009F908F907F906F905F904F903F902F9033
:10A57000089560E08AE09CE2E5CE61E083E09CE241
:10A58000E1CE62E08CEF9BE2DDCE0F931F93CF9381
:10A59000DF9300D01F92CDB7DEB7182F0E9431682D
:10A5A000882329F0109283050E94516464C0609151
:10A5B000790570917A0580917B0590917C056115F4
:10A5C00071058105910571F10F94961420916A052A
:10A5D00030916B0540916C0550916D050F943216CA
:10A5E0009B01AC016091930C7091940C8091950C3F
:10A5F0009091960C0F941B136093930C7093940C92
:10A600008093950C9093960C612F83E05EDE81E041
:10A6100080931F021092790510927A0510927B05A3
:10A6200010927C0580911F02882329F1113019F4C2
:10A630000FE81BE202C00AE91BE2209109053091F4
:10A640000A0540910B0550910C056091930C709197
:10A65000940C8091950C9091960C0F941A13698329
:10A660007A838B839C83CE0101960E941686BC015F
:10A67000C8010E94A03D0F900F900F900F90DF91A6
:10A68000CF911F910F9108958FEF7FCF80E07DCF05
:10A6900081E07BCF21E02093830560936A0570936E
:10A6A0006B0580936C0590936D0540E050E0BA0116
:10A6B00080910705909108050C94266460E070E095
:10A6C00080E291E4E7CF60E070E080E89FE3E2CFD2
:10A6D0006DEC7CEC8CEC9DE3DDCFEF92FF920F9361
:10A6E0001F93CF93DF93F82EE42E709308056093A9
:10A6F000070561E081E00E940165D0915205C0E04C
:10A7000091E081E0F816A9F1F81628F082E0F81639
:10A7100009F45DC08AC0D11103C19923D9F0809199
:10A720001B051816BCF04091790550917A0560918F
:10A730007B0570917C054F5F5F4F6F4F7F4F40935C
:10A74000790550937A0560937B0570937C058F5F44
:10A7500080931B0580911F02882309F452C100E0F9
:10A7600010E021E041E065EF7BE28C2F0E94A83CE5
:10A7700048C1D111D5C09923D9F080911B05181675
:10A78000BCF04091790550917A0560917B057091FC
:10A790007C054F5F5F4F6F4F7F4F4093790550931C
:10A7A0007A0560937B0570937C058F5F80931B0512
:10A7B00080911F02882309F424C100E010E021E009
:10A7C00041E06EEE7BE28C2F0E94A83C1AC1D111B1
:10A7D000A7C09923D9F080911B051816BCF04091B1
:10A7E000790550917A0560917B0570917C054F5FEA
:10A7F0005F4F6F4F7F4F4093790550937A05609379
:10A800007B0570937C058F5F80931B0580911F02F1
:10A81000882309F4F6C000E010E021E041E067EE93
:10A820007BE28C2F0E94A83CECC04091930C50918D
:10A83000940C6091950C7091960C4093090550937F
:10A840000A0560930B0570930C05D1112CC0992358
:10A85000D9F080911B051816BCF0409179055091F4
:10A860007A0560917B0570917C054F5F5F4F6F4F5C
:10A870007F4F4093790550937A0560937B057093E1
:10A880007C058F5F80931B0580911F02882309F44C
:10A89000F0C000E010E021E041E06DED7BE28C2FA4
:10A8A0000E94A83CE6C083E0F8123AC0E7FC02C070
:10A8B000EE2D02C0E091760C84E0E89FF0011124B7
:10A8C000EA54F44F60817181828193812091610B00
:10A8D000211126C00F94631420912F023091300271
:10A8E00062177307ECF4D130C9F480911B058130F5
:10A8F00021F40E94316881118EC080911F0288234B
:10A9000069F081E090911B05913009F080E004E04E
:10A9100024E04DEC5BE26C2F0E940B3D82E072C0A4
:10A92000D130D9F480911B05813021F40E94316827
:10A93000811179C080911F02882309F462C081E0EF
:10A9400090911B05913009F080E004E024E043EC95
:10A950005BE26C2F0E940B3D54C0D230D9F4809141
:10A960001B05823021F40E943168811164C08091FE
:10A970001F02882309F445C081E090911B059230A5
:10A9800009F080E003E02EE349EB5BE26C2F0E94CC
:10A990000B3D37C0D330D1F480911B05833021F4B7
:10A9A0000E943168811151C080911F02882349F1B2
:10A9B00081E090911B05933009F080E003E02EE3E5
:10A9C00040EB5BE26C2F0E940B3D1BC0D430C9F4FE
:10A9D00080911B05843021F40E94316881113FC0B1
:10A9E00080911F02882369F081E090911B059430CB
:10A9F00009F080E003E02EE345EA5BE26C2F0E9461
:10AA00000B3D85E0CF5FDF5F90E0C53009F079CE88
:10AA100080931A0532C00E94516480912C058823CE
:10AA200009F46BCF2AC00E94516480912C058823C1
:10AA300009F480CF22C08EE593E50E947D4280918B
:10AA40002C05882309F493CF18C083E693E50E9470
:10AA50007D4280912C05882309F4A6CF0EC088E69C
:10AA600093E50E947D4280912C05882309F4B8CF9C
:10AA700004C083E0F812C5CF19CFDF91CF911F91A9
:10AA80000F91FF90EF9008954FEF69EB72E580E032
:10AA900024CE4FEF6DEB72E581E01FCE4FEF61ECFE
:10AAA00072E582E01ACE4FEF64E473E583E015CEE1
:10AAB00040E066E473E583E010CE41E068E473E5CE
:10AAC00083E00BCE0F93CF93DF9361E081E00E9490
:10AAD0000165D0915205C0E0D1111AC080911B05CB
:10AAE000811104C00E94316881118BC080911F02C6
:10AAF000882309F47EC081E090911B05911180E0CC
:10AB000004E024E04CE45BE26C2F0E940B3D71C03A
:10AB1000D130D9F480911B05813021F40E94316835
:10AB2000811177C080911F02882309F462C081E0FF
:10AB300090911B05913009F080E003E02EE342E4A0
:10AB40005BE26C2F0E940B3D54C0D230D9F480914F
:10AB50001B05823021F40E943168811164C080910C
:10AB60001F02882309F445C081E090911B059230B3
:10AB700009F080E000E22EE344E35BE26C2F0E94E8
:10AB80000B3D37C0D330D1F480911B05833021F4C5
:10AB90000E943168811151C080911F02882349F1C0
:10ABA00081E090911B05933009F080E000E22EE3F4
:10ABB00046E25BE26C2F0E940B3D1BC0D430C9F40F
:10ABC00080911B05843021F40E94316881113FC0BF
:10ABD00080911F02882369F081E090911B059430D9
:10ABE00009F080E000E22EE341E15BE26C2F0E947D
:10ABF0000B3DCF5FDF5FC53009F06ECFC0931A0504
:10AC00002FC00E94516480912C05882309F46ECFD7
:10AC100027C084E490E50E947D4280912C05882322
:10AC200009F480CF1DC08EE39BE20E94A063809157
:10AC30002C05882309F493CF13C083E39BE20E9481
:10AC4000A06380912C05882309F4A6CF09C082E275
:10AC50009BE20E94A06380912C05882309F4B8CF61
:10AC6000DF91CF910F910895CF93DF93EC01CB014A
:10AC7000BA010F9496140F94631479836883DF915B
:10AC8000CF91089564E376E585ED96E50C946564CF
:10AC90000F931F93CF93DF9361E081E00E940165E2
:10ACA000C0915205D0E081E0C1112CC08823D9F0B9
:10ACB00080911B051816BCF04091790550917A05DA
:10ACC00060917B0570917C054F5F5F4F6F4F7F4FA9
:10ACD0004093790550937A0560937B0570937C05CA
:10ACE0008F5F80931B0580911F02882309F441C068
:10ACF00000E010E020E041E069E67DE28D2F0E9457
:10AD0000A83C37C0C130D1F480911B05813021F4BB
:10AD10000E943168811137C080911F02882349F158
:10AD200081E090911B05913009F080E000E22EE374
:10AD30004EE55DE26D2F0E940B3D1BC0C230C9F491
:10AD400080911B05823021F40E943168811122C05C
:10AD500080911F02882369F081E090911B05923059
:10AD600009F080E000E22EE34AE45DE26D2F0E94EC
:10AD70000B3DDF5FCF5F80E0D53009F095CF83E0FA
:10AD800080931A050DC0C093CB0A80912C058823AF
:10AD900019F206C0C093CB0A80912C058823C1F21A
:10ADA000DF91CF911F910F9108950F9496140F94F6
:10ADB0006314CB010C94D984EF92FF920F931F93ED
:10ADC000CF93DF93CDB7DEB72B970FB6F894DEBFE6
:10ADD0000FBECDBF7C0120910E05422F022E000C2C
:10ADE000550B80910F05823051F0833019F089EDB9
:10ADF0009DE20AC027FF06C085EE9DE205C087EFF1
:10AE00009DE202C08EEE9DE25F932F939F938F93FE
:10AE10008E010F5F1F4F1F930F930F943D1C809166
:10AE20000E05282F30E0220F331FF901E255F44FB1
:10AE3000D901A95DBD4F2D913C912F5031090F9043
:10AE40000F900F900F900F900F90E216F3060CF4F6
:10AE50009701318320830E948499C8010E948165F3
:10AE60002B960FB6F894DEBF0FBECDBFDF91CF910A
:10AE70001F910F91FF90EF900895E0910E05EE0F56
:10AE8000FF0BE255F44F8081918196CF5F926F92D4
:10AE90007F928F929F92AF92BF92CF92DF92EF926A
:10AEA000FF920F931F93CF93DF93582E80930F053C
:10AEB00060930E0561E081E00E940165D09152052A
:10AEC000C0E081E02DE3622E27E5722ED11138C05B
:10AED0008823D9F080911B051816BCF040917905A4
:10AEE00050917A0560917B0570917C054F5F5F4FB3
:10AEF0006F4F7F4F4093790550937A0560937B05A0
:10AF000070937C058F5F80931B0580911F028823BF
:10AF100009F492C022E0521649F083E0581203C0AF
:10AF20006BEB7DE205C06BEA7DE202C06BEC7DE27B
:10AF300000E010E021E041E08C2F0E94A83C7CC0A2
:10AF4000D130D9F480911B05813021F40E94316801
:10AF500081117BC080911F02882309F46DC081E0BC
:10AF600090911B05913009F080E004E024E046E375
:10AF70005EE26C2F0E940B3D5FC0D230D9F480910D
:10AF80001B05823021F40E943168811166C08091D6
:10AF90001F02882309F450C081E090911B05923074
:10AFA00009F080E000E22EE34AE25EE26C2F0E94AC
:10AFB0000B3D42C0D330D1F480911B05833021F486
:10AFC0000E943168811154C080911F028823A1F131
:10AFD00081E090911B05933009F080E000E22EE3C0
:10AFE0004EE15EE26C2F0E940B3D26C0D43021F56D
:10AFF00080911B05843021F40E943168811143C087
:10B0000080911F028823C1F011E080911B058430DC
:10B0100009F010E0E0910E05EE0FFF0BE255F44F42
:10B02000808191810E94D98400E09C0140E05EE231
:10B030006C2F812F0E943F3DCF5FDF5F80E0C530E6
:10B0400009F044CFC0931A0551C00E945164809109
:10B050002C05882309F47ECF49C080911605909174
:10B060001705AADE80912C05882309F490CF3EC0F5
:10B0700080911805909119059FDE80912C058823F9
:10B0800009F4A2CF33C081E00E94266860910E05CA
:10B09000660F770B6255744FFB01A080B180C5012C
:10B0A000BB0CAA0BBB0B5C016D01F8E7AF1AB10832
:10B0B000C108D1081F927F926F9282E4882E86E5A4
:10B0C000982E1AEAE12EF12C00E010E028E730E09B
:10B0D00040E050E08FE09EE20E94A2630F900F904C
:10B0E0000F9080912C05882309F48ACFDF91CF91AE
:10B0F0001F910F91FF90EF90DF90CF90BF90AF9096
:10B100009F908F907F906F905F90089560E081E0B6
:10B11000BDCE61E081E0BACE0F93CF93DF9361E0C3
:10B1200081E00E940165C0915205D0E0C11118C0B4
:10B1300080911B05811104C00E943168811198C063
:10B1400080911F02882361F081E090911B0591118D
:10B1500080E004E024E046EA5DE26D2F0E940B3DB2
:10B160002091AE0B3091AF0B8091610B81115AC0D1
:10B1700080912F029091300228173907E4F4C130F2
:10B1800031F580911B05813021F40E9431688111D5
:10B1900077C080911F028823D1F081E090911B0538
:10B1A000913009F080E003E02EE343E95DE26D2F8A
:10B1B0000E940B3D0CC0C13009F0A7C080911B0557
:10B1C000813009F485C080911F02811186C0809171
:10B1D000B00B9091B10B2091610B211125C02091F2
:10B1E0002F023091300282179307F4F4C230B9F580
:10B1F00080911B05823021F40E94316881114FC07B
:10B2000080911F02882359F181E090911B059230B3
:10B2100009F080E003E02EE340E85DE26D2F0E943C
:10B220000B3D1DC0C13051F2C230C9F480911B05E5
:10B23000823021F40E943168811140C080911F0248
:10B24000882369F081E090911B05923009F080E03D
:10B2500000E22EE340E85DE26D2F0E940B3DDF5FD0
:10B26000CF5FD53009F062CF83E080931A0552C0DA
:10B270000E94516480912C05882309F461CF4AC053
:10B280000E94806340E050E0BA0186E898E50E94A1
:10B29000266480912C05882309F47BCF3BC00E9453
:10B2A000806340E050E0BA0189E898E50E94266496
:10B2B00080912C05882309F4A3CF2CC08AE69DE257
:10B2C0000E94A06380912C05882309F4B7CF22C087
:10B2D0000E94316881110FC076CF81E090911B05EB
:10B2E000913009F080E000E22EE343E95DE26D2F4A
:10B2F0000E940B3D6CCF85E79DE20E94A063809188
:10B300002C05882309F45FCF05C08091B00B909184
:10B31000B10B65CFDF91CF910F9108958F929F92DE
:10B32000AF92BF92CF92DF92EF92FF920F931F9353
:10B33000CF93DF934C015B016A0160E085E00E94DE
:10B340000165D0915205F12C82E0E82ED1111AC08E
:10B3500080911F02882321F180911E02823041F0EA
:10B36000833019F46FE17DE205C06DE07DE202C03B
:10B370006FE27DE200E010E021E041E08F2D0E94CD
:10B38000A83C0EC0D13061F480911F02882341F0A7
:10B3900000E010E020E041E0B4018F2D0E94A83CC5
:10B3A000A114B10481F0D23081F480911F0288236E
:10B3B00009F46EC000E010E020E041E0B5018F2DFF
:10B3C0000E94A83C65C0C2E001C0C3E0C114D10422
:10B3D00091F0DC130FC080911F02882351F000E030
:10B3E00010E020E041E0B6018F2D0E94A83CCD2F57
:10B3F00001C0CD2FCF5F21E030E0A114B10411F4E2
:10B4000020E030E081E090E0C114D10411F480E04C
:10B4100090E0820F931F029781F0DC130DC08091A2
:10B420001F02882349F000E010E020E041E068E4DA
:10B430007DE28F2D0E94A83CCF5FDC1314C0809169
:10B440001F02882371F000E010E021E040E06DE38E
:10B450007DE28F2D0E94A83C60910D058F2D0E94EA
:10B460003D3CE0921F02F394DF5F85E0F8126ECF5F
:10B47000CF5FC0931A05DF91CF911F910F91FF907D
:10B48000EF90DF90CF90BF90AF909F908F900895F6
:10B49000C3E0C114D10409F0ADCFADCF44E05DE20B
:10B4A00064EF7CE28BEE9CE239CF40E050E06BED44
:10B4B0007CE282ED9CE232CF40E050E063EC7CE243
:10B4C00084EB9CE22BCF40E050E065EA7CE288E927
:10B4D0009CE224CF4CE85CE26BE77CE28BE69CE2EA
:10B4E0001DCF40E050E06DE57CE284E59CE216CFA4
:10B4F00040E050E064E47CE287E39CE20FCF40E070
:10B5000050E06AE27CE289E29CE208CF40E050E051
:10B510006AE17CE281E19CE201CF611160931E024D
:10B5200040930D05082E000C990BAA0BBB0B8B301A
:10B53000910580F5FC018827EA56FF4F8F4F0D9447
:10B54000781785E59AE51CC088E79AE519C08AE670
:10B550009AE516C081E79AE513C086E89AE510C01F
:10B560008FE79AE50DC083E69AE50AC08CE59AE577
:10B5700007C01092CB0A88E496E502C08EE49AE5F3
:10B58000009741F021E02093830540E050E0BA01AC
:10B590000C9426640C944B6480916E05882321F0F2
:10B5A000109283050E9451640C94A23B9091ED0788
:10B5B00093FB882780F993FF06C081E090911D06D8
:10B5C000911101C080E008954091760C61E080E027
:10B5D000A4DF8CEE9EE20F94A1090C94EAD3E6DF7F
:10B5E000882319F08091ED0782FD0C94B09388EECA
:10B5F0009EE20F94A109F9CF1092E915109268020A
:10B600008091ED0780628093ED070E94B8936FEF01
:10B610008AED9EE20E94FE690C944B640F93CF93D7
:10B62000DF9361E081E00E940165D0915205C0E0A6
:10B630008C2F8D0FC9F480911B05811104C00E94CD
:10B640003168811133C080911F02882341F181E06C
:10B6500090911B05911180E004E024E045ED5EE24D
:10B660006C2F0E940B3D1BC08130C9F480911B05DB
:10B67000813021F40E94316881111FC080911F0226
:10B68000882369F081E090911B05913009F080E0FA
:10B6900000E22EE34AEC5EE26C2F0E940B3DCF5F8E
:10B6A000C53031F682E080931A050CC00E945164C7
:10B6B00080912C05882339F205C09EDF80912C05EE
:10B6C0008823E1F2DF91CF910F910895EF92FF92DD
:10B6D0000F931F93CF93DF9361E081E00E94016598
:10B6E000C091520510E0C11118C080911B05811155
:10B6F00004C00E94316881116CC180911F028823AF
:10B7000061F081E090911B05911180E004E024E05C
:10B710004EEB5EE2612F0E940B3D0E940F64D82F1A
:10B720009091ED0793FBEE24E0F893FF03C03EDF1A
:10B73000F82E01C0F12CDD2309F459C0C130D9F431
:10B7400080911B05813021F40E943168811148C12C
:10B7500080911F02882309F46FC181E090911B053D
:10B76000913009F080E000E22EE342EB5EE2612FCF
:10B770000E940B3D61C1C230D9F480911B0582301B
:10B7800021F40E943168811132C180911F02882307
:10B7900009F452C181E090911B05923009F080E0DC
:10B7A00003E02EE347EA5EE2612F0E940B3D44C1B5
:10B7B000C33009F057C080911B05833021F40E94EB
:10B7C000316881111EC180911F02882309F434C1A0
:10B7D00081E090911B05933009F080E003E02EE3B7
:10B7E00042EA5EE2612F0E940B3DD4E05BC0C130B3
:10B7F000D9F480911B05813021F40E9431688111B8
:10B800000AC180911F02882309F418C181E0909138
:10B810001B05913009F080E000E22EE345E95EE28D
:10B82000612F0E940B3D0AC1C230F1F480911B05CB
:10B83000823021F40E9431688111F4C080911F028E
:10B84000882309F4FBC081E090911B05923009F038
:10B8500080E003E02EE34CE85EE2612F0E940B3DA6
:10B86000D3E020C0D4E001C0D3E0CD131BC0809151
:10B870001B058C1304C00E9431688111E1C08091C6
:10B880001F02882371F081E090911B059C1380E0DA
:10B8900003E02EE340E85EE2612F0E940B3DDC2FC7
:10B8A00001C0DC2F81E08D0FC81318C080911B05EB
:10B8B0008C1304C00E9431688111CCC080911F029A
:10B8C000882361F081E090911B059C1380E003E0E8
:10B8D0002EE342E75EE2612F0E940B3D82E08D0F76
:10B8E000C81318C080911B058C1304C00E943168D6
:10B8F0008111BAC080911F02882361F081E090918C
:10B900001B059C1380E003E02EE342E65EE2612F1C
:10B910000E940B3D83E08D0FC81318C080911B055A
:10B920008C1304C00E9431688111A8C080911F024D
:10B93000882361F081E090911B059C1380E003E077
:10B940002EE344E55EE2612F0E940B3D94E09D0FE3
:10B95000EE20E9F0F11035C0C91331C080911B050C
:10B960008C1304C00E943168811192C080911F0223
:10B97000882329F181E090911B059C1380E003E06E
:10B980002EE346E45EE2612F0E940B3D18C0C9130E
:10B9900016C080911B058C1302C00E9431688091F3
:10B9A0001F02882361F081E090911B059C1380E0C9
:10B9B00000E22EE34BE35EE2612F0E940B3D95E037
:10B9C0009D0F1F5FCF5F153009F08DCE90931A0544
:10B9D00068C067D780912C05882309F48ECE61C09A
:10B9E000F3DD80912C05882309F4B2CE5AC08EE095
:10B9F0009BE50E947D4280912C05882309F4C5CEE9
:10BA000050C088EF9DE50E947D4280912C058823DF
:10BA100009F4D9CE46C0E3DD80912C05882309F4D2
:10BA2000F0CE3FC082E695E50E947D4280912C05D4
:10BA3000882309F403CF35C0D4E034CFD3E032CF2C
:10BA40008DE190E60E947D4280912C05882309F4C7
:10BA500016CF27C08DE892E60E947D4280912C058A
:10BA6000882309F42BCF1DC08CE898E50E947D4205
:10BA700080912C05882309F43DCF13C08CEC9AE506
:10BA80000E947D4280912C05882309F44FCF09C084
:10BA900087E390E40E947D4280912C05882309F47D
:10BAA00065CFDF91CF911F910F91FF90EF90089597
:10BAB0006091AA0B70E080E00C94A09460915B020E
:10BAC00070915C02072E000C880B990B0F94961452
:10BAD0002AE037ED43E25CE30F94321660935302A1
:10BAE000709354028093550290935602089560918A
:10BAF0005D0270915E02072E000C880B990B0F946B
:10BB000096142AE037ED43E25CE30F94321660931B
:10BB10005702709358028093590290935A020895E5
:10BB2000CF93DF93EC01CB01BA010F9496140F94DD
:10BB300068146883DF91CF91089560E97DE582EA1A
:10BB40009DE5C3C60F9496140F946814862F0C9429
:10BB5000B3840F946314CB010C94D9844F925F92F9
:10BB60006F927F928F929F92AF92BF92CF92DF920D
:10BB7000EF92FF920F931F93CF93DF93F901D801B8
:10BB80009E2C9A01550F440B550BEB01A880B980F0
:10BB90006501BB0CEE08FF0856016701A21AB30A43
:10BBA000C40AD50A2F01FF0F6608770883017201C6
:10BBB000E21AF30A040B150B9F92BF93AF93E2E4D2
:10BBC0008E2EE6E59E2EBED50F900F900F90DF9142
:10BBD000CF911F910F91FF90EF90DF90CF90BF908A
:10BBE000AF909F908F907F906F905F904F9008954F
:10BBF0006F927F928F929F92AF92BF92CF92DF927D
:10BC0000EF92FF920F931F93CF93DF9361E081E058
:10BC1000F8D6D0915205C0E028E5622E2DE5722EAF
:10BC2000D1111AC080911B05811104C00E94316896
:10BC3000811131C180911F02882309F423C181E061
:10BC400090911B05911180E004E024E042E65FE260
:10BC50006C2F0E940B3D16C1D13039F580911B0528
:10BC6000813021F40E94316881111CC180911F0232
:10BC7000882309F407C111E080911B05813009F088
:10BC800010E060914D0270914E02072E000C880B5F
:10BC9000990B0F9496145DDF00E09C0146E55FE28E
:10BCA0006C2F812F0E943F3DEDC0D23039F580913D
:10BCB0001B05823021F40E943168811105C18091F9
:10BCC0001F02882309F4DEC011E080911B05823039
:10BCD00009F010E06091AE0B7091AF0B072E000CD5
:10BCE000880B990B0F94961434DF00E09C0144E418
:10BCF0005FE26C2F812F0E943F3DC4C0D33039F5E5
:10BD000080911B05833021F40E9431688111F1C0BC
:10BD100080911F02882309F4B5C011E080911B05B2
:10BD2000833009F010E06091B00B7091B10B072ED9
:10BD3000000C880B990B0F9496140BDF00E09C010C
:10BD400042E35FE26C2F812F0E943F3D9BC0D430C5
:10BD500039F580911B05843021F40E9431688111EE
:10BD6000DDC080911F02882309F48CC011E080910E
:10BD70001B05843009F010E06091A20B7091A30BB9
:10BD8000072E000C880B990B0F949614E2DE00E04E
:10BD90009C014AE25FE26C2F812F0E943F3D72C0FE
:10BDA000D53001F580911B05853021F40E94316862
:10BDB0008111C9C080911F02882309F463C011E07A
:10BDC00080911B05853009F010E08091AA0B0E943C
:10BDD000B38400E09C0142E15FE26C2F812F0E945E
:10BDE0003F3D50C0D63039F580911B05863021F497
:10BDF0000E9431688111CBC080911F02882309F411
:10BE000041C011E080911B05863009F010E060917F
:10BE10005B0270915C02072E000C880B990B0F944B
:10BE2000961497DE00E09C0144E05FE26C2F812FC6
:10BE30000E943F3D27C0D73029F580911B058730F0
:10BE400021F40E9431688111B4C080911F028823BF
:10BE5000C9F011E080911B05873009F010E0609176
:10BE60005D0270915E02072E000C880B990B0F94F7
:10BE700096146FDE00E09C0146EF5EE26C2F812F8E
:10BE80000E943F3DCF5FDF5FC53009F0C9CE88E03B
:10BE900080931A059FC005D580912C05882309F44D
:10BEA000C9CE98C0E12C00E010E027EE33E04AE074
:10BEB00050E06DE472E08CE59FE250DE80912C054D
:10BEC000882309F4D3CE86C081E00E942668E12C45
:10BED00009E715E622E231E040E050E06EEA7BE05F
:10BEE0008DE49FE23BDE80912C05882309F4E7CEA8
:10BEF00071C081E00E942668E12C0CE715E622E281
:10BF000031E040E050E060EB7BE08BE39FE226DE37
:10BF100080912C05882309F4FBCE5CC081E00E944F
:10BF20002668E12C0FE715E627E830E040E050E016
:10BF300062EA7BE08EE29FE211DE80912C0588238D
:10BF400009F40FCF47C081E00E942668A090AA0B99
:10BF5000B12CC12CD12C1F927F926F928DE9882E2B
:10BF60008DE5982EE12CF12C8701EA9420E030E059
:10BF7000A9016AEA7BE08EE19FE2E4D30F900F9083
:10BF80000F9080912C05882309F414CF23C0E12C55
:10BF90000EE51DE527EE33E04AE050E06BE572E088
:10BFA0008BE09FE2DBDD80912C05882309F424CF10
:10BFB00011C0E12C07E71DE527EE33E04AE050E031
:10BFC0006DE572E08DEF9EE2C9DD80912C0588233E
:10BFD00009F43BCFDF91CF911F910F91FF90EF902C
:10BFE000DF90CF90BF90AF909F908F907F906F9099
:10BFF00008956091AB0B70E081E00C94A094262F23
:10C0000030E0220F331FF901E255F44FD901A95D49
:10C01000BD4F2D913C912F503109821793070CF49D
:10C020009C0131832083862F0C948499ECEAFBE0F9
:10C03000108211820E942C9A2EC44F925F926F92AE
:10C040007F928F929F92AF92BF92CF92DF92EF92A8
:10C05000FF920F931F93CF93DF9361E081E0D1D4E0
:10C06000D0915205C0E049EF642E4FE5742E58E59B
:10C07000452E5DE5552ED11119C080911B0581110A
:10C0800003C0EFD78111F7C080911F02882309F404
:10C09000B5C081E090911B05911180E004E024E09F
:10C0A0004CEC5FE26C2F0E940B3DA8C0D13009F52B
:10C0B00080911B05813019F4D4D78111E3C08091A0
:10C0C0001F02882309F49AC011E080911B0581307A
:10C0D00009F010E08091AE0B9091AF0B0E94D984D3
:10C0E00000E09C014AEB5FE26C2F812F0E943F3DF4
:10C0F00085C0D23009F580911B05823019F4B1D783
:10C100008111D4C080911F02882309F477C011E007
:10C1100080911B05823009F010E08091B00B909166
:10C12000B10B0E94D98400E09C0148EA5FE26C2FC9
:10C13000812F0E943F3D62C0D33009F580911B05DD
:10C14000833019F48ED78111C5C080911F028823D6
:10C1500009F454C011E080911B05833009F010E010
:10C160008091A20B9091A30B0E94D98400E09C01C6
:10C1700040EA5FE26C2F812F0E943F3D3FC0D430E8
:10C18000F1F480911B05843019F46BD78111B6C08E
:10C1900080911F02882391F111E080911B0584306A
:10C1A00009F010E08091AA0B0E94B38400E09C018A
:10C1B00048E85FE26C2F812F0E943F3D1FC0D530C1
:10C1C000E9F480911B05853019F44BD78111B9C072
:10C1D00080911F02882391F011E080911B0585302A
:10C1E00009F010E08091AB0B0E94B38400E09C0149
:10C1F00040E75FE26C2F812F0E943F3D8091AE0BA4
:10C200009091AF0B892B49F481E02091B00B3091D4
:10C21000B10B232B19F480E001C081E02091A20B27
:10C220003091A30B232B11F48823E1F0D630C1F415
:10C2300080911B05863019F414D78111A5C0809117
:10C240001F02882369F081E090911B05963009F068
:10C2500080E000E22EE347E65FE26C2F0E940B3D98
:10C2600087E001C086E0CF5FDF5FC53009F003CF14
:10C2700080931A058FC015D380912C05882309F46B
:10C2800003CF88C081E0E2D6E12C09E715E622E27F
:10C2900031E040E050E06EEA7BE083EC9FE25EDC60
:10C2A00080912C05882309F40ACF74C081E0CED692
:10C2B000E12C0CE715E622E231E040E050E060EBD3
:10C2C0007BE081EB9FE24ADC80912C05882309F416
:10C2D00019CF60C081E0BAD6E12C0FE715E627E858
:10C2E00030E040E050E062EA7BE084EA9FE236DC46
:10C2F00080912C05882309F428CF4CC081E0A6D674
:10C30000A090AA0BB12CC12CD12C1F925F924F92FE
:10C310002DE9822E2DE5922EE12CF12C8701EA9455
:10C3200020E030E0A9016AEA7BE084E99FE20AD2DA
:10C330000F900F900F9080912C05882309F428CF3F
:10C3400029C081E083D6A090AB0BB12CC12CD12C9D
:10C350001F927F926F928DE9882E8DE5982EE12CA9
:10C36000F12C8701EA9420E030E0A9016BEA7BE040
:10C370008CE79FE2E7D10F900F900F9080912C05F2
:10C38000882309F425CF06C051DE80912C0588232F
:10C3900009F455CFDF91CF911F910F91FF90EF904E
:10C3A000DF90CF90BF90AF909F908F907F906F90D5
:10C3B0005F904F9008957F928F929F92AF92BF921D
:10C3C000CF92DF92EF92FF920F931F93CF93DF9361
:10C3D00061E081E016D370905205C0E08C2F870D8C
:10C3E000C9F480911B05811103C03BD6811158C04F
:10C3F00080911F02882309F44BC081E090911B05B6
:10C40000911180E004E024E042E350E36C2F0E94AD
:10C410000B3D3EC08130E1F580911B05813019F460
:10C4200020D6811144C080911F02882389F1D1E078
:10C4300080911B05813009F0D0E0C090C70BD090EF
:10C44000C80BE090C90BF090CA0B20E030E0A901C6
:10C45000C701B6010F94F41387FD05C020E030E05A
:10C4600040E05FE304C020E030E040E05FEBC70164
:10C47000B6010F941B130F946314CB010E94D9844F
:10C4800000E09C0142E250E36C2F8D2F0E943F3D63
:10C49000CF5FC53009F0A2CF82E080931A052FC08C
:10C4A00000D280912C05882309F4A2CF28C0609186
:10C4B000C70B7091C80B8091C90B9091CA0B0F9458
:10C4C00063141F921F921F922FE9822E21E4922E55
:10C4D0005B016C011AE0E12EF12C00E010E020E09D
:10C4E00030E0A90167EC7BE08AE290E32BD10F906A
:10C4F0000F900F9080912C05882309F494CFDF9141
:10C50000CF911F910F91FF90EF90DF90CF90BF9050
:10C51000AF909F908F907F9008950F931F93CF932C
:10C52000DF9361E081E06DD2D0915205C0E0D1117E
:10C5300015C080911B05811103C093D581119AC04C
:10C5400080911F02882321F181E090911B059111B8
:10C5500080E004E024E04DE150E317C0D130C1F4A5
:10C5600080911B05813019F47CD581118AC080919E
:10C570001F02882369F081E090911B05913009F03A
:10C5800080E003E02EE34BE050E36C2F0E940B3D74
:10C5900046D1182FD230B9F480911B05823019F49E
:10C5A00060D581117BC080911F02882309F495C05A
:10C5B00081E090911B05923009F080E003E02EE3CA
:10C5C0004FEF5FE218C0D330D1F480911B05833068
:10C5D00019F447D581116FC080911F02882309F497
:10C5E0007CC081E090911B05933009F080E000E26F
:10C5F0002EE340EF5FE26C2F0E940B3D6EC0811175
:10C600006FC0D430B1F480911B05843019F429D562
:10C61000811158C080911F02882319F181E0909107
:10C620001B05943009F080E000E22EE342EE5FE269
:10C6300015C0D530B1F480911B05853009F449C08F
:10C6400080911F02882369F081E090911B0595304D
:10C6500009F080E000E22EE341ED5FE26C2F0E94E2
:10C660000B3D86E0CF5FDF5FC53009F060CF809380
:10C670001A0541C016D180912C05882309F460CF9A
:10C680003AC03ED040E050E0BA018BEC92E4DED0FC
:10C6900080912C05882309F46ACF2DC031D040E069
:10C6A00050E0BA018BED91E6D1D080912C05882322
:10C6B00009F479CF20C02DD280912C05882309F46C
:10C6C0008BCF19C029D280912C05882309F4A2CFE1
:10C6D00012C0C7D4811106C0B3CF112309F4C1CF52
:10C6E00084E0C0CF0E94E2BC81E0EFD180912C05B4
:10C6F000882309F4A5CFDF91CF911F910F91089561
:10C7000080912D058630D8F496E0899FF0011124A0
:10C71000E25DFA4F209174053091750531832083D5
:10C720004091790550917A0560917B0570917C0567
:10C7300042835383648375838F5F80932D050895AF
:10C740000D94A1092F923F924F925F926F927F9228
:10C750008F929F92AF92BF92CF92DF92EF92FF9211
:10C760000F931F93CF93DF9300D000D0CDB7DEB7E8
:10C770001C012B833C834D835E8369837A83C0DFF6
:10C7800083E080931F0230922B0520922A05698155
:10C790007A8170932905609328052B813C814D8116
:10C7A0005E81209324053093250540932605509300
:10C7B0002705E0922005F0922105009322051093B1
:10C7C0002305A0927905B0927A05C0927B05D0929C
:10C7D0007C0590927505809274058C8D9D8D90934B
:10C7E0001F0580931E058E8D80931D0526960FB61E
:10C7F000F894DEBF0FBECDBFDF91CF911F910F9197
:10C80000FF90EF90DF90CF90BF90AF909F908F9070
:10C810007F906F905F904F903F902F900895809100
:10C82000980D9091950D891B8F7071F49091ED0783
:10C8300092FB882780F992FD08C081E09091DE1577
:10C84000913019F080E0089581E0089520917405F9
:10C850003091750528173907E9F090937505809395
:10C8600074054093790550937A0560937B05709326
:10C870007C058658974621F41092830510922D0569
:10C880000E943C3C82E080931F0281E080932C0553
:10C8900010927E05089540E050E0BA0186E897E6E0
:10C8A000D5CFE0912D05EE2379F0E150E0932D05F1
:10C8B00086E0E89FF0011124E25DFA4F40E050E08D
:10C8C000BA0180819181C2CFE6CF0F931F93CF939E
:10C8D000DF93FC01EB018091790590917A05A0919D
:10C8E0007B05B0917C05B7FF08C0109279051092C6
:10C8F0007A0510927B0510927C058091200590911D
:10C900002105A0912205B091230540917905509110
:10C910007A0560917B0570917C0584179507A607C1
:10C92000B70744F48093790590937A05A0937B052B
:10C93000B0937C0580911F02882301F1809124052A
:10C9400090912505A0912605B09127054091790584
:10C9500050917A0560917B0570917C058C019D0159
:10C96000040F151F261F371FC901B8011995BC01F7
:10C9700080912A0590912B050E94A03D80916E0523
:10C98000811108C080911D058823B1F180911F029B
:10C99000882391F180912805909129050097B1F0A5
:10C9A0000091240510912505209126053091270539
:10C9B0004091790550917A0560917B0570917C05D5
:10C9C000400F511F621F731FFE011995E0911E0554
:10C9D000F0911F05309741F080911D05811103C032
:10C9E00080916E05811119953CD3882329F0DF9140
:10C9F000CF911F910F9155CFDF91CF911F910F9143
:10CA00000895282F109273058091790590917A05E9
:10CA1000A0917B05B0917C0581309048A105B105BE
:10CA200040F01092790510927A0510927B051092D1
:10CA30007C0580917D05882331F080917905809374
:10CA40001B0510922C0580911A051816FCF4082E6F
:10CA5000000C990B821B910920911B05022E000CE2
:10CA6000330B2817390794F097FF02C080E090E05D
:10CA700080931B05092E000CAA0BBB0B8093790534
:10CA800090937A05A0937B05B0937C0580911B055C
:10CA90006623C1F090915205891714F480935205D2
:10CAA00020915205022E000C330B2C5F3F4F482F74
:10CAB000082E000C550B2417350734F4845080934E
:10CAC00052050895809352050895882361F063E923
:10CAD00072E084E690E00F9412106AEB72E084E654
:10CAE00090E00D94121068EB71E084E190E00D94F9
:10CAF000121080E00C94849981E00C9484990C9439
:10CB0000DF9921E020931C050F94A60910921C05C3
:10CB100008950E9439B9D9CF0E94E1C7D6CFFC0150
:10CB200080810895FC01849108954F925F926F92E5
:10CB30007F928F929F92AF92BF92CF92DF92EF92AD
:10CB4000FF920F931F93CF93DF936C017B015A01E8
:10CB50002901672B31F088248394912CC0E0D0E028
:10CB600019C0F8011182108227C03701680C791CA6
:10CB700076946794E3012197A201BE01C601F501F5
:10CB800019951816190654F0892BC9F04301FFEFC7
:10CB90008F1A9F0AE814F90440F702C07E01FACF09
:10CBA000CE15DF0530F4CE0102968816990620F0E6
:10CBB0002196F801D183C0838FEF9FEF05C0F80164
:10CBC000D183C08380E090E0DF91CF911F910F91DE
:10CBD000FF90EF90DF90CF90BF90AF909F908F909D
:10CBE0007F906F905F904F9008958F929F92AF9239
:10CBF000BF92CF92DF92EF92FF920F931F93CF934A
:10CC0000DF93EC016B017A01FB01199587FD06C0EA
:10CC1000082F10E020E030E0219620C1982F907E70
:10CC2000903CC1F4082F0F7110E020E030E0480183
:10CC3000590186E0880C991CAA1CBB1C8A95D1F767
:10CC4000CE010196F60119958F7395018401082B89
:10CC5000229604C1982F907F903E19F58F70882EF0
:10CC6000912CA12CB12C16E0880C991CAA1CBB1C81
:10CC70001A95D1F7CE010196F60119958F73882A7E
:10CC800006E0880C991CAA1CBB1C0A95D1F7CE01A2
:10CC90000296F60119958F7395018401082B23964E
:10CCA000DDC0982F987F903F81F58770882E912C5A
:10CCB000A12CB12CF6E0880C991CAA1CBB1CFA957F
:10CCC000D1F7CE010196F60119958F73882AA6E057
:10CCD000880C991CAA1CBB1CAA95D1F7CE01029600
:10CCE000F60119958F73882AB6E0880C991CAA1C46
:10CCF000BB1CBA95D1F7CE010396F60119958F7337
:10CD000095018401082B2496A9C0982F9C7F983FF9
:10CD1000E9F58370882E912CA12CB12C56E0880C5B
:10CD2000991CAA1CBB1C5A95D1F7CE010196F6019D
:10CD300019958F73882A66E0880C991CAA1CBB1C65
:10CD40006A95D1F7CE010296F60119958F73882A5C
:10CD500076E0880C991CAA1CBB1C7A95D1F7CE01F1
:10CD60000396F60119958F73882AE6E0880C991CC2
:10CD7000AA1CBB1CEA95D1F7CE010496F6011995C1
:10CD80008F7395018401082B259668C0982F9E7F8C
:10CD90009C3F09F04AC08170882E912CA12CB12CA7
:10CDA00086E0880C991CAA1CBB1C8A95D1F7CE0181
:10CDB0000196F60119958F73882A96E0880C991CC4
:10CDC000AA1CBB1C9A95D1F7CE010296F6011995C3
:10CDD0008F73882A26E0880C991CAA1CBB1C2A95F4
:10CDE000D1F7CE010396F60119958F73882A36E0A4
:10CDF000880C991CAA1CBB1C3A95D1F7CE0104964D
:10CE0000F60119958F73882A46E0880C991CAA1C94
:10CE1000BB1C4A95D1F7CE010596F60119958F7383
:10CE200095018401082B269619C0982F907C903884
:10CE300049F4082F007C003871F42196CE01F601E8
:10CE40001995F7CF082F0E7F0D3F28F02196CE01C0
:10CE5000F6011995F7CF00E010E09801E114F10414
:10CE600029F0F7010083118322833383CE01DF9100
:10CE7000CF911F910F91FF90EF90DF90CF90BF90D7
:10CE8000AF909F908F9008951F93CF93DF9300D022
:10CE90001F92CDB7DEB710E0AE014F5F5F4F6FE876
:10CEA00075E6A3DE49815A816B817C81452B462B37
:10CEB000472B11F01F5FF0CF812F0F900F900F9035
:10CEC0000F90DF91CF911F9108951F93CF93DF9320
:10CED00000D01F92CDB7DEB710E0AE014F5F5F4FBD
:10CEE00062E975E682DE49815A816B817C81452B3E
:10CEF000462B472B11F01F5FF0CF812F0F900F9023
:10CF00000F900F90DF91CF911F91089510927305AC
:10CF100080916E0510926E05882341F040E050E04C
:10CF2000BA0186E69BE592DC0C94073C20914D0209
:10CF300030914E024091790550917A0560917B05C0
:10CF400070917C05C901840F951F2436310571F459
:10CF5000473051056105710514F0069732C04A3F0C
:10CF60005F4F6F4F7F4F54F506962BC02436310527
:10CF700024F48536910514F504C08436910524F413
:10CF80001DC08A3091053CF0883E43E094072CF0A8
:10CF900087EE93E002C08AE090E02817390761F03D
:10CFA00090934E0280934D021092790510927A056B
:10CFB00010927B0510927C050C94ED3384E690E092
:10CFC000E3CF8A30910504F78AE090E0E9CFCF9370
:10CFD000DF931F92CDB7DEB780919E07811103C00A
:10CFE00080EE97E02FC0211103C08EE997E02AC0A0
:10CFF0008DE0815048F0440F411DE82FF0E0E052F1
:10D00000F84F90814927F5CF809164058417A9F0E6
:10D01000409364058EE997E0698336DF90E069818B
:10D02000861B910997FF02C080E090E0809376050F
:10D030001092770588E0809321028091770590E037
:10D040008256984F0F90DF91CF910895809373058A
:10D0500010926F0510927005109271051092720572
:10D06000089580916E0510926E050895CF92DF921B
:10D07000EF92FF920F931F930E9464280091600526
:10D080001091610520916205309163056B017C016F
:10D09000C01AD10AE20AF30AF7FC13C020915F0517
:10D0A000209520935F05DC01CB018A549C4FAF4F44
:10D0B000BF4F8093600590936105A0936205B09384
:10D0C000630581E090915F05911101C080E01F919F
:10D0D0000F91FF90EF90DF90CF9008958091ED0732
:10D0E00082FF09C083FF04C080911D06811106C024
:10D0F00020E0209386058091860508958091A805FB
:10D100009091A905A091AA05B091AB050097A10542
:10D11000B10571F3BC01CD016D597F4F8F4F9F4F0A
:10D1200024E630E040E050E00F943A176091A40507
:10D130007091A5058091A6059091A7050F943A17C7
:10D14000D8CFCF9393E090931F0281111092850561
:10D150000E946428DC01CB018C509E4FAF4FBF4F23
:10D1600080937F0590938005A0938105B0938205FD
:10D1700068E873E182E090E00F941210C6E0C150BD
:10D1800049F00F94B10F62E070E080E090E00E94FF
:10D190009528F5CFCF910895AF92BF92CF92DF92AD
:10D1A000EF920F931F93CF93DF9300D01F92CDB7D1
:10D1B000DEB7809120028F3F09F44AC00E946428A4
:10D1C0000091660510916705209168053091690509
:10D1D000DC01CB01801B910BA20BB30BB7FD38C058
:10D1E0009091950D8091980D8F5F8F70981781F1B8
:10D1F000E0912002E33019F4E090650502C0E09070
:10D20000760C84E0E802F0011124E65AFC4F20E09D
:10D2100030E040E752E460817181828193810F9414
:10D22000FB1369837A838B839C83A12CB12C6501CA
:10D230008E010F5F1F4F23E93CE04FE85CE06BE895
:10D240007CE087E89CE00E944FE38FEF8093200210
:10D250000F900F900F900F90DF91CF911F910F9132
:10D26000EF90DF90CF90BF90AF9008950F931F93F2
:10D270000E94642800917F0510918005209181050E
:10D2800030918205DC01CB01801B910BA20BB30B0B
:10D29000B7FD0FC08091030185FB992790F981E0CC
:10D2A00089279091030196FF8260629B846080933E
:10D2B00085058091850581709091850591FD82603D
:10D2C00090915305891741F18130A9F028F08230FF
:10D2D00041F0833059F01EC0913089F09230A9F0AE
:10D2E00019C0992361F0933081F014C0913069F036
:10D2F000923081F404C0992341F0933059F4909115
:10D3000078059F5F9093780505C0909178059150BE
:10D3100090937805809353051F910F910895CF93B3
:10D32000DF930E94073CE4E0F1E080818F7D808301
:10D33000C5E0D1E0888180958072A3E0B1E08C9354
:10D3400080818F7B80838881809580748C936A989C
:10D35000729A54985C9A82E08093840587DF1092D9
:10D360007805DF91CF91089581E090918705911123
:10D3700001C080E00895CF93DF9320919E05211195
:10D380001EC0FC0101900020E9F73197EF01C81B96
:10D39000D90BC731D10534F031972081207C20385A
:10D3A000D9F3F4CFBC01DD27AE0187E895E00F94F7
:10D3B000231CC957DA4F188283E080931F02DF9144
:10D3C000CF910895CF93DF93CDB7DEB78E81909143
:10D3D0009E05891780F080939E059E01275F3F4F31
:10D3E0004F81588566E170E087E895E00F946C1CEA
:10D3F00083E080931F02DF91CF9108950F931F93D5
:10D40000CF93DF938C0167FF03C010929E0560E00D
:10D4100080919E0590E0262F062E000C330B2817D6
:10D4200039070CF160939E05C8010F94851BF80124
:10D43000E80FF91FEF01C01BD10BC731D10534F044
:10D4400031978491807C8038D9F3F4CFDD27AE0109
:10D45000B80187E895E00F94A61BC957DA4F1882E8
:10D4600083E080931F02DF91CF911F910F91089568
:10D470004F925F926F927F928F929F92AF92BF92E4
:10D48000CF92DF92EF92FF920F931F9385DEEEDE35
:10D490008091850582FF15C080915E05811113C0C2
:10D4A00091E090935E052091E915211103C08091D0
:10D4B0001C05892780936E051092E91581E041DEF5
:10D4C00002C010925E0589B184FB992790F981E032
:10D4D0008927109184058117B9F0809384058823EA
:10D4E00009F4A6C164EF71E080E090E00E946F84CF
:10D4F0000E94AB75123009F096C10E947B7683E0E2
:10D5000080931F020E94073C0E9464286B017C01EB
:10D5100080915A0590915B05A0915C05B0915D05E5
:10D52000A7019601281B390B4A0B5B0B57FF05C05F
:10D5300080917E05882309F426C2D701C6018C5943
:10D540009F4FAF4FBF4F80935A0590935B05A093B9
:10D550005C05B0935D0560917805062E000C770B95
:10D5600077FF03C0719561957109062E000C770B4A
:10D57000880B990B0F9496142B013C0120E030E0AE
:10D5800040E050E40F94F71587FF05C080916E05C9
:10D59000811183C093C080917305882309F456C01C
:10D5A00080906F0590907005A0907105B090720505
:10D5B00081149104A104B104E1F120E030E040E0E5
:10D5C0005FE3C301B2010F9432162B013C01C70186
:10D5D000B601681979098A099B090F9494149B0173
:10D5E000AC01C301B2010F94FB1320E030E04AE725
:10D5F00054E40F9432164B015C0120E030E040EA25
:10D6000052E40F94F71587FF0FC020E030E040EFA1
:10D6100051E4C501B4010F94F71587FD0AC02AE053
:10D6200030E040E050E009C024E630E040E050E067
:10D6300004C021E030E040E050E0C0926F05D0929D
:10D640007005E0927105F092720504C021E030E0AF
:10D6500040E050E0A09178050A2E000CBB0B0F941F
:10D66000991722E030E040E050E00F945C17809181
:10D67000790590917A05A0917B05B0917C05820F88
:10D68000931FA41FB51F8093790590937A05A093EB
:10D690007B05B0937C0510927805D701C6018856AA
:10D6A000954CAF4FBF4F8093560590935705A0936D
:10D6B0005805B093590581E080931F0220917405AD
:10D6C0003091750547E62638340741F480912102F0
:10D6D000882309F4BFC0815080932102275330442E
:10D6E00071F48091770590917605891740F49091B7
:10D6F0002102992309F4BEC0915090932102809198
:10D700006F0081FB222720F981FF05C080916F0007
:10D710008D7F80936F008091B30C9091B40CA09199
:10D72000B50CB091B60C222329F020916F00226035
:10D7300020936F003AE0B695A795979587953A950F
:10D74000D1F7009721E0A207B10520F08FEF9FEFFE
:10D75000A0E0B0E09695879520911F02211105C0A9
:10D7600030917E0531110BC151C0009741F04091BD
:10D770005405509155054817590708F047C0809146
:10D780007E05811117C0223008F08CC080910604FC
:10D79000811107C081E0809306048DEC93E00E9424
:10D7A0002C2D8DEC93E00E94632D81E080937D050C
:10D7B00080937E0583E00E94203B61E08DEC93E046
:10D7C0000E948C2DE0917405F091750519951092C9
:10D7D0007D0580917E05811171C010926E050E94B9
:10D7E0006428DC01CB018C199D09AE09BF090091A9
:10D7F00054051091550520E030E0081719072A0755
:10D800003B0720F49093550580935405809174054F
:10D81000909175058658974609F4A2C080918305BA
:10D8200081119EC071C060E082E790E3E7DD67CEC2
:10D830008AD5123009F463CE60E085E690E3DEDD40
:10D8400080917405909175058658974609F457CED6
:10D8500022D855CE8CE0809321028091540590917E
:10D8600055050197909355058093540581E0809369
:10D870001F0234CF96E09093210291E090931F0213
:10D880008F5F80937705D701C6018856954CAF4FBF
:10D89000BF4F8093560590935705A0935805B093BA
:10D8A00059052DCF243030F0243009F06FCF10927D
:10D8B0001F026CCF81E080931F0268CF8DEC93E054
:10D8C0000E94672D91E0811101C090E090937E0548
:10D8D000992309F482CF0E946428DC01CB018C19C2
:10D8E0009D09AE09BF09C0905405D0905505E12CA3
:10D8F000F12CC816D906EA06FB0608F044C090933E
:10D900005505809354053FC0809156059091570569
:10D91000A0915805B0915905C81AD90AEA0AFB0A1C
:10D92000F7FE0E944B6480917E0581112CC080918E
:10D930001F02813091F0833031F51F910F91FF90DC
:10D94000EF90DF90CF90BF90AF909F908F907F909F
:10D950006F905F904F900C943C3C10921F0213C04C
:10D9600048E9C40E4AE3D41EE11CF11CC0925605DE
:10D97000D0925705E0925805F0925905D4CF009700
:10D9800009F418CFF4CE1F910F91FF90EF90DF9024
:10D99000CF90BF90AF909F908F907F906F905F904F
:10D9A0004F90089561E02ADD0C944B64CF93DF9390
:10D9B0001F921F92CDB7DEB789839A83B0DC89812D
:10D9C0009A81F0DF0F900F90DF91CF910C940C3C77
:10D9D0008091ED0782FD05C08091DE15823061F4F3
:10D9E00010C080919E07811103C080EE97E002C0B5
:10D9F0008EE997E061E0BFCC813031F087E390E3BE
:10DA000005C088E590E302C08CE490E36FEFF6CCAC
:10DA100086E897E69093750580937405089561E014
:10DA2000FC0180810E94892A8FEF0C94488ECF934D
:10DA3000DF93EC018A810E94098E60E08881DF918A
:10DA4000CF910C94892A8F929F92AF92BF92EF92BE
:10DA5000FF920F931F93CF93DF93EC018B017A0119
:10DA60000E9464284B015C012CE2820E21E0921E90
:10DA7000A11CB11C0E94228E8B838F3F61F40E94F7
:10DA80006428DC01CB0188199909AA09BB09B7FDF3
:10DA9000F1CF81E10DC08E3F51F4B701C8010E9462
:10DAA000298E0E94228E0E94228E11E003C08FE0F8
:10DAB000898310E0CE01B3DF812FDF91CF911F91D9
:10DAC0000F91FF90EF90BF90AF909F908F9008952F
:10DAD000CF92DF92EF92FF926A017B010E9464284D
:10DAE000C60ED71EE81EF91E0E94228E8F3F61F0DF
:10DAF0000E946428DC01CB018C199D09AE09BF0985
:10DB0000B7FDF2CF80E001C081E0FF90EF90DF90A1
:10DB1000CF900895EF92FF921F93CF93DF9300D0A1
:10DB20001F92CDB7DEB77C01162F29833A834B8332
:10DB30005C837DDF48E552E060E070E0C701C8DF4C
:10DB4000812F80640E94488E8C810E94488E8B8138
:10DB50000E94488E8A810E94488E89810E94488E48
:10DB6000112311F087E801C085E90E94488E1C301E
:10DB700011F40E94228E10E00E94228EF70183830E
:10DB800087FF04C01F3F11F01F5FF6CF0F900F906B
:10DB90000F900F90DF91CF911F91FF90EF9008951C
:10DBA0008F929F92AF92BF92CF92DF92EF92FF92AD
:10DBB0000F931F93CF93DF93EC01162F1C821982D2
:10DBC00048830E9464286B017C0120EDC20E27E08F
:10DBD000D21EE11CF11CA89561E088810E94892A6F
:10DBE00061E088810E944D2A0E941A8E85E08A8316
:10DBF0000E94098E0AE08FEF0E94488E0150D9F7EB
:10DC0000A89520E030E0A90160E0CE0183DF8B839E
:10DC1000813061F00E946428DC01CB018C199D09E0
:10DC2000AE09BF09B7FDEDCF81E055C0A8952AEA3E
:10DC300031E040E050E068E0CE016CDF853011F467
:10DC400081E009C004E00E94228E8B830150D9F745
:10DC50008A3A51F482E08C83A8958C81823081F0DD
:10DC6000812C912C540111C00E946428DC01CB014D
:10DC70008C199D09AE09BF09B7FDD9CF82E02BC031
:10DC8000812C912CA12C80E4B82E20E030E0A90159
:10DC900067E3CE013FDFA501940169E2CE013ADFDF
:10DCA0008B83882361F00E946428DC01CB018C19EE
:10DCB0009D09AE09BF09B7FDE8CF8AE00CC08C8191
:10DCC0008230D1F420E030E0A9016AE3CE0122DF06
:10DCD000882329F088E08983CE01A1DE16C00E9446
:10DCE000228E807C803C11F483E08C830E94228E03
:10DCF0000E94228E0E94228ECE0191DE173018F4EF
:10DD00001A8381E003C088E1898380E0DF91CF91AD
:10DD10001F910F91FF90EF90DF90CF90BF90AF9049
:10DD20009F908F9008950F931F93CF93DF93EC01F3
:10DD300089018C81833039F089E0440F551F661FBB
:10DD4000771F8A95D1F79A01AB0161E1CE01E2DE3E
:10DD5000811109C040E052E0B801CE01DF91CF91BE
:10DD60001F910F9170CE84E08983CE0158DE80E050
:10DD7000DF91CF911F910F910895CF93DF93EC0125
:10DD8000862FBA010E944D8E8FEF0E94488E8FEF32
:10DD90000E94488E0E94228E8B83982F9F7195300F
:10DDA00031F083E18983CE013ADE80E001C081E079
:10DDB000DF91CF9108950F931F93CF93DF93EC01E1
:10DDC00089018C81833039F089E0440F551F661F2B
:10DDD000771F8A95D1F79A01AB0168E1CE019ADEEF
:10DDE00081111EC0A8016EEFCE01C7DF8823E1F0CC
:10DDF00048E552E060E070E0CE016ADE882371F011
:10DE000020E030E0A9016DE0CE0184DE81110AC07E
:10DE10000E94228E811106C011E007C087E103C075
:10DE200086E001C086E1898310E0CE01F8DD812F14
:10DE3000DF91CF911F910F910895CF93DF931F92A0
:10DE4000CDB7DEB72091EB153091EC15CE010196E0
:10DE50002115310519F0821B930B02C0815F95419A
:10DE60000F90DF91CF910895FC01238121110C9433
:10DE7000D57F08958091ED07847F8B7F8093ED0798
:10DE80001092A4051092A5051092A6051092A70560
:10DE90001092A8051092A9051092AA051092AB0540
:10DEA00010921906109258068EE091E0E9E5F6E02E
:10DEB000DF019C011D9221503040E1F78FEF8093EC
:10DEC0009D070895FC0120E03EE2DB014C914032C9
:10DED00041F0283011F430833196DB014C914083BE
:10DEE00031962F5F6F5F7F4F2B3079F71082089547
:10DEF0002F923F924F925F926F927F928F929F925A
:10DF0000AF92BF92CF92DF92EF92FF920F931F9347
:10DF1000CF93DF93CDB7DEB7C356D1090FB6F894D0
:10DF2000DEBF0FBECDBF8C015B014A014DB65EB6B0
:10DF3000312C7E0187E5E80EF11C9BE1292E4EE98C
:10DF400057E0BE016F5F7F4FC5010E94457E1816E6
:10DF50000CF005C18C85282F2871203109F074C080
:10DF60009091A3059150923008F46EC06DB67EB6C4
:10DF7000BE016F5F7F4FC701A5DF0115110521F0BD
:10DF8000F8018081811173C021E081E090E0F70108
:10DF900001900020E9F73197EE19FF09E80FF91F0A
:10DFA00032968DB79EB78E1B9F0B0FB6F8949EBF0F
:10DFB0000FBE8DBFEDB7FEB731966F01211102C0C4
:10DFC000B80102C06AE673E0C6010F940E1CB701E7
:10DFD000C6010F94F81B6AE673E0C6010F94F81BA4
:10DFE0001CAE1FAE21E0A701B501CE01CC960E9468
:10DFF000D18181110DC08091A305811109C00E94BA
:10E00000248A82E692E30E94168AC7010E94DF8C6E
:10E01000FE01FC96DE019196822D01900D928A956B
:10E02000E1F740E050E0BE016F5D7F4FC60160DF69
:10E03000CE01819619DFCE01CC9616DF0FB6F8948B
:10E040007EBE0FBE6DBE7BCF9981992309F487C038
:10E05000953E09F474CF9E3209F471CF90919E07DA
:10E060009E3209F46CCF8A7009F069CF0AC0F801BA
:10E0700001900020E9F73197CF01801B910B20E040
:10E0800086CF81E0203109F080E09091ED0780FBA0
:10E0900094F99093ED07811108C08985873409F0C0
:10E0A0004ECF8A858E3709F44ACF8091A3058130FF
:10E0B00021F068F08230B9F142CF8091A1059091B2
:10E0C000A20501969093A2058093A10538CFBE01C9
:10E0D0006F5F7F4F80EE97E0F5DE0115110511F0BF
:10E0E000680105C080EEC82E87E0D82E08C0F60172
:10E0F00081916F018823B1F30E94888CF8CFF601DB
:10E1000081916F01882319F00E94888CF8CF80E2FA
:10E110000E94888C6D8D7E8D8F8D98A14AE050E095
:10E120000E94958D0CCFBE016F5F7F4F80EE97E010
:10E13000C9DE8114910441F060EE77E0C4010F94D0
:10E14000E51B892B51F40BC0832D90E020919F0596
:10E150003091A0058217930711F03394F0CE0FB6DB
:10E16000F8945EBE0FBE4DBECD59DF4F0FB6F8948A
:10E17000DEBF0FBECDBFDF91CF911F910F91FF90FA
:10E18000EF90DF90CF90BF90AF909F908F907F9057
:10E190006F905F904F903F902F900895CF93DF93B3
:10E1A000CDB7DEB76B970FB6F894DEBF0FBECDBF0D
:10E1B0001092A30540E050E0BA0182E897E00E9487
:10E1C000F47E8BE1E2E8F7E0DE01119601900D921A
:10E1D0008A95E1F740E050E0BE016F5F7F4F80E03D
:10E1E00090E086DECE0101963FDE6B960FB6F89486
:10E1F000DEBF0FBECDBFDF91CF9108950F931F9368
:10E20000CF93DF93CDB7DEB72D970FB6F894DEBF6F
:10E210000FBECDBF80911D06882391F0BE016F5FB8
:10E220007F4F8AE196E00E94677C8E010F5F1F4F4F
:10E23000F80181918F01882339F00E94888CF8CFF2
:10E2400088E592E30E94168A8AE00E94888C2D96C7
:10E250000FB6F894DEBF0FBECDBFDF91CF911F91F7
:10E260000F910895CF92DF92EF92FF920F931F9339
:10E27000CF93DF93CDB7DEB7EDB6FEB6DC010D90E0
:10E280000020E9F79D01281B390B2C5F3F4F4DB74C
:10E290005EB7421B530B0FB6F8945EBF0FBE4DBF67
:10E2A0000DB71EB70F5F1F4F9F938F9382E192E3CD
:10E2B0009F938F931F930F930F943D1C680154E01D
:10E2C000C50ED11C0F900F900F900F900F900F90D4
:10E2D000F6018081882349F0082E000C990B0F94D9
:10E2E000691BF60181936F01F3CFC8010F94A60952
:10E2F0008EE092E30F94A1090FB6F894FEBE0FBE14
:10E30000EDBEDF91CF911F910F91FF90EF90DF90C5
:10E31000CF9008958091ED0783FF03C084608093C0
:10E32000ED0708951092BA0A8091ED078F7D8B7FDB
:10E330008093ED070E94D65A882321F08AE196E067
:10E340000C94D57F0895EEDF8091ED07877F809351
:10E35000ED0708950F931F93CF93DF938B01EA018D
:10E36000DB016D917C910E94677CD801ED91FC915D
:10E370009081888191110EC08936B0F48FE280833C
:10E38000F8018081918101969183808388818F5FDC
:10E3900088830AC0893680F73196D801ED93FC93C3
:10E3A00088818F5F8883E1CFDF91CF911F910F919B
:10E3B00008950F931F93CF93DF9300D0CDB7DEB7AF
:10E3C0009C012F5F3F4F3B832A832FE2FC01208378
:10E3D00081E0898310E00BE180915806181770F4F2
:10E3E000019FC0011124AE014F5F5F4FBE016E5F00
:10E3F0007F4F875A994FAEDF1F5FEECF89818B35F4
:10E4000070F4AE014F5F5F4FBE016E5F7F4F8AE1D8
:10E4100096E0A0DF8A819B8101979B838A83EA81B2
:10E42000FB8110820F900F900F90DF91CF911F9181
:10E430000F9108958091ED0782FF1FC08FED90E34B
:10E440000E94168A6091A4057091A5058091A60589
:10E450009091A7054AE050E00E948A8D8FE20E94C9
:10E46000888C6091A8057091A9058091AA0590916A
:10E47000AB054AE050E00C94958D8EEC90E30C9443
:10E48000168AEF92FF920F931F93CF93DF938C0125
:10E49000FC0101900020E9F73197EF01C81BD90B6F
:10E4A00010921A066EE470E00F94031C7C01009732
:10E4B00029F4FE013197E00FF11F0EC060E270E019
:10E4C0000F94031C8C010F5F1F4F6AE270E0C701BD
:10E4D0000F94031CFC0131978DE081838AE08283D5
:10E4E0001382B8018AE196E00E94648480911A0642
:10E4F000882361F00E94278A87EB90E3DF91CF9118
:10E500001F910F91FF90EF900C94168ADF91CF919D
:10E510001F910F91FF90EF9008958AE196E00E947D
:10E520008A7F8AE196E00E94D57F8091ED078D7FFA
:10E530008E7F8093ED071092A4051092A50510928E
:10E54000A6051092A70581E08093B30A08950F9362
:10E550001F93CF93DF93CDB7DEB76B970FB6F894C9
:10E56000DEBF0FBECDBF8B0122E02093A3059093A9
:10E57000A00580939F0540E050E0BA0187E697E050
:10E580000E94F47E8BE1E7E6F7E0DE011196019050
:10E590000D928A95E1F7A801BE016F5F7F4F80E081
:10E5A00090E0A6DCCE0101965FDC6B960FB6F89486
:10E5B000DEBF0FBECDBFDF91CF911F910F910895A8
:10E5C000CF93DF93CDB7DEB76B970FB6F894DEBF6E
:10E5D0000FBECDBF81E08093A3051092A2051092DB
:10E5E000A10540E050E0BA0187E697E00E94F47E82
:10E5F0008BE1E7E6F7E0DE01119601900D928A9536
:10E60000E1F740E050E0BE016F5F7F4F80E090E0B7
:10E610006FDCCE01019628DC8091A1059091A205C6
:10E620006B960FB6F894DEBF0FBECDBFDF91CF91D2
:10E6300008952F923F924F925F926F927F928F92A6
:10E640009F92AF92BF92CF92DF92EF92FF920F9381
:10E650001F93CF93DF93CDB7DEB76C970FB6F894C7
:10E66000DEBF0FBECDBF5C014C8F2DB63EB619820A
:10E670001C82FB0180819E012F5F3F4F49018F3239
:10E6800039F087E697E0F501918380838B0162C0C2
:10E6900082E897E0F501918380838B010F5F1F4F24
:10E6A0000115110509F456C04DB65EB66FE270E073
:10E6B000C8010F94031C3C010817190708F04AC051
:10E6C0007C01E01AF10AFF24C70101962DB73EB77D
:10E6D000281B390B0FB6F8943EBF0FBE2DBF8DB768
:10E6E0009EB701966C01A701B8010F94231CF60197
:10E6F000EE0DFF1D10823C8D332319F0C6010E94E0
:10E70000DF8CF5016081718121E0A601C4010E94C6
:10E71000D181811113C0B6018AE990E30E942A8A4F
:10E720008EE20E94888C8AE00E94888C0FB6F89452
:10E730005EBE0FBE4DBE00E010E00CC0F501918240
:10E74000808283010F5F1F4F0FB6F8945EBE0FBE2D
:10E750004DBEA6CFC40188DBC8010FB6F8943EBEFB
:10E760000FBE2DBE6C960FB6F894DEBF0FBECDBFA8
:10E77000DF91CF911F910F91FF90EF90DF90CF909D
:10E78000BF90AF909F908F907F906F905F904F90D1
:10E790003F902F9008950F931F93CF93DF931F9275
:10E7A0001F92CDB7DEB72091ED0723FF27C0BC0134
:10E7B00040E0CE0101963DDF8C010097F9F0BC01ED
:10E7C00089819A810E94AB82B801882381F089E017
:10E7D00091E30E942A8A8AE00E94888C1092A40504
:10E7E0001092A5051092A6051092A70507C081EF0B
:10E7F00090E30E942A8A8EE20E94888C0F900F90EC
:10E80000DF91CF911F910F910895EF92FF920F9397
:10E810001F93CF93DF9300D0CDB7DEB72091ED07E4
:10E8200023FF07C1F42EE62E8C010E94D65A8823BE
:10E8300009F451C0FF2009F45BC0809119068823B8
:10E8400059F00E94278A89EC91E30E94168A80E0A1
:10E8500090E00F946011EDC08CEA95E0AADDE091A4
:10E86000190684E0E89FF0011124EB5EF94F8091D6
:10E87000A4059091A505A091A605B091A705808358
:10E880009183A283B3830E94248AB80180EB91E331
:10E890000E942A8A8091190699E6899FB001112465
:10E8A00064557A4F85EA91E30E942A8A4091A40533
:10E8B0005091A5056091A6057091A7058FE991E398
:10E8C0000E948B8A8AE00E94888C809119068F5F53
:10E8D0008093190625C0FF2039F00E94248A8FE812
:10E8E00091E30E94168A1CC01092190622E001C012
:10E8F00021E02B830E94248A8AE891E30E94168AF1
:10E900002B81213009F492C08EE791E30E94168A90
:10E91000B80186E791E30E942A8A8AE00E94888CE7
:10E9200001DD40E0B801CE01019683DE8C01009745
:10E9300009F47FC069817A81EE2009F44BC021E09F
:10E94000AC018AE196E00E94D181882309F43EC09F
:10E9500080912B0690912C06A0912D06B0912E0649
:10E960008093A8059093A905A093AA05B093AB0541
:10E970001092A4051092A5051092A6051092A70565
:10E98000B80188E691E30E942A8A4091A805509137
:10E99000A9056091AA057091AB0580E691E30E94FC
:10E9A0008B8A8AE00E94888C81E591E30E94168A16
:10E9B000B80180E090E0CBDD80919E07811102C01C
:10E9C000C80102C08EE997E060E02DC0B8018DE378
:10E9D00091E30BC026E5AC018AE196E00E94D1816B
:10E9E00081110CC0B80189E291E30E942A8A8EE26B
:10E9F0000E94888C8AE00E94888C1BC08091ED0761
:10EA000081608093ED07B80180E090E0A0DD109276
:10EA1000B30AB80187E191E30E942A8A8AE00E9442
:10EA2000888C60E0C8010E94BB6903C084E891E360
:10EA30006DCF0F900F900F90DF91CF911F910F919D
:10EA4000FF90EF9008952091ED0722602093ED074D
:10EA500040E060E0DACE0F931F93CF93DF93CDB702
:10EA6000DEB76B970FB6F894DEBF0FBECDBF8C013B
:10EA700019821C8280916A07811103C062E877E0E5
:10EA800002C067E677E021E0A801CE0101960E946E
:10EA9000D1818823F1F08BE1FE013196A7E6B7E042
:10EAA00001900D928A95E1F7A0915806AA30D8F40A
:10EAB00081E08A0F809358068BE18A9FD001112450
:10EAC000A75AB94FE7E6F7E001900D928A95E1F772
:10EAD0000AC00E94248AB80184E890E30E942A8A2E
:10EAE0008AE00E94888CCE010196BED96B960FB643
:10EAF000F894DEBF0FBECDBFDF91CF911F910F9174
:10EB00000895809158068823C9F081508093580653
:10EB1000882359F090E001972BE1289FF001299F6D
:10EB2000F00D1124E75AF94F02C0E2E8F7E08BE15B
:10EB3000A7E6B7E001900D928A95E1F7809158061B
:10EB400008958BE1E2E8F7E0A7E6B7E001900D92C7
:10EB50008A95E1F708958091ED07877F8093ED070F
:10EB600080918507882321F082E897E00E94D57F75
:10EB700045E360E083E596E013D8811105C00E946B
:10EB8000248A8AE492E32AC041E063E576E085E3E3
:10EB900096E07DD481110DC040E063E576E085E329
:10EBA00096E075D4811105C00E94278A86E392E31E
:10EBB00015C065E376E082E897E0E5D6811105C0EF
:10EBC0000E94278A85E292E309C08091ED07886060
:10EBD0008093ED070E94248A89E192E30E94168ABD
:10EBE000B0DF83E080931F020895AF92BF92CF926F
:10EBF000DF92EF92FF921F93CF93DF93CDB7DEB7F3
:10EC0000A8970FB6F894DEBF0FBECDBF80919D07C9
:10EC100087FD61C08091ED0782FD5DC083FF9BDFB2
:10EC20008091ED0783FF54C080919D07082E000C52
:10EC3000990BC0969F938F938EEA90E39F938F9347
:10EC40006E0181E2C80ED11CDF92CF920F943D1C61
:10EC500040E050E0BA0182E897E00E94F47E0F9015
:10EC60000F900F900F900F900F90FE0131967F0143
:10EC700040E050E0B70182E897E00E94457E181618
:10EC80003CF5F70101900020E9F731971E2F1E197E
:10EC9000115068F05701A10EB11C17FDBA94F5018F
:10ECA000808190E00F94691BF5018083F1CF8A8504
:10ECB0008E37F1F245E050E0B601C7010F94151C04
:10ECC000892BB1F6C601CEDA80919D078F5F01C016
:10ECD0008FEF80939D07A8960FB6F894DEBF0FBE06
:10ECE000CDBFDF91CF911F91FF90EF90DF90CF903C
:10ECF000BF90AF90089510929D0723CF61CC0E94E2
:10ED0000EAD38AE196E00E94D57F80911906882394
:10ED100029F181508093190629E6829FC0011124B0
:10ED200041E061E084559A4F70DDE091190684E07E
:10ED3000E89FF0011124EB5EF94F4081518162811F
:10ED400073814093A4055093A5056093A605709325
:10ED5000A7058AE196E00E94F47EDCCAE3DA0E940D
:10ED6000C4D30F9451100F9496106D337105810523
:10ED7000910520F080E890E30F94A1091092860598
:10ED80000C94E86C10928207109285071092670726
:10ED900010926A0780E090E0FC01E75AF94F108278
:10EDA00013824B968E3021E09207B1F789E1809370
:10EDB00054061092570610924C0610921A061092A2
:10EDC0001D060895CF93DF938AE196E04DD8C7E6FC
:10EDD000D7E06B97CE0148D886E0C935D807C9F788
:10EDE00087E697E041D882E897E0DF91CF913CC871
:10EDF000CF938091F2078823B9F14091F5095091A2
:10EE0000F6096091F7097091F80925EF37E08091D4
:10EE1000F3079091F4070E94DB6EC82F811102C0A6
:10EE2000C0E023C04091EE075091EF076091F007DA
:10EE30007091F107411551056105710591F025EFBC
:10EE400037E08091F3079091F4070E94DB6E8823EE
:10EE500039F31092EE071092EF071092F00710921C
:10EE6000F1071092F20701C0C1E08C2FCF910895F5
:10EE7000CF92DF92EF92FF92CF936B017C01C42F70
:10EE80008091F5099091F609A091F709B091F809E0
:10EE90008C159D05AE05BF05C9F0AADF811102C022
:10EEA00080E018C025EF37E0B701A6018091F30795
:10EEB0009091F4070E94936E882391F3C092F50914
:10EEC000D092F609E092F709F092F80981E0C111B9
:10EED0008093F207CF91FF90EF90DF90CF9008954D
:10EEE000CF92DF92EF92FF920F931F93CF93DF9316
:10EEF000FC0181859285A385B4850196A11DB11D74
:10EF000084179507A607B70710F480E060C08789CB
:10EF1000803149F4BB27A72F962F852FC388D4882B
:10EF2000E588F6880FC0803281F783899489A589A6
:10EF3000B6896A017B01C7E0F694E794D794C79439
:10EF4000CA95D1F78C0D9D1DAE1DBF1DE9016A014B
:10EF50007B018F014091F5095091F6096091F70905
:10EF60007091F80984179507A607B70731F040E0BC
:10EF7000BC01CD017DDF882341F2F8018789803112
:10EF800079F4B701A601552766277727440F551F47
:10EF9000FA01EB50F84F80819181A0E0B0E012C0FF
:10EFA000B701A6014F77552766277727440F551FCE
:10EFB000440F551FFA01EB50F84F80819181A281D7
:10EFC000B381BF7088839983AA83BB8381E0DF917B
:10EFD000CF911F910F91FF90EF90DF90CF90089508
:10EFE0004F925F926F927F92AF92BF92CF92DF92D9
:10EFF000EF92FF920F931F93CF93DF9300D01F9256
:10F00000CDB7DEB78C0149835A836B837C8359016A
:10F01000C12CD12C7601412C82E0582E612C712C10
:10F0200049815A816B817C819E012F5F3F4FC801CE
:10F0300057DF882341F1D301C201F801058404C0E0
:10F04000880F991FAA1FBB1F0A94D2F7C80ED91E9A
:10F05000EA1EFB1E49815A816B817C818789803140
:10F0600039F481E0483F5F4F6105710538F4D8CF2E
:10F0700081E0483F5F4F6F4F7F4090F2F501C082C3
:10F08000D182E282F3820F900F900F900F90DF9168
:10F09000CF911F910F91FF90EF90DF90CF90BF9095
:10F0A000AF907F906F905F904F9008954F925F92D6
:10F0B0006F927F928F929F92AF92BF92CF92DF9288
:10F0C000EF92FF920F931F93CF93DF93EC016A01AE
:10F0D0007B0128013901423051056105710510F4A9
:10F0E00080E064C089859A85AB85BC850196A11DA9
:10F0F000B11D84179507A607B70790F38F89803154
:10F1000049F48D2C9E2CAF2CBB248B899C89AD8916
:10F11000BE890FC0803221F78B889C88AD88BE885D
:10F12000DB01CA0157E0B695A795979587955A9543
:10F13000D1F7880E991EAA1EBB1E41E0C501B4017D
:10F1400097DE882369F29F89903161F4DD24EE24F3
:10F15000FF249601220F331FF901EB50F84F518223
:10F16000408211C0E894C7F8DD24EE24FF24960104
:10F17000220F331F220F331FF901EB50F84F40824B
:10F180005182628273829A89923080F04D815E81D1
:10F190006F817885840E951EA61EB71E8092EE079D
:10F1A0009092EF07A092F007B092F107DF91CF9114
:10F1B0001F910F91FF90EF90DF90CF90BF90AF9095
:10F1C0009F908F907F906F905F904F9008952F92B7
:10F1D0003F924F925F926F927F928F929F92AF92E7
:10F1E000BF92CF92DF92EF92FF920F931F93CF9334
:10F1F000DF93CDB7DEB72F970FB6F894DEBF0FBE03
:10F20000CDBF1C014D835E836F8378873B872A8740
:10F21000FC0181859285A385B4858C019D010F5FDA
:10F220001F4F2F4F3F4F0C871D872E873F87AA8583
:10F23000BB85CD90DD90ED90FC90C114D104E1042C
:10F24000F10431F0BFEFCB1ADB0AEB0AFB0A10C066
:10F25000F101C080D180E280F380F1E0F9870D8177
:10F260001E812F813885013011052105310509F0F6
:10F27000198646015701412C512C3201F10181853B
:10F280009285A385B485481659066A067B0608F060
:10F290004EC00C851D852E853F85081519052A054C
:10F2A0003B0550F482E0882E912CA12CB12C92E0E9
:10F2B000C92ED12CE12CF12C9E012F5F3F4FB501BF
:10F2C000A401C1010DDE882391F149815A816B812E
:10F2D0007C81D501C4010196A11DB11D452B462B92
:10F2E000472B19F06C017D010FC0AC01BD014C1919
:10F2F0005D096E097F090D811E812F8138854017B8
:10F3000051076207730741F01FEF411A510A610A62
:10F31000710A4C015D01B2CF0FEF1FEF2FEF3FE0FD
:10F32000B501A401C101C2DE8D83811113C01D820C
:10F330003DC02401350121E0421A510861087108DD
:10F3400095018401B301A201C101B0DE882379F3E4
:10F3500053014201C814D904EA04FB0450F3AA85FE
:10F36000BB854D915D916D917C9141155105610574
:10F370007105A9F4EA85FB85C082D182E282F3821D
:10F38000F985FF2399F00FEFC01AD00AE00AF00ABE
:10F39000D101CD92DD92ED92FC92139707C09701B7
:10F3A0008601C10183DE8111E5CFC1CF8D812F960A
:10F3B0000FB6F894DEBF0FBECDBFDF91CF911F9186
:10F3C0000F91FF90EF90DF90CF90BF90AF909F9004
:10F3D0008F907F906F905F904F903F902F90089507
:10F3E000AF92BF92CF92DF92EF92FF920F931F9353
:10F3F000CF93DF9300D01F92CDB7DEB75C016A01D7
:10F400007B0182E090E0A0E0B0E0F5018083918391
:10F41000A283B3839E012F5F3F4FB701A601C501B1
:10F420005FDD882321F100E010E09801B701A6011B
:10F43000C5013CDE8823D9F0C980DA80EB80FC80EE
:10F44000F5018789803149F481E0F8EFCF16FFEFAD
:10F45000DF06E104F10460F4DDCF81E098EFC91626
:10F460009FEFD906E9069FE0F90610F4D3CF80E0BC
:10F470000F900F900F900F90DF91CF911F910F91F0
:10F48000FF90EF90DF90CF90BF90AF9008954F9294
:10F490005F926F927F928F929F92AF92BF92FF92F4
:10F4A0000F931F93CF93DF93EC01142F7093F40706
:10F4B0006093F3071F8A82E090E0A0E0B0E08883C9
:10F4C0009983AA83BB831092F2071092EE071092E1
:10F4D000EF071092F0071092F1078FEF9FEFDC011A
:10F4E0008093F5099093F609A093F709B093F80972
:10F4F000442371F1453008F0E0C040E060E070E086
:10F50000CB01B6DC882309F4D8C020E1129FA0010A
:10F5100011244B51584FFA01E254FE4F80818F77EE
:10F5200009F0CBC03C9680819181A281B381843661
:10F530009105A105B10508F4C0C034978080918081
:10F54000A280B38081149104A104B10421F4B5C058
:10F55000812C912C540140E0C501B40189DCF82EC6
:10F56000882309F4AAC080910008909101088115B0
:10F57000924009F0A2C090910508992309F49DC01A
:10F580002091030830910408232B09F496C0809140
:10F590000208882309F491C09A8B8C831D8690E021
:10F5A00061E070E02D85E22FAB01022E02C0440F16
:10F5B000551F0A94E2F78417950731F031E0320FB6
:10F5C0003D87283078F379C020910B0830910C08E2
:10F5D0002115310519F040E050E008C020911908CC
:10F5E00030911A0840911B0850911C082D833E83CE
:10F5F0004F835887809103089091040824013501B6
:10F60000480E591E611C711C4B8A5C8A6D8A7E8A69
:10F610000091060810910708198F088FA09105081E
:10F62000B0E00F948F17460E571E681E791E4A8E43
:10F630005B8E6C8E7D8E85E0000F111F8A95E1F741
:10F6400001501E4F012F11270695400E511E611CBF
:10F65000711C4E865F86688A798A209108083091ED
:10F6600009082115310521F0890120E030E008C0AA
:10F67000009115081091160820911708309118086C
:10F68000B501A4014419550966097709400F511FB6
:10F69000621F731F04C07695679557954795EA9545
:10F6A000D2F749875A876B877C87453F8FE0580799
:10F6B0006105710520F48CE08F8BF12C15C0453F5E
:10F6C0005F4F6105710510F480E10DC08091210844
:10F6D00090912208A0912308B09124088A8F9B8FD3
:10F6E000AC8FBD8F80E28F8B8F2DDF91CF911F91DB
:10F6F0000F91FF90BF90AF909F908F907F906F90F1
:10F700005F904F900895CF93DF93EC019C012C5FA5
:10F710003F4F41E050E060E070E0898D9A8D57DD09
:10F72000882399F04D895E896F89788D452B462B0A
:10F73000472B59F44C815D816E817F814D8B5E8BAF
:10F740006F8B788F998190689983DF91CF9108951D
:10F75000CF92DF92EF92FF920F931F93CF93DF939D
:10F76000DC0151964D915D916D917C915497403E95
:10F770005F4F6F41710510F010E067C0EC01C3DF0F
:10F780008823D1F335DB182F8823B1F3E98DFA8D67
:10F790008C819D81AE81BF810297A109B109058449
:10F7A00004C0880F991FAA1FBB1F0A94D2F7C684F2
:10F7B000D784E088F188C80ED91EEA1EFB1E81E0BE
:10F7C0008093F207C092F509D092F609E092F7090A
:10F7D000F092F80980E092E0E5EFF7E0DF019C01AC
:10F7E0001D9221503040E1F701E0E98DFA8D8481CE
:10F7F000081798F425EF37E0B701A601400F511D17
:10F80000611D711D8091F3079091F4070E94DB6EDA
:10F81000882309F4B1CF0F5FE8CF40E052E060E009
:10F8200070E0058404C0440F551F661F771F0A94BB
:10F83000D2F789899A89AB89BC89480F591F6A1FF9
:10F840007B1F498B5A8B6B8B7C8B812FDF91CF91E8
:10F850001F910F91FF90EF90DF90CF900895CF937D
:10F86000DF93EC0141E0611101C040E06C857D85D2
:10F870008E859F85FDDA882341F0888920E2829F6A
:10F88000C00111248B50984F02C080E090E0DF91BE
:10F89000CF910895FC0120E090E08EE2308130327B
:10F8A00069F0283029F4DB01A90FB11D8C939F5F0B
:10F8B000DB01A90FB11D30813C939F5F2F5F319613
:10F8C0002B3061F7FB01E90FF11D10820895CF93F2
:10F8D000DF93FC012381211102C080E010C022507F
:10F8E000223028F48FE2FB018083118207C0EB01F4
:10F8F00060E0B5DF009789F3BE01CCDF81E0DF91E6
:10F90000CF9108952BE030E22150FB01E20FF11D71
:10F9100030832111F9CFDC0197E03A2FEB2F8D9145
:10F9200081110AC0DA013C931196EC9381E0FB014E
:10F930009081903239F525C08F32A1F38E3229F4AF
:10F940009A30F9F028E09AE0E8CFE6E7F2E3349164
:10F95000332321F031963813FACF13C0921788F071
:10F96000813278F08F3769F031E0320FFB01E20F1E
:10F97000F11D2FE9280F2A3108F480528083232FAC
:10F98000CCCF80E008950F931F93CF93DF93FC01BA
:10F990002381222311F080E043C08B01EC01FB01A5
:10F9A0008789803131F18032B1F783E08B83F801B0
:10F9B000428D538D648D758D4D8B5E8B6F8B788FE3
:10F9C0009E012F5E3F4FC8010BDB882321F31A8F66
:10F9D000098F81E08983188619861A861B861C8206
:10F9E0001D821E821F82188A1C861D861E861F8607
:10F9F00017C082E08B831D8A1E8A1F8A188EFB0126
:10FA0000808D918DA0E0B0E025E0880F991FAA1F9E
:10FA1000BB1F2A95D1F7898B9A8BAB8BBC8BD7CF29
:10FA2000DF91CF911F910F9108952F923F924F92A6
:10FA30005F926F927F928F929F92AF92BF92CF927E
:10FA4000DF92EF92FF920F931F93CF93DF9300D03B
:10FA50001F92CDB7DEB79C838B834B015A01DC012B
:10FA600013968C91811103C08FEF9FEFE1C0EB8162
:10FA7000FC81818180FFF8CFEB81FC8181899289B3
:10FA8000A389B4894085518562857385841B950B54
:10FA9000A60BB70BA50160E070E084179507A607D9
:10FAA000B70708F45C0175018B819C8104969A83E9
:10FAB0008983612C92E0792EE114F10409F48AC063
:10FAC000AB81BC8118964D915D916D917C911B9796
:10FAD0006A01B1E0DB22EB81FC8123811A012B0159
:10FAE00089E056944794379427948A95D1F7818D6D
:10FAF000928D223061F4FC01828D938DA48DB58DA1
:10FB0000BC01CD01620D731D841D951D49C0DC0132
:10FB100014961C9111501221C114D104F9F4111141
:10FB20001DC0452B462B472B59F4EB81FC81858961
:10FB30009689A789B08D84839583A683B7830EC0E9
:10FB4000AB81BC8114964D915D916D917C9117971D
:10FB500029813A81C5D9882309F486CFEB81FC81BC
:10FB6000218D328D84819581A681B7810297A1096B
:10FB7000B109F901058404C0880F991FAA1FBB1F92
:10FB80000A94D2F74685578560897189840F951F3D
:10FB9000A61FB71FBC01CD01610F711D811D911DF5
:10FBA00093012C193D0987012E153F0508F48901A1
:10FBB0000115F2E01F0779F52091F5093091F6095A
:10FBC0004091F7095091F809621773078407950768
:10FBD00019F421C0C5012CC09401AB01BC01809176
:10FBE000F3079091F4070E94936E882309F43CCFA9
:10FBF000800E911EEB81FC8180859185A285B38565
:10FC0000800F911FA11DB11D80879187A287B387A7
:10FC1000E01AF10A51CF40E02BD9882309F424CF10
:10FC2000B6016B50784FA801C4010F94DC1BE0CFE4
:10FC30000F900F900F900F90DF91CF911F910F9128
:10FC4000FF90EF90DF90CF90BF90AF909F908F90FC
:10FC50007F906F905F904F903F902F900895CF933B
:10FC6000DF931F92CDB7DEB741E050E0BE016F5F7A
:10FC70007F4FDBDE019719F4898190E002C08FEF9E
:10FC80009FEF0F90DF91CF910895DF92EF92FF9257
:10FC90000F931F93CF93DF93FC012381223060F0F9
:10FCA00000851185228533850F711127222733277F
:10FCB000012B022B032B11F08FEF5DC04115510575
:10FCC00011F0FA0110827A01EB018C018DE0D82E3F
:10FCD00040E250E0BE01C801A8DE8032910539F053
:10FCE00021E0892B09F420E0822F819544C02881EE
:10FCF0002223C9F1253E11F02E3231F4E114F10432
:10FD000039F3F7011082E4CFE114F10441F13B85AE
:10FD10003F733F3021F54A8D5B8D452B01F52F71E7
:10FD20003FEF320F3530D8F430E021503109D29E08
:10FD3000C001D39E900D1124D701A80FB91FFE0159
:10FD400020E0AD01253088F431813D932F5F32965C
:10FD50002D30C1F7288126FF02C0FA0115862B85B8
:10FD600023FDB6CF08C080E006C02B3010F43481EC
:10FD7000ECCF3681EACFDF91CF911F910F91FF90A9
:10FD8000EF90DF9008951F93CF93DF93FC012381C1
:10FD9000223018F480E090E023C0EC0140855185CA
:10FDA0006285738585E076956795579547958A9521
:10FDB000D1F7142F1F70CF0152DF97FDEBCF88854D
:10FDC0009985AA85BB854F96A11DB11D8887998706
:10FDD000AA87BB87F0E21F9FC00111248B50984F68
:10FDE000DF91CF911F9108958F929F92AF92BF9212
:10FDF000CF92DF92EF92FF920F931F93CF93DF93F7
:10FE0000EC018B81811102C080E077C009891A89D9
:10FE10002B893C890417150726073707A8F36A01C1
:10FE20007B01823029F4C886D986EA86FB860DC01C
:10FE3000C114D104E104F10451F4188619861A861C
:10FE40001B861C821D821E821F8281E056C0888410
:10FE50009984AA84BB84E98DFA8D258530E0275FDB
:10FE60003F4FB501A4014150510961097109022EAA
:10FE700004C076956795579547950A94D2F7D701B0
:10FE8000C6010197A109B10904C0B695A795979538
:10FE900087952A95D2F784179507A607B70720F00C
:10FEA00089288A288B2849F44D895E896F89788D45
:10FEB0004C835D836E837F8304C0841B950BA60BEC
:10FEC000B70B4C015D018E010C5F1F4F8114910433
:10FED000A104B10409F4A7CF4C815D816E817F81BB
:10FEE0009801898D9A8D0E94707791E0891A910806
:10FEF000A108B1088111EACF87CFDF91CF911F917F
:10FF00000F91FF90EF90DF90CF90BF90AF909F90B8
:10FF10008F9008950F931F93CF93DF93EC018B8104
:10FF20008823D9F1898187FF32C061E0CE0197DC57
:10FF30008C01009791F1FC018081853E71F18B81EC
:10FF4000823040F489899A89AB89BC89848F958FE6
:10FF5000A68FB78F8D899E89AF89B88DF801938F51
:10FF6000828FB58BA48BE091F909F091FA09309753
:10FF700059F0B8016A5E7F4FC80148961995F8019B
:10FF8000808D918D938B828B89818F778983DF918F
:10FF9000CF911F910F910C94F87681E0888380E0D7
:10FFA000DF91CF911F910F910895CF93DF93EC01D3
:10FFB000B1DF1B82DF91CF9108954F925F926F92D4
:10FFC0007F928F929F92AF92BF92EF92FF920F9388
:10FFD0001F93CF93DF9300D01F92CDB7DEB7FC0104
:10FFE00083818130E1F4818181FF19C08189928907
:10FFF000A389B48984179507A607B70780F0892BD2
:020000021000EC
:100000008A2B8B2B09F474C04A015B017F01408469
:10001000518462847384CF01E7DE811102C080E0E5
:1000200068C0F701818D928D81149104A104B104FF
:1000300069F4458956896789708DD2D9882379F307
:10004000F701158A168A178A108E39C0F701448184
:100050005581668177819E012F5F3F4F0E947077A7
:100060008823E9F249815A816B817C81F701818D76
:10007000928DFC012789203139F4483FFFEF5F075B
:1000800061057105E0F407C0483F2FEF5207620792
:100090002FE07207A0F4A4D9882309F4C0CFF70198
:1000A00044815581668177810FEF1FEF2FEF3FE08D
:1000B000818D928D0E945678882309F4B0CFF70184
:1000C000818A928AA38AB48A818180688183C701E8
:1000D00021DF882309F4A3CFB501A40148145904F2
:1000E0006A047B0410F4B301A201C7017DDE01C0E4
:1000F00081E00F900F900F900F90DF91CF911F91A3
:100100000F91FF90EF90BF90AF909F908F907F9056
:100110006F905F904F9008951F93CF93DF93EC0102
:10012000142F80E2689FF00111249F012B50384F5B
:10013000D9011B968C91817121F0842F827109F075
:1001400057C08091F5099091F609A091F709B091F7
:10015000F8098C879D87AE87BF87688BEB50F84F77
:100160004489558960E070E0BA01552744274D8BDA
:100170005E8B6F8B788F828D938DA0E0B0E0482BE3
:10018000592B6A2B7B2B4D8B5E8B6F8B788FD90114
:100190001B968C91887151F4848D958DA68DB78DA9
:1001A000898B9A8BAB8BBC8B81E00CC0803101F5C5
:1001B0009E012F5E3F4F898D9A8D0E94F077882394
:1001C000B9F084E08B83812F8F7089831C821D821C
:1001D0001E821F82188619861A861B8614FF0BC082
:1001E00040E050E0BA01CE01E8DE811104C00FC04A
:1001F0001B8280E00CC015FF09C049895A896B89B0
:100200007C89CE01DF91CF911F91EECD81E0DF910E
:10021000CF911F910895BF92CF92DF92EF92FF92FC
:100220000F931F93CF93DF938C01EB016A01E22EB2
:10023000898D9A8DF801928F818F40E050E0BA014C
:10024000CE01D2DDF12C88859985AA85BB854989A7
:100250005A896B897C8984179507A607B707C0F56B
:1002600025E0B695A795979587952A95D1F7F82F0C
:10027000FF70BF2ECE0187DDDC01892B09F486C01B
:100280008C91882319F0853EB9F47DC0F1100EC021
:100290004091F5095091F6096091F7097091F809BC
:1002A000F8014487558766877787B08A8C918823C1
:1002B00069F0FF24F394C7CF4BE050E0BD01C601C5
:1002C0000F94CF1B892B09F0BECF5AC0FF24F394A3
:1002D0008E2D8274823409F059C0FF2049F0F80154
:1002E000B08861E0C801BBDAEC01892B69F44EC02B
:1002F0008B81823009F44AC0CE012ADA882309F4BE
:1003000045C0C5EFD7E0B12C80E2FE0111928A957D
:10031000E9F78BE0F601DE0101900D928A95E1F795
:10032000E091F909F091FA09309739F0BE01625F66
:100330007F4FCE014096199508C081E298E2998BD3
:10034000888B80E098E09F878E87888999899B8B2E
:100350008A8B998F888F8E859F859F8B8E8B0E942D
:10036000F876882399F04E2D6B2DC801DF91CF913F
:100370001F910F91FF90EF90DF90CF90BF90CCCE68
:10038000E7FEF1CF03C0F11094CF82CF80E0DF9180
:10039000CF911F910F91FF90EF90DF90CF90BF9082
:1003A00008953F924F925F926F927F928F929F92A9
:1003B000AF92BF92CF92DF92EF92FF920F931F9373
:1003C000CF93DF93CDB7DEB7C354D1090FB6F894FE
:1003D000DEBF0FBECDBF5C016B0124965FAF4EAF99
:1003E0002497522E1C8E1F8E19821C826115710556
:1003F00011F410E074C0FC0183818111FACF2496BE
:10040000EEADFFAD249780818F32F1F4F601838148
:100410008250823058F0618D728DCE010196B3DA30
:10042000882339F38E010F5F1F4F01C08601249688
:10043000EEADFFAD249780818F3239F4319624964A
:10044000FFAFEEAF2497F3CF8B017E01FCE1EF0EFF
:10045000F11C3701CE0101964C014E2C3F2CAE0110
:100460004E5B5F4FBE01695C7F4F24968EAD9FADA2
:10047000249748DA882309F4BCCF2496EEADFFAD6B
:10048000249780818F3231F431962496FFAFEEAFFE
:100490002497F3CF8823D9F021E0AE01495C5F4F68
:1004A000B801C701B8DE882309F4A3CF0C151D05D8
:1004B00011F0C8017ADDE614F70431F0942D832D94
:1004C0008701E92EF82ECBCF982D892DF9CF252D38
:1004D000AE01495C5F4FB801C5019DDE182FCE010A
:1004E00001960E94346FCE014C960E94346F812F8A
:1004F000CD5BDF4F0FB6F894DEBF0FBECDBFDF91EF
:10050000CF911F910F91FF90EF90DF90CF90BF9010
:10051000AF909F908F907F906F905F904F903F90A3
:100520000895CF93DF93EC0140E050E0BA0145DD40
:10053000882369F061E0CE0192D9009741F025EE61
:10054000FC0120831B82DF91CF910C94F87680E030
:10055000DF91CF9108951F93CF93DF93CDB7DEB78F
:100560006B970FB6F894DEBF0FBECDBFAB011982FB
:100570001C8222E0BC01CE01019613DF182F8823D4
:1005800021F0CE010196CDDF182FCE0101960E94F9
:10059000346F812F6B960FB6F894DEBF0FBECDBFC0
:1005A000DF91CF911F9108952F923F924F925F92CA
:1005B0006F927F928F929F92AF92BF92CF92DF9273
:1005C000EF92FF920F931F93CF93DF9300D01F9270
:1005D000CDB7DEB78C014B013A01DC0113968C914B
:1005E00013978130C1F411968C9181FF14C082FF62
:1005F00018C0F80141895289638974898085918581
:10060000A285B38584179507A607B70751F0C801DF
:10061000EBDB811106C081E0D8018C938FEF9FEF57
:100620003CC1530184C0D80159968D919C915A9731
:10063000FC0154805A946A017B0129E0F694E79406
:10064000D794C7942A95D1F75C207A01F1E0FF2274
:10065000552009F478C080E092E08E199F09650169
:100660008A159B0508F46C01D80159962D913C918F
:100670005A9714968D919D910D90BC91A02D029743
:10068000A109B109F901058404C0880F991FAA1FA7
:10069000BB1F0A94D2F74685578560897189840FFC
:1006A000951FA61FB71F9C01AD01250D311D411DD2
:1006B000511D19012A01C11432E0D30609F08AC084
:1006C0008091F5099091F609A091F709B091F80988
:1006D00082159305A405B50569F41092F2078FEF12
:1006E0009FEFDC018093F5099093F609A093F70939
:1006F000B093F8099401B201A1018091F3079091A0
:10070000F4070E94DB6E882309F485CFF801808509
:100710009185A285B3858C0D9D1DA11DB11D80877E
:100720009187A287B3878C0C9D1CAC18BD08D8019B
:1007300018964D915D916D917C911B97A114B10418
:1007400009F071CF7DC0E114F10409F084CF149653
:100750004D915D916D917C91179741155105610502
:10076000710559F455968D919D910D90BC91A02DD8
:100770000097A105B10541F521C09E012F5F3F4FB4
:100780000E947077882309F446CF89819A81AB81D2
:10079000BC81F801218D328DF9012789203139F48E
:1007A000883FFFEF9F07A105B10540F40DC0883FCA
:1007B0002FEF9207A2072FE0B20730F0C8010E9486
:1007C000837B811148CF27CFF80184839583A6834B
:1007D000B78341CFE114F10419F5D80118964D9172
:1007E0005D916D917C911B9751968D919D910D908E
:1007F000BC91A02D481759076A077B0788F00E9413
:10080000F876882309F407CF81E08093F2072092DD
:10081000F5093092F6094092F7095092F80908C09C
:1008200041E0C201B1010E943877882309F4F3CE78
:10083000A601B401C7018B50984F0F94DC1B66CF03
:100840005196CD90DD90ED90FC90549711968C913F
:10085000C416D506E606F70640F4F801418B528B24
:10086000638B748B806881830DC02091F90930916E
:10087000FA09232B39F06114710421F08068D80142
:1008800011968C93F801818183FD02C0C30105C0DC
:10089000C80140DB8111FACFBECE0F900F900F90B0
:1008A0000F90DF91CF911F910F91FF90EF90DF900C
:1008B000CF90BF90AF909F908F907F906F905F9000
:1008C0004F903F902F900895FB0101900020E9F791
:1008D0003197AF01461B570B67CE08950895CF920D
:1008E000DF92EF92FF926B017C0183E3C816D10483
:1008F000E104F10470F082E3C81AD108E108F108BC
:1009000062E370E080E090E00E9495280E94E09B06
:10091000ECCFC701B6010E949528FF90EF90DF90C1
:10092000CF900C94E09BDC01FB01460F571FE417AE
:10093000F507C1F081912D913C911197382798E0EE
:10094000B901660F771F37FF06C09B0181E2282798
:1009500080E1382701C09B01915091F711963C939B
:100960002E93E5CF0895282F843640F064E60F9447
:1009700007176AE00F940717905D01C090E290930B
:10098000FF092A3048F03AE0822F632F0F940717AF
:100990000F940717905D01C090E29093000A822F98
:1009A0006AE00F940717905D9093010A8FEF99E02A
:1009B00008959C0197FD0EC08436910584F064E68D
:1009C00070E00F942717CB016AE070E00F942717AF
:1009D000805D06C03195219531098DE201C080E22C
:1009E0008093FF092A30310564F0EAE0F0E0C901A4
:1009F000BF010F942717CB01BF010F942717805D0C
:100A000001C080E28093000AC9016AE070E00F949F
:100A10002717805D8093010A8FEF99E00895AC015C
:100A2000952F991F9927991F29F022273327241BD7
:100A3000350B01C09A01483E5340ACF0C90168EE45
:100A400073E00F942717CB01EAE0F0E0BF010F94A9
:100A50002717805D8093FE09C90164E670E00F945A
:100A60002717CB0112C0243631050CF1911102C0B9
:100A700080E201C08DE28093FE09C90164E670E066
:100A80000F942717CB01EAE0F0E0BF010F9427177E
:100A9000805D8093FF09C901BF010F942717CB0127
:100AA000BF010F942717805D8093000A16C080E273
:100AB0008093FE098093FF092A3031053CF09111A3
:100AC0008DE28093FF09EAE0F0E0E5CF911102C0EA
:100AD00080E201C08DE28093000AC9016AE070E003
:100AE0000F942717805D8093010A8EEF99E0089597
:100AF0008F929F92AF92BF92CF92DF92EF92FF922E
:100B0000CF93FC01C080D180E280F38020E030E010
:100B10004AE754E4C701B6010F9432164B015C0159
:100B200020E030E0A901C701B6010F94F41387FD5E
:100B300005C020E030E040EA50E404C020E030E0AE
:100B400040EA50ECC501B4010F941B1320E030E0E3
:100B500040E251E40F94FB130F9463146B017C018A
:100B600097FD10C020E137E240E050E00F945C17A1
:100B7000CA01B9012AE030E040E050E00F945C1770
:100B8000605D09C0F094E094D094C094C11CD11C65
:100B9000E11CF11C6DE26093FC09C701B60128EE6F
:100BA00033E040E050E00F945C178AE0882E912CEF
:100BB000A12CB12CCA01B901A50194010F945C17B5
:100BC000605D6093FD09C701B60124E630E040E0B6
:100BD00050E00F945C17CA01B901A50194010F946C
:100BE0005C17605D6093FE098EE28093FF09C70188
:100BF000B601A50194010F945C17C62FCA01B90173
:100C0000A50194010F945C17605D6093000AC05DBC
:100C1000C093010A8CEF99E0CF91FF90EF90DF90A5
:100C2000CF90BF90AF909F908F9008958F929F929A
:100C3000AF92BF92CF92DF92EF92FF92FC01C08001
:100C4000D180E280F38020E030E048EC52E4C7013C
:100C5000B6010F9432164B015C0120E030E0A9018F
:100C6000C701B6010F94F41387FD05C020E030E002
:100C700040EA50E404C020E030E040EA50ECC50116
:100C8000B4010F941B1320E030E040E251E40F94D4
:100C9000FB130F9463149B0177FF06C022273327B1
:100CA000261B370B8DE201C08BE28093FC09C90142
:100CB00068EE73E00F942717CB01EAE0F0E0BF0184
:100CC0000F942717805D8093FD09C90164E670E0E9
:100CD0000F942717CB01BF010F942717805D8093D6
:100CE000FE09C901BF010F942717282FCB01BF01AF
:100CF0000F942717805D8093FF098EE28093000A8E
:100D0000205D2093010A8CEF99E0FF90EF90DF9037
:100D1000CF90BF90AF909F908F9008958F929F92A9
:100D2000AF92BF92CF92DF92EF92FF92CF93C62FF6
:100D3000FC01C080D180E280F38020E030E44CE10F
:100D400056E4C701B6010F9432164B015C0120E056
:100D500030E0A901C701B6010F94F41387FD05C067
:100D600020E030E040EA50E404C020E030E040EA17
:100D700050ECC501B4010F941B1320E030E040E2B9
:100D800051E40F94FB130F9463146B017C01611504
:100D900071058105910561F097FF0CC0F094E09416
:100DA000D094C094C11CD11CE11CF11C6DE203C0A5
:100DB00060E201C06C2F6093FC09C701B60128EE08
:100DC00033E040E050E00F945C178AE0882E912CCD
:100DD000A12CB12CCA01B901A50194010F945C1793
:100DE000605D6093FD098EE28093FE09C701B60144
:100DF00024E630E040E050E00F945C17CA01B901EE
:100E0000A50194010F945C17605D6093FF09C70111
:100E1000B601A50194010F945C17C62FCA01B90150
:100E2000A50194010F945C17605D6093000AC05D9A
:100E3000C093010A8CEF99E0CF91FF90EF90DF9083
:100E4000CF90BF90AF909F908F9008958F929F9278
:100E5000AF92BF92CF92DF92EF92FF92FC01C080DF
:100E6000D180E280F38020E030E0A901C701B60123
:100E70000F94F41387FF08C0C701B601905820E013
:100E800030E040E251E406C020E030E040E251E4CE
:100E9000C701B6010F94321620E030E040EA50E47A
:100EA0000F941B1320E030E040E251E40F94FB1359
:100EB0000F9463146B017C016031F7E27F078105B9
:100EC000910584F020E137E240E050E00F945C1798
:100ED000CA01B9012AE030E040E050E00F945C170D
:100EE000605D01C060E26093FD0988EEC81683E092
:100EF000D806E104F10494F0C701B60128EE33E00E
:100F000040E050E00F945C17CA01B9012AE030E0DC
:100F100040E050E00F945C17605D01C060E26093B8
:100F2000FE09E4E6CE16D104E104F10494F0C70111
:100F3000B60124E630E040E050E00F945C17CA01AF
:100F4000B9012AE030E040E050E00F945C17605DAA
:100F500001C060E26093FF09FAE0CF16D104E1041A
:100F6000F1049CF08AE0882E912CA12CB12CC701B1
:100F7000B601A50194010F945C17CA01B901A5013E
:100F800094010F945C17605D01C060E26093000AF9
:100F9000C701B6012AE030E040E050E00F945C1752
:100FA000605D6093010A8DEF99E0FF90EF90DF9014
:100FB000CF90BF90AF909F908F9008958F929F9207
:100FC000AF92BF92CF92DF92EF92FF92CF93FC014C
:100FD000C080D180E280F38020E030E04AE754E432
:100FE000C701B6010F9432164B015C0120E030E0DE
:100FF000A901C701B6010F94F41387FD05C020E0D5
:1010000030E040EA50E404C020E030E040EA50EC38
:10101000C501B4010F941B1320E030E040E251E41D
:101020000F94FB130F9463146B017C0197FF0AC0AC
:10103000F094E094D094C094C11CD11CE11CF11C2C
:101040008DE201C08BE28093FB09C701B60120E16C
:1010500037E240E050E00F945C178AE0882E912C34
:10106000A12CB12CCA01B901A50194010F945C1700
:10107000605D6093FC09C701B60128EE33E040E0F3
:1010800050E00F945C17CA01B901A50194010F94B7
:101090005C17605D6093FD09C701B60124E630E08E
:1010A00040E050E00F945C17CA01B901A50194011A
:1010B0000F945C17605D6093FE098EE28093FF09D8
:1010C000C701B601A50194010F945C17C62FCA0190
:1010D000B901A50194010F945C17605D6093000A4B
:1010E000C05DC093010A8BEF99E0CF91FF90EF9024
:1010F000DF90CF90BF90AF909F908F9008958F9288
:101100009F92AF92BF92CF92DF92EF92FF92CF93D6
:10111000FC01C080D180E280F38020E030E0A901B2
:10112000C701B6010F94F41387FF08C0C701B601C9
:10113000905820E030E04AE754E406C020E030E078
:101140004AE754E4C701B6010F94321620E030E0BC
:1011500040EA50E40F941B1320E030E040E251E4F9
:101160000F94FB130F9463146B017C01603AF6E853
:101170007F07F1E08F07910584F020EA36E841E02F
:1011800050E00F945C17CA01B9012AE030E040E05A
:1011900050E00F945C17605D01C060E26093FB0952
:1011A00080E1C81687E2D806E104F10494F0C70193
:1011B000B60120E137E240E050E00F945C17CA012D
:1011C000B9012AE030E040E050E00F945C17605D28
:1011D00001C060E26093FC09E8EECE16E3E0DE06B3
:1011E000E104F10494F0C701B60128EE33E040E0D9
:1011F00050E00F945C17CA01B9012AE030E040E0EA
:1012000050E00F945C17605D01C060E26093FD09DF
:10121000C701B60124E630E040E050E00F945C17CF
:101220008AE0882E912CA12CB12CCA01B901A5010C
:1012300094010F945C17605D6093FE098EE28093C9
:10124000FF09C701B601A50194010F945C17C62FD1
:10125000CA01B901A50194010F945C17605D609308
:10126000000AC05DC093010A8BEF99E0CF91FF9017
:10127000EF90DF90CF90BF90AF909F908F900895A8
:101280008F929F92AF92BF92CF92DF92EF92FF9296
:10129000FC01C080D180E280F38020E030E04AE7AA
:1012A00054E4C701B6010F9432164B015C0120E0F3
:1012B00030E0A901C701B6010F94F41387FD05C002
:1012C00020E030E040EA50E404C020E030E040EAB2
:1012D00050ECC501B4010F941B1320E030E040E254
:1012E00051E40F94FB130F9463146B017C0197FF7F
:1012F0000AC0F094E094D094C094C11CD11CE11CAD
:10130000F11C8DE201C080E28093FB09F0E1CF1671
:10131000F7E2DF06E104F10494F0C701B60120E131
:1013200037E240E050E00F945C17CA01B9012AE0AF
:1013300030E040E050E00F945C17605D01C060E277
:101340006093FC0988EEC81683E0D806E104F10436
:1013500094F0C701B60128EE33E040E050E00F946E
:101360005C17CA01B9012AE030E040E050E00F9478
:101370005C17605D01C060E26093FD09C701B601C2
:1013800024E630E040E050E00F945C178AE0882EBD
:10139000912CA12CB12CCA01B901A50194010F9483
:1013A0005C17605D6093FE09C701B601A501940159
:1013B0000F945C176B017C01672B682B692B89F0FC
:1013C0008EE28093FF09CA01B901A50194010F942F
:1013D0005C17605D6093000A80E38C0D8093010AC6
:1013E0001AC0CA01B901A50194010F945C176115D7
:1013F00071058105910539F02EE22093FF09605DAA
:101400006093000A05C080E28093000A8093FF0980
:1014100080E28093010A8BEF99E0FF90EF90DF90DC
:10142000CF90BF90AF909F908F900895CF93DF9310
:10143000FC018491EF012196882319F069D2FE0105
:10144000F8CFDF91CF9108958DE892E3EFCF83E954
:1014500092E3ECCF0F931F93CF93DF931F921F92D2
:10146000CDB7DEB769837A83E1DF6981062F7A81A0
:10147000172FF80181918F01882311F049D2F9CFFC
:101480000F900F90DF91CF911F910F910895CF93FF
:10149000DF93EB01CBDF6AE070E0CE01DF91CF910B
:1014A0002AC3CF92DF92EF92FF926A017B01BEDFE7
:1014B0004AE050E0C701B601FF90EF90DF90CF9077
:1014C00009C3CF92DF92EF92FF926A017B01AEDFF8
:1014D00042E050E0C701B601FF90EF90DF90CF905F
:1014E00097C3CF92DF92EF92FF926A017B019EDF5A
:1014F00042E050E0C701B601FF90EF90DF90CF903F
:1015000087C3CF93DF93EB0191DF6AE070E0CE01F8
:10151000DF91CF9105C3CF92DF92EF92FF926A01E4
:101520007B0184DF4AE050E0C701B601FF90EF90F5
:10153000DF90CF90EFC2811103C086E892E302C032
:101540008AE892E373CF0C941D6F81E0089581E0E7
:1015500008958F929F92AF92BF92CF92DF92EF92B7
:10156000FF920F931F93CF93DF931F921F92CDB7DC
:10157000DEB76C0159018B017B01E40EF51E0E15DF
:101580001F0561F1F60180809180F80161918F0162
:101590006983C4016A830F94411F6A81681779F0D7
:1015A000C4010F94491FC4010F94411F99818917E9
:1015B00031F04ADF8AE992E339DF81E010C041E08F
:1015C00050E0BE016F5F7F4FC501ADD9F60140818C
:1015D00051814F5F5F4F51834083D1CF80E00F90A7
:1015E0000F90DF91CF911F910F91FF90EF90DF90BF
:1015F000CF90BF90AF909F908F9008958F929F92C1
:10160000AF92BF92CF92DF92EF92FF920F93CF9360
:10161000DF931F92CDB7DEB75C016B017A01490100
:10162000F501808191810F94411F8983002311F07E
:10163000F601808341E050E0BE016F5F7F4FC4013F
:1016400072D9F501408151814F5F5F4F51834083D3
:10165000FFEFCF1ADF0A81E0E81AF10809F780E00E
:101660000F90DF91CF910F91FF90EF90DF90CF908F
:10167000BF90AF909F908F90089598E288E10FB649
:10168000F894A895809360000FBE90936000089531
:101690001F920F920FB60F9211240BB60F920F9359
:1016A0001F932F933F934F935F936F937F938F93EA
:1016B0009F93AF93BF93CF93DF93EF93FF930091EB
:1016C000290AD091280A11E01D0F1F77C091C6008A
:1016D0009091040A492F092E000C550B660B770BCD
:1016E0004C30510508F046C0FA018827EF55FF4FEE
:1016F0008F4F0D947817CD3441F0CE34B9F481E09A
:1017000005C0CA3330F0CD3471F582E08093040A0D
:101710004AC0C03308F047C0C03209F444C0CD32DB
:1017200011F541C0C13329F0C43329F0C032D9F4D6
:101730003AC083E0EBCF88E0E9CFC03321F0C1337A
:1017400091F486E0E3CF84E0E1CFC83361F485E033
:10175000DDCFC23341F487E0D9CFC13321F489E032
:10176000D5CFC03311F08BE0D1CF8AE0CFCFCA30D4
:10177000D1F417C0CA30B9F48091B30A882389F034
:10178000973049F09A3059F0953059F41092680228
:101790001092E91506C081E08093B40A02C00F944C
:1017A00019111092040A101731F0ED2FF0E0E85DE6
:1017B000F54FC283D12FD093280AFF91EF91DF918B
:1017C000CF91BF91AF919F918F917F916F915F91D9
:1017D0004F913F912F911F910F910F900BBE0F9042
:1017E0000FBE0F901F9018951F920F920FB60F9279
:1017F00011240BB60F922F938F939F93EF93FF9328
:101800008091070A2091060A281791F0E82FF0E04E
:10181000EA5FF54F92818F5F8F719093C60080933E
:10182000070A9091C00090649093C000281305C0EF
:101830008091C1008F7D8093C100FF91EF919F91B6
:101840008F912F910F900BBE0F900FBE0F901F9096
:1018500018959B01AC011092C000211581EE38074C
:1018600041055105C1F08091C00082608093C000A5
:1018700060E079E08DE390E00F945C17CA01B90154
:10188000615071098109910922E030E040E050E0A7
:101890000F945C1702C020E130E03093C500209324
:1018A000C4008091C10080618093C1008091C1001B
:1018B00088608093C1008091C10080688093C100DE
:1018C0008091C1008F7D8093C1001092050A089518
:1018D0008091280A9091290A891759F0E92FF0E0A0
:1018E000E85DF54F82819F5F9F779093290A90E092
:1018F00008958FEF9FEF0895E8E2FAE080818183F9
:101900000895E8E2FAE080819181891B8F7708953C
:1019100091E09093050A9091C10095FD04C09091CB
:10192000C00095FD40C02091060A2F5F2F710FB6B1
:1019300007FC34C09091070A291322C09091C0007F
:1019400095FF1DC09091070A4091060A491791F032
:10195000E92FF0E0EA5FF54F32819F5F9F7130938E
:10196000C6009093070A3091C00030643093C000E5
:10197000491305C09091C1009F7D9093C100DACFBB
:10198000E091060AF0E0EA5FF54F82832093060AB1
:101990008091C10080628093C10008959091070AF0
:1019A0002913EECFFBCF8093C6008091C0008064E6
:1019B0008093C00008958DE0ABDF8AE0A9CFCF937C
:1019C000DF93EC018991882311F0A2DFFBCFDF9137
:1019D000CF91F1CF8F929F92AF92BF92EF92FF92F1
:1019E0001F93CF93DF93CDB7DEB7A0970FB6F894D0
:1019F000DEBF0FBECDBF611571058105910579F17F
:101A000010E0842E912CA12CB12CEE24E394F12C27
:101A1000EC0EFD1EE10EF11C17FDFA94A5019401D8
:101A20000F943A17F7016083B901CA011F5F61156E
:101A300071058105910549F7115010F1E1E0F0E0E1
:101A4000EC0FFD1FE10FF11D17FDFA9580818A3023
:101A500010F097E301C090E3890F5ADFEDCF80E3E8
:101A6000A0960FB6F894DEBF0FBECDBFDF91CF9129
:101A70001F91FF90EF90BF90AF909F908F9048CFB5
:101A8000A0960FB6F894DEBF0FBECDBFDF91CF9109
:101A90001F91FF90EF90BF90AF909F908F9008950F
:101AA000CF92DF92EF92FF926B017C0197FF0AC009
:101AB0008DE22EDFF094E094D094C094C11CD11C30
:101AC000E11CF11C4AE0C701B601FF90EF90DF90E6
:101AD000CF9080CF4115510511F4862F19CF4A3090
:101AE000510509F4DDCF76CFAB01682F880F770B56
:101AF000880B990BEFCFAB01BC01990F880B990BA9
:101B0000E9CFAB01BC01990F880B990BE3DF53CFF1
:101B1000E1DF51CF4115510511F4862FF9CE5ACF8F
:101B2000AB01BC0180E090E0F5CFF4DF44CF8F92B1
:101B30009F92AF92BF92CF92DF92EF92FF92CF939C
:101B40006B017C01B42E20E030E0A9010F94F41366
:101B500087FF06C08DE2DCDEF7FAF094F7F8F09428
:101B6000C0E060E070E080E09FE3CB1541F02DEC39
:101B70003CEC4CEC5DE30F943216CF5FF6CF9B014B
:101B8000AC01C701B6010F941B136B017C010F94CC
:101B900068144B015C014AE01DDFCC2379F1C501DB
:101BA000B4010F9494149B01AC01C701B6010F94CA
:101BB0001A136B017C018EE2ABDE20E030E040E2E4
:101BC00051E4C701B6010F9432164B015C010F942A
:101BD00063146B01770FEE08FF08C701B60160DFE1
:101BE000C701B6010F9496149B01AC01C501B40165
:101BF0000F941A136B017C01C150F9F6CF91FF903D
:101C0000EF90DF90CF90BF90AF909F908F9008950E
